:020000040000FA
:06000000DCEFB8F0120075
:0600080046EFB4F0120007
:0600180054EFB4F01200E9
:06002A002DEC08F0146843
:10003000156AFD0EDBCF08F0FE0EDBCF09F014C011
:100040000DF015C00EF0C6ECB8F008C0DEFF09C018
:10005000DDFF63EC07F0EE50ED1009E0E66AAFEC6F
:10006000B8F0E552DF06010EF4E2DB06F2D723EC2E
:1000700007F00D680E6A14C008F015C009F0C6EC50
:10008000B8F004C014F005C015F004C0DEFF05C0D0
:10009000DDFF63EC07F0EE50ED1005E0DFCFE6FF8B
:1000A000AFECB8F0E552020EE15C02E2E16AE55223
:1000B000E16E3DEF06F0010ED16E1200D16A120022
:1000C0000501505101E1040012000501010E506FBD
:1000D000120002EC08F0D3EC07F0FB0EDBCFEEFFD2
:1000E000FC0EDBCFEDFFDF5001E09D80E5523DEFE0
:1000F00006F038EC06F0030EE1263AEC08F0EDCFFE
:10010000DBFFDF5001E09D8091EC07F09FEC07F0F2
:10011000030EE15C02E2E16AE552E16E3DEF06F0BA
:1001200002EC08F0D3EC07F0F90EDBCFEEFFFA0E8D
:10013000DBCFEEFFFB0EDBCFEEFFFC0EDBCFEEFFE7
:10014000DF5001E09D80E5523DEF06F031EC08F014
:100150003AEC08F0EECFDBFF030EEECFDBFF040E30
:10016000EECFDBFFDF5001E09D8091EC07F0030E46
:10017000DBCF16F0040EDBCF17F014C006F015C06D
:1001800007F016C008F017C009F0050EE15C02E2A6
:10019000E16AE552E16E3DEF06F00501806B80C536
:1001A0007FF580C569F580C568F5120002EC08F09E
:1001B00005016829DF6E070EDF5C01E3DF6A695124
:1001C000DF5C02E1010E2ED06851C3EC06F098EC22
:1001D00007F06851C3EC06F083EC07F0DFCF68F559
:1001E00023EC07F0000E1416F00E1516145002E161
:1001F000200E15180FE0FD0EDBCF16F0FE0EDBCF44
:1002000017F0000E1616F00E171616500AE1100E13
:10021000171807E1FD0EDB50010B03E10901010E88
:10022000056F000EE5523DEF06F038EC06F00501D3
:100230006951685D02E1010E10D06951C3EC06F00E
:1002400005EC08F06951C3EC06F010EC07F0692BDF
:10025000070E695D01E3696B000E3DEF06F002ECED
:1002600008F005017F29DF6E070EDF5C01E3DF6A1E
:100270008051DF5C02E1010E0DD07F51CDEC06F024
:1002800098EC07F07F51CDEC06F083EC07F0DFCF60
:100290007FF5000EE5523DEF06F038EC06F0050163
:1002A00080517F5D02E1010E10D08051CDEC06F04F
:1002B00005EC08F08051CDEC06F010EC07F0802B37
:1002C000070E805D01E3806B000E3DEF06F031EC20
:1002D00008F027DB000970E146EC07F0A6DFFAEC36
:1002E00007F0000969E174EC07F006E248EC06F05B
:1002F000A7DAFAEC07F060D0010EDB50C00B2BE060
:10030000AEEC06F0DBCF64F3040EDBCF65F3010E39
:10031000DB50800B0DE08CEC06F0F5CF63F30301AE
:10032000676B686B04C966F36A6B6B6B696B07D0AC
:100330000301C80E636F010E676F686B666B020E78
:10034000DBCF1AFDDBCF5CFD81EC06F09D900D014B
:1003500036899D8031D06DEC07F015E1100E15182F
:1003600012E1020EDBCFE6FF03C9E6FF02C9E6FF9A
:1003700013EC08F0D890E936EA36E806FBE1F6EC33
:1003800006F01AE117D06DEC07F016E1200E1518F3
:1003900013E1020EDBCFE6FF01C9E6FF00C9E6FF6D
:1003A00013EC08F0D890E936EA36E806FBE1F6EC03
:1003B00006F002E10901056B050EE15C02E2E16A6B
:1003C000E552E16E3DEF06F031EC08F0B4DA0009D9
:1003D00032E146EC07F061DFFAEC07F000092BE1AF
:1003E00074EC07F006E248EC06F05BDAFAEC07F092
:1003F00022D0010EDB50800B1EE0AEEC06F0DBCF0E
:1004000065F2040EDBCF66F28CEC06F0F5CF64F2F9
:100410000201686B696B04C967F26B6B6C6B6A6B8A
:10042000020EDBCF1CFDDBCF5EFD81EC06F09D9064
:100430000D01368D9D80050EE15C02E2E16AE55218
:10044000E16E3DEF06F038EC06F0FE0EDB50200AC0
:1004500001E17FD0290A01E17CD0530A70E00E0A45
:1004600064E0770A5AE0670A50E0070A4BE0010AA5
:1004700046E0030A41E06B0A37E01A0A2DE0090A58
:1004800028E0010A23E00F0A1EE0010A19E0030A2E
:1004900014E0010A0FE0070A0AE0010A05E0030A76
:1004A00060E1FFEC07F022D0FFEC07F017D0FFEC83
:1004B00007F035D0E5EC07F019D0E5EC07F00ED0E9
:1004C000E5EC07F02CD0EAEC07F010D0EAEC07F0EE
:1004D00005D0EAEC07F023D0EFEC07F0A1EC06F032
:1004E000060EEE6E230E43D0EFEC07F0A1EC06F003
:1004F000B10EEE6E1F0E3BD0FFEC07F008D0E5EC1E
:1005000007F005D0EAEC07F002D0EFEC07F0A1EC21
:1005100006F0CF0EEE6E2A0E2AD0EFEC07F0A1EC1B
:1005200006F0B80EEE6E260E22D09BDB2D0EEE6E80
:10053000090EA1EC06F0890EEE6E0B0E18D091DBC1
:10054000950EEE6E0C0EA1EC06F0410EEE6E100E46
:100550000ED087DBEE6AED6A20EC08F0EE6AED6AF9
:1005600007D0FFEC07F0EDDB450EEE6E120EED6EE0
:1005700084D37EDB040EE12623EC07F014C0DFFFFA
:10058000010E15C0DBFF020EDB6A030EDB6A63ECB3
:1005900007F0FD0E0B6EB50E0C6E060E0D6E0E6A9C
:1005A000EECF06F0EECF07F0EECF08F0EFCF09F078
:1005B0005EECB8F005C0EDFF04C0EDFF03C0EDFF39
:1005C00002C0EFFF63EC07F0EE52800EEE26000E45
:1005D000EE22EE2263EC07F0A4EC07F0EECF16F06B
:1005E000EFCF17F0100ED8901732163215321432A2
:1005F000E806F9E19FEC07F0040EE15C02E2E16A33
:10060000E552E16E3AD302EC08F0050EF36EFE0EF1
:10061000DBCFF4FFF350F45C05E2050EF36EFE0E43
:10062000F3CFDBFFFE0EDB50166E176AFE0EDB50BB
:100630007AEC07F014C008F015C009F016C00DF0F0
:1006400017C00EF0C6ECB8F00850DF6EDFCF37FDF4
:100650000D013751E8240D01386F030E0D013703EA
:10066000F3CF39FD040E3703F3CF3AFDDF507AECB8
:1006700007F014C009F0DFCF0EF00AECB9F0095012
:10068000E552FBD2F5DAF4EC07F0F3CF51F5F4CFF5
:1006900052F5F3D2EDDA040EE1269D900D0136916C
:1006A0009D800D01320E496F060E4A6F020E49CD34
:1006B000DBFF030E4ACDDBFFDF6ADF6ADF50D9ECD8
:1006C00007F0EF503CE0310EDF5C39E2DF50D9EC4F
:1006D00007F0EF507F0BE76E010EE7CFDBFFDBCFBC
:1006E00014F05F0EE76E1418E8AE02D0143403D095
:1006F000E750D88014540AE2200E146E010EDBCFAE
:10070000E7FF1450E75E010EE7CFDBFF5A0E146ED1
:10071000470E156E010E166E010EDBCF17F0186A2C
:10072000196A17AE02D018681968C4EC07F0F550C2
:10073000E66E90DBE552E750EF6EDF2ABFD78ADB2B
:10074000EF6A0D014B6B51C518FD52C519FD9D9007
:100750003F0E0D0111170D0136819D80040EE15CE5
:1007600002E2E16AE552E16E88D20CEC08F085D233
:100770000CEC08F00D0136B1FDD77FD29D900D0134
:1007800036910D01119D9D801200400E0D01111535
:10079000146E010E0D0136151410120002EC08F053
:1007A000DF6AD2DA0800F55010E0F90EDB50DF5CAA
:1007B0000CE2D3DBD950FD0FACDBEF22D950FA0F9E
:1007C000A8DBEE22EE22DF2AECD7C7DBE55255D2BA
:1007D0004FDAFE0EDB50040A32E0070A1CE0010A81
:1007E0000EE0030A2CE19D900D0136990D01119147
:1007F000DEDA630EE66E030E38DB83DA20D09D90DE
:100800000D01369B0D011195D2DA000EE66E030E36
:100810002CDBE1DA14D09D900D01369D0D0111996C
:10082000C6DA640EE66E020E20DB0D01640E506F18
:10083000020E516F0D01640E586F020E596F1DD2DA
:10084000E1DBDF6A4FD853DA37DB09E050DADEDA72
:10085000010EF4DADBCF1AFDDBCF5CFDDF88AEDB07
:100860002BDB18E0ABDB0900F5500900F5CFE7FF03
:100870000800F5CFF8FFE7CFF7FFF66E0800F55058
:1008800009E09CDBC3DA020ED9DADBCF1BFDDBCF3C
:100890005DFDDF8A9D90DF500D0136139D80E5528E
:1008A000ECD1E6D937D823DA07DB0CE020DAAEDA70
:1008B000030EC4DADBCF1CFDDBCF5EFD9D900D0186
:1008C000368D9D80DAD1D4D90DD88EDBF3CF12FDD1
:1008D000F4CF13FDFC0EDBCF1AFD9D900D011181AD
:1008E0009D80CBD19D90CF0E0D013617FA0E0D01D4
:1008F00011179D801200BCD90DD876DBF3CF16FD01
:10090000F4CF17FDFC0EDBCF1CFD9D900D0111896E
:100910009D80B3D19D900D01369D0D0111999D8053
:100920001200300E0D01361505E1050E0D011115F1
:1009300001E1000C010C400E0D01361505E1100E11
:100940000D01111501E1000C010C5CDBCBDF3CDA81
:1009500066ECABF0E552E552110EF35C000EF45874
:1009600003E3100E26DBEF6A0D01630E4C6F030EDE
:100970004D6F0D01000E4E6F030E4F6FFD0EDBCF5E
:10098000E9FFDB2AFE0EDBCFEAFF01E3DB2AEFCF34
:10099000DFFFDF5028E070DAFC0E59DB72DAEE522E
:1009A000E9CF14F0EACF15F0E9CFE6FFEACFE6FF92
:1009B00063DAEE52E9CF16F0EACF17F0E9CFE6FF9F
:1009C000EACFE6FFDFCFE6FF3EDD186E050EE15E03
:1009D000185067DA51DAFB0E3ADB2CDBEE52EE6A86
:1009E000ED6A5FDACBD748DAEF6A24DBEF6A49DADF
:1009F000EE52EE6AED6A85D9EED9FA0EDBCF1BFD19
:100A00001BCD1AFDDBCF5DFD5DCD5CFD9D90300EF5
:100A10000D0136139D80E55230D12AD963DF140EC3
:100A2000E66E0D0EE66E120EE66E0D0EE66EFE0E14
:100A3000DBCFE6FF08DD146E050EE15E14509D90DD
:100A4000050E0D0111139D8018D14CDF0301640EBA
:100A5000636F0301006F0301950E646F0C0E656FE9
:100A60000301410E016F100E026F0301640E666FE9
:100A70000301036F0301676B686B0301046B056B74
:100A80000301696B0301066B010E03016A6F6B6B57
:100A90000301076F086B35D99ED99D90300E0D016B
:100AA00036139D801200300E0D0136151200400ED7
:100AB0000D013615120005016951685D01E1000C58
:100AC000010C050180517F5D01E1000C010C9ADAF7
:100AD000FE0EDBCFE6FFE66AC3EC17F0E552E55207
:100AE000F350F41004E0FE0EDB50D00F04D0FE0EE5
:100AF000DB50BF0F0A0FDF6EDF50E552BED0ADDA1C
:100B0000FD0EDBCFDEFFDBCFDDFFE2D9EF5005E0EE
:100B1000DF2A010EFAE3DB2AF8D7DAD9FC0EDBCFA5
:100B2000EFFFD6D9010EACDAEF6A8DD908DA020EE2
:100B3000E15C02E2E16AE552E16E9FD09D929F8204
:100B4000D08EF90E94160F0EBD6EBA6E1C0ECA6EC4
:100B5000CB680D01116B0D017F0E1E6F0D011A6F19
:100B60000D011B6F0D011C6F0D011D6F0D01370E67
:100B7000126F1A0E136F0D01370E146F1A0E156FC8
:100B80000D01370E166F1A0E176F0D01370E186F05
:100B90001A0E196F1200810ECD6E9F90140EE66E24
:100BA00032DDE552E80EE66E030EE66E6BDDE552D1
:100BB000E5520D017F0E5F6F5FCD5EFD5FCD5DFD88
:100BC0005FCD5CFD0D01366B0D013B6B1200870E96
:100BD000D56EB16AF18EF26A9D6AA06AAFDFCBEF83
:100BE00005F046D8AA6AFE0EDB50A96EA69EA69C0A
:100BF000A680A85042D031DAA198AA6AFE0EDB5036
:100C0000A96EFD0EDB50A86EA69EA69CA684F2508F
:100C1000800B01E0010EDF6EF250400B01E0010E8F
:100C2000E76E010EE7CFDBFFF29EF29C550EA76E3A
:100C3000AA0EA76EA682DF50E8B0F28EE8A0F29E60
:100C4000010EDB50E8B0F28CE8A0F29CA1A8FED720
:100C5000A198A694020EE15C02E2E16AE552E16E1F
:100C60000CD0FC0EDBCFE9FFFD0EDBCFEAFF12005C
:100C7000D9CFE6FFE1CFD9FF1200E552E7CFD9FF88
:100C80001200FD0EDBCFE9FFFE0EDBCFEAFF120004
:100C9000020EDBCFE6FF710E176E4B0E186E010EC3
:100CA000196EDECF1AF0DDCF1BF01C6A060E0C6E3B
:100CB0000D6A0E6A1AC007F01BC008F01CC009F0CC
:100CC0002FECB5F004C01AF005C01BF006C01CF0F4
:100CD00017500424146E18500520156E1950062064
:100CE000166E14C0E6FF15C0E6FFE66E1200FC0E9D
:100CF000DBCFF6FFFD0EDBCFF7FFFE0EDBCFF8FFFD
:100D000012000D01630E4C6F030E4D6F0D01630E4B
:100D1000546F030E556F1200C70E146E4C0E156EF5
:100D2000010E166EDECF17F0DDCF18F01838186AF6
:100D30000F0B176E070E1716000E1816196AC4EF60
:100D400007F0ED6E20EF08F0FA0EDBCFF6FFFB0E9A
:100D5000DBCFF7FFFC0EDBCFF8FF120086D9FF0ECA
:100D600014160F0E151614C0E6FF15C0E6FFB9ECF9
:100D700002F0E552E552030EF3CFDBFF040EF4CF91
:100D8000DBFF030E1200030DF3CFE9FFF4CFEAFF00
:100D9000530EE926050EEA221200030DF3CFE9FFF8
:100DA000F4CFEAFF6A0EE926050EEA2212009D80C2
:100DB000210EE66EFB0EDBCFE6FFFC0EDBCFE6FF7F
:100DC000FD0EDBCFE6FF1200FD0EDBCFE6FFFE0ED1
:100DD000DBCFE6FF12000D01000E4E6F030E4F6FCA
:100DE0000D01000E566F030E576F1200060EE92616
:100DF000090EEA22EECFE6FFEFCFE6FFA6DD146E86
:100E0000050EE15E1450DF50010B12000900F5CF12
:100E1000E6FF0900F5CFE6FF0800F5CFE6FF120078
:100E2000020E2ED9EF50E66EFB0EDBCFE9FFFC0E73
:100E3000DBCFEAFFE552E750EF6E1200E66EC8DC4A
:100E4000D9D8FB0E1200FD0EDBCF14F0FE0EDBCF67
:100E500015F01200DF50E76E020EDBCFE9FF030E44
:100E6000DBCFEAFFE75040EF08F0E66E97DC146E48
:100E7000060EE15E145012004CCDE9FF4DCDEAFFA5
:100E800012004ECDE9FF4FCDEAFF1200D950020FFC
:100E9000E66E000EDA20E66ED9CFE6FFDACFE6FF87
:100EA00012000D01030E4C27000E4D230D01030E01
:100EB0004E27000E4F2312000900F5500900F510CF
:100EC0000800F5101200D9CFE9FFDACFEAFF1200CF
:100ED000DECFE9FFDDCFEAFF1200C7D8000E1416FF
:100EE000F00E151614501200C0D8390E145C000E06
:100EF00015581200156AE8307F0B146EF00E142698
:100F0000000E15221200020EBBD8FC0EDBCFEFFF45
:100F10001200E96EFF0EDA20EA6E030EEE26000ED6
:100F20001200010EDBCF14F0020EDBCF15F0120021
:100F3000FD0EDBCFEEFFFE0EDBCFEDFF120014C087
:100F4000F3FF15C0F4FF1200EECF14F0EECF15F052
:100F50001200450EEE6E120E1200F6DE0800F5507D
:100F6000E66E8FDEE552E750EF6EEEDE0900090017
:100F7000F5CF15F00800F5CF16F083DEEE5215C060
:100F8000EEFF16C0EDFF120014501724F36E15503B
:100F90001820F46E16501920F86EF4CFF7FFF3CF37
:100FA000F6FF080012009D50010BDF6E9D9041EF8F
:100FB00006F0E76E66DEE75040EF08F098DE030EBD
:100FC000F626000EF722F82212004BDE2F0EEE6EF0
:100FD000140E120046DE560EEE6E160E120041DEA4
:100FE000AB0EEE6E180E1200EFDEB9EC02F0E55219
:100FF000E5521200E552E552E552E552120031DEAB
:10100000A9EF07F035DEE65212009EDF3ADE14C08B
:10101000EEFF15C0EDFF12002BDED6DE4AEC03F02A
:10102000E552E552120054DF010EE916000EEA16F1
:10103000010E120021DFEE52EE6AED6A41EF07F079
:10104000FA0EDBCFE9FFFB0EDBCFEAFF1200DBCFAE
:10105000EFFF17DFDBCFEFFF12000ADE020EE12603
:10106000120006DE050EE1261200DECF14F0DDCF01
:1010700015F0120098DF010EEECFDBFF020E12001A
:08108000E926000EEA2212002D
:0810880080EC0DF0FB0EDBCF44
:10109000F3FFDB06F35000090AE0CEEC0DF0FA0E88
:1010A00039EC0EF0F3E1151CF1E1010E01D0000E58
:1010B000AFEF0DF080EC0DF03B0EE12402E3E168B0
:1010C000E652E16E010EDB6A020EDB6AF90EDBCF3F
:1010D000F6FFFA0EDBCFF7FFFB0EDBCFF8FF0800C1
:1010E000F550DF6EDF5002E1D3EF0CF0250EDF5C30
:1010F00002E0C6EF0CF0030EDB6A040EDB6A050E9D
:10110000DB6A060EDB6A070EDB6AE8EC0CF02D0EDC
:10111000DF5C0CE02B0EDF5C09E0200EDF5C06E0FC
:10112000230EDF5C03E0300EDF5C1AE1DF50300A93
:1011300014E0130A0FE0030A0AE00B0A05E0060AAE
:10114000E4E1030EDB80E1D7030EDB82DED7030E82
:10115000DB84DBD7030EDB86D8D7030EDB88D5D73D
:101160002A0EDF5C1BE1E4EC0CF032EC0DF010E039
:10117000030EDB8008680968130EDBCF0DF0140E38
:10118000DBCF0EF078ECB5F0040E06C0DBFF03D029
:10119000130E1BEC0DF0E8EC0CF00BD0090EDB6A23
:1011A00089EC0DF003E0FDEC0DF0FAD7090E1BEC15
:1011B0000DF0030EDBB0DB982E0EDF5C1BE1E8ECDC
:1011C0000CF02A0EDF5C0BE1E4EC0CF032EC0DF0DD
:1011D00003E1130E6DEC0DF0E8EC0CF00BD0090EF2
:1011E000DB6A89EC0DF003E0FDEC0DF0FAD7090E97
:1011F0006DEC0DF0680EDF5C07E1E8EC0CF0680EBA
:10120000DF5C1DE1030E18D0740EDF5C17E07A0E70
:10121000DF5C14E0480EDF5C06E0540EDF5C03E0A8
:101220005A0EDF5C02E1020E07D06C0EDF5C03E0B9
:101230006A0EDF5C04E1010EC0EC0DF0C9DBDF508B
:101240006E0A01E17FD31E0A01E192D1200A01E179
:101250008FD13F0A01E149D11A0A01E146D10D0AB5
:1012600001E143D1200A01E140D13A0A01E13DD137
:10127000200A01E13AD1260A01E135D10D0A01E146
:1012800032D11A0A01E1D9D0200A4AE0300A1FE01F
:10129000460A0EE0250A01E083D3D950F90FE96E22
:1012A000FF0EDA20EA6E010EEE5E000EEE5AEE5AE6
:1012B000CEEC0DF0250EE66E95DB03E1151C01E189
:1012C00069D3CAEC0DF001E26BD3DB2A69D3080EB7
:1012D000DB6A040EDB50010806E2040EDB0492EC2C
:1012E0000DF0DB508BDB080EDB5009E0030EDB500A
:1012F000010B05E172DB01E04DD3080EDB6A64DB14
:10130000EFCFDFFF42EC0EF003E1151C01E142D309
:10131000CAEC0DF001E3DB2A60DB01E141D33AD3F3
:10132000070EDB5002080FE10EEC0EF0030ED5ECB9
:101330000DF00E0EEECFDBFF0F0EEECFDBFF100E2B
:10134000EECFDBFF20D0F70EDBCF17F0F80EDBCFB0
:1013500018F0020E175E000E185AF70E17C0DBFFCA
:10136000F80E18C0DBFF17C0E9FF18C0EAFFC5EC94
:101370000DF0166A0E0E14C0DBFF0F0E15C0DBFF5A
:10138000100E16C0DBFF0E0EDBCFE6FF0F0EDBCF1D
:10139000E6FF100EDBCFE6FF74ECABF0E552E55252
:1013A000E552130E07C0DBFF140E08C0DBFF060E6C
:1013B000DB5005E0130E09EC0EF001E26ADB2DECC8
:1013C0000EF002E2130E37DBF0EC0DF006E0040E37
:1013D00009EC0EF002E2050E2EDB030EDBB005D0A9
:1013E000FCDA01E0D7D2080EDB6A090EDB6A0E0ECA
:1013F000DBCFF6FF0F0EDBCFF7FF100EDBCFF8FFD2
:101400000800F550DF6EDF5014E033EC0EF011E20F
:1014100042EC0EF003E1151C01E1BCD2BBDB01E3A1
:10142000DB2A090EDB2AD9500E0FE96E000ECBDB4A
:10143000E7D7D3DA01E1B4D2ADD2C6DA110EEECFDE
:10144000DBFF120EEDCFDBFF110EDBCFE6FF120E3E
:10145000DBCFE6FF66ECABF0E552E552130EF3CFBF
:10146000DBFF140EF4CFDBFF060EDB5004E0130E9F
:10147000D0DB01E20EDB2DEC0EF002E2130EDBDA24
:10148000AFDB05E0040EC5DB02E2050ED4DA030E85
:10149000DBB005D0A2DA01E07DD2080EDB6A090ECE
:1014A000DB6A110EDBCFE9FF120EDBCFEAFFEFCFD5
:1014B000DFFFDF5014E0D7DB12E2E4DB03E1151CB1
:1014C00001E168D267DB01E3DB2A090EDB2A110E9A
:1014D000DB2ADBCFE9FF120EE8E3DB2AE6D77DDA71
:1014E00001E15ED257D2030EDB8E070EDB0410E162
:1014F00095DB040E5ADB0A0EEECFDBFF0B0EEECFB0
:10150000DBFF0C0EEECFDBFF0D0EEECFDBFF6CD062
:10151000070EDB5003082CE1030EDBAE0DD0B2DA70
:10152000020E76DAEFCF14F0156A166A176A14AE57
:1015300039D01568166835D0F70EDBCF15F0F80EE8
:10154000DBCF16F0020E155E000E165AF70E15C010
:10155000DBFFF80E16C0DBFF15C0E9FF16C0EAFF7F
:10156000EFCF14F00A0E14C0DBFF0B0EDB6A38D08D
:10157000070EDB50020809E1030EDBAE04D059DB95
:1015800016AE10D00ED055DB0DD0030EDBAE12D050
:1015900079DA020E3DDAF9DA166A176A15AE02D068
:1015A00016681768E2DA0C0E16C0DBFF0D0E17C0C6
:1015B000DBFF1AD0F70EDBCF16F0F80EDBCF17F0FB
:1015C000020E165E000E175AF70E16C0DBFFF80E5D
:1015D00017C0DBFF16C0E9FF17C0EAFFD6DAC5DA8D
:1015E0000C0EDB6A0D0EDB6A060EDB5005E1010E08
:1015F000F36E050EF3CFDBFF150EDB6A160EDB6A0A
:10160000D950370F146E000EDA20156E390E14C043
:10161000DBFF3A0E15C0DBFF380EDB6A080EDB6A13
:101620000A0EAEDADF50780A12E0200A10E0280A2B
:101630000CE0200A0AE03F0A06E00D0A02E0200A58
:1016400008E1020E05D0080E03D0080EDF26100EAA
:1016500097DA030EDBBE02D0DB92DB94DB50800B0B
:1016600024E08ADAD890030EEB50000A08E6000E58
:10167000EE5C000EEE58000EEE58000EEE5815E22D
:1016800013DA0B680C680D680E685EECB8F00A0E91
:1016900002C0DBFF0B0E03C0DBFF0C0E04C0DBFF40
:1016A0000D0E05C0DBFF2D0E08D0030EDBA202D00D
:1016B0002B0E03D0DBA408D0200EF36E170EF3CF51
:1016C000DBFF150EDB2A02D0170EDB6A050EDB509E
:1016D00003E1B7D901E189D0300E146E720E156E98
:1016E000010E166E070EDBCF17F0186A196A1A6A18
:1016F00017C00BF018C00CF019C00DF01AC00EF096
:10170000D3D9D9EC0FF014500224F36E15500320F6
:10171000F46E16500420F86EF4CFF7FFF3CFF6FF07
:101720000800090EF5CFDBFF580EDF5C0FE1610EFC
:10173000F36E090E7BD90AE3200E146E090EDBCF7F
:10174000E7FF1450E75E090EE7CFDBFF070EDBCFA4
:1017500014F0156A166A176A0FDA14C00BF015C078
:101760000CF016C00DF017C00EF0EECF06F0EECF65
:1017700007F0EECF08F0EFCF09F0D9EC0FF009C079
:10178000EDFF08C0EDFF07C0EDFF06C0EFFF390E0B
:10179000DBCFE9FFDB063A0EDBCFEAFF01E2DB0637
:1017A000090EDBCFEFFF150EDB2A4BD995E1030EB7
:1017B000DBA61DD06F0EDF5C06E1C1D918E3150E64
:1017C000DB285BDA14D0780EDF5C09E0580EDF5CB2
:1017D00006E0620EDF5C03E0420EDF5C08E1020E11
:1017E000F36E160EF3CFDBFF02D0150EDB6A030E8D
:1017F000DB50100B0EE0040EDBCF14F0050EDB50B7
:10180000D880145406E2060EDB5003E1040EDB50D0
:1018100034DA95D90AE2050EDBCFE7FF150EDB506F
:10182000E75E050EE7CFDBFF02D0050EDB6A040E94
:10183000DBCF14F0160E45D9D880145414E2160EDE
:10184000DBCFE6FF150EDBCFE6FF040EDBCFE6FFB6
:10185000050EDB50E552E75CE552D880E754E552CF
:10186000D880E7545FD9030EDB50010B0BE1080E63
:10187000DB5008E0B2D801E08DD0080EDB50BED8B6
:10188000080EDB6A170EDB5007E088D9170EF1D976
:1018900003E1151C01E17ED0160EDB5016E07ED967
:1018A000300EE66E9FD802E1151C74E077D9DFCFC9
:1018B000E6FFDCECB7F0E552E552E552F4CF15F067
:1018C0000001F31C02E1151C65E0050EDBCF14F0EE
:1018D000160EDB50D880145409E2050EDBCFE7FF6B
:1018E000160EDB50E75E050EE7CFDBFF300EE66E2F
:1018F000050ECBD94FE1390EDB2ADBCFE9FF3A0EDB
:1019000001E3DB2ADBCFEAFF090EEFCFDBFFDB5081
:101910000EE044D9090EADD902E1151C3BE0390EA9
:10192000DB2ADBCFE9FF3A0EEDE3DB2AEBD755D814
:1019300031E1160EDBCFE6FF080EC3D8E552E724EF
:101940005DD82ED0070EDB50030A1CE0010A14E01C
:10195000030A07E07BD9DBCFEEFF020EDBCFEDFF02
:101960001FD0F5D8196A17AE02D0186819682CD89C
:10197000BCD819C0EEFF14D0EAD817BE186824D816
:10198000B4D80ED063D9DBCFEFFF0AD07BD905E105
:10199000151C03E1F368F46810D0FCD801E3DB2ADE
:1019A00079D96FEF08F0010EDBCF14F0020EDBCF18
:1019B00015F014C0F3FF15C0F4FF3B0EE15C02E22A
:1019C000E16AE552E16ECBD029D9020ED5EF0DF0D8
:1019D00061D90800F550DF6E1200200EE66E080E89
:1019E00045EF0EF0DCECB7F0E552E552E552F3CFEF
:1019F00014F0F4CF15F00001F31C1200146E156AF8
:101A0000D950010F4DD91450EE261550ED22120079
:101A1000185E000E195AF70E18C0DBFFF80E19C039
:101A2000DBFF18C0E9FF19C0EAFF1200DBCFF4FFAB
:101A3000F350F45C1200DB50E76E040EE7CFDBFFDF
:101A400012000A0EDBCF14F00B0EDBCF15F00C0EDC
:101A5000DBCF16F00D0EDBCF17F01450151016105B
:101A600017101200130EEECFDBFF140EEDCFDBFFCD
:101A7000130EDBCF14F0140EDBCF15F00001800E37
:101A800015141200F70EDBCF18F0F80EDBCF19F0AB
:101A90001200050EDB50E66ED950130F01D9E55246
:101AA000E750EE6EED6A12000A0EDBCF06F00B0E69
:101AB000DBCF07F00C0EDBCF08F00D0EDBCF09F00B
:101AC0001200DBCFE6FF150EDBCFE6FF050EDB5085
:101AD000E552E724E552E7241200DB50CED8010E90
:101AE000F36E060EF3CFDBFF1200EE50EFCFEAFFEE
:101AF000E96E16C0EEFF17C0EEFF18C0EEFF120031
:101B0000D9CFE6FFDACFE6FFE1CFD9FFE2CFDAFFA8
:101B10001200DFCFE6FFE66AC3EC17F0E552E552AC
:101B2000F3501200E76E080EE7CFDBFF1200EECF96
:101B300014F0EECF15F0EFCF16F0176A1200050E75
:101B4000DBCF14F0150EDB50D88014541200010EB8
:101B5000DBCF16F0020EDBCF17F0186A1200E55249
:101B6000E5CFDAFFE7CFD9FF12000A0E14C0DBFF82
:101B70000B0E15C0DBFF1200D9500A0F50EF0EF00C
:101B8000F36E070EF3CFDBFF1200EECF14F0EFCFB2
:101B900015F01200010EDB2A020E1200FC0EDBCF44
:101BA000E6FFFD0EDBCFE6FF1200145E000E155AB5
:101BB000F70E14C0DBFFF80E15C0DBFF14C0E9FF01
:101BC00015C0EAFF1200DA20EA6EEF2AEECFF6FF28
:101BD000000EEF22EECFF7FFEF22EECFF8FF12005C
:101BE000040EDBCFE6FF130EDB50E552E75C9ADF15
:101BF000DB5004DF060EDB501200090EDB500A0D2D
:101C0000F350DF24D00FE76E090EE7CFDBFFE8EFDC
:101C10000CF0DB50F36E050E16EF0DF0F70EDBCF78
:101C200014F0F80EDBCF15F01200DFCFE6FFF2EF75
:101C30000CF028DF030EECDE97EF0DF044EC08F01B
:101C4000E552E552E552E55200091200BDDEEE50C4
:101C5000EFCFEAFFE96E010E1200130EDB50F36EB8
:101C6000040E16EF0DF0040EDB50F36E090E16EFA6
:101C70000DF0DBCFE6FFF2EF0CF0E76E050EE7CFDD
:101C8000DBFF12008BDF15EF0EF0DBCFE6FF86DF08
:101C90001EEF0EF0D950F90FE96EFF0EE3EF0DF0D5
:0A1CA000E96E000EDA20EA6E120071
:061CAA00A398A39A7ED866
:101CB00008018C6B98929884A59AA598240E6C6E56
:101CC000900E6B6E7C86800EE66E250EE66EE66AE2
:101CD000E66A02D8B5EF0FF038D9020EE126D950E6
:101CE000FB0FE96EFF0EDA20EA6EEECFE6FFEECFD5
:101CF000E6FFEECFE6FFEFCFE6FF88ECACF035D99C
:101D0000F3CFDEFFF4CFDDFFDECF14F0DDCF15F033
:101D100015C014F0156A14507D6EDF506F6E020E00
:101D2000E15C02E2E16AE552E16E14D1A450100BCD
:101D300005E0A350100B02E00AD8010CA450200BC0
:101D400005E0A350200B02E010D8010C000CFDD8D8
:101D5000E65226D976D8E552E552000903E0DF5075
:101D60006D6E01D0A398E552F5D0EFD8E6526BA284
:101D700003D06B986B880BD06E50DF6E6BB407D0BE
:101D8000DFCFE6FF970EE66E080EFCD802D0080102
:101D90008C81E552DFD009D901E1000C010C05D995
:101DA00003E19651010B01E1000C010C320EE66ECD
:101DB000000EE66E060EE66E970EE66E080EDAD898
:101DC000640EE66E000EE66E020EE66E910EE66E94
:101DD000080EBAEF0FF0B9D8A39AC0D8970EE66EE6
:101DE000080EE66E71ECB6F0C0D8000903E0A38AD5
:101DF000010E02D0A38A000EADD0A7D808019CB175
:101E000013D09B51EA6A9725E96E9851EA22EF5068
:101E1000E66EFD0EDBCFE9FFFE0EDBCFEAFFE552FB
:101E2000E750EF6E010E01D0000E94D08ED8A3982B
:101E3000FE0EDBCFE6FF910EE66E080EA3D8A38858
:101E400089D083D88BD8910EE66E080EE66E71ECC1
:101E5000B6F08BD87FD079D8A8D80DE19AD87ED8A3
:101E600066ECABF0E552E552F3CF8FF8F4CF90F883
:101E700013D8010E01D0000E6DD067D896D80AE1B4
:101E800088D8FB0EDBCF8FF8FC0EDBCF90F804D8A0
:101E9000010E01D0000E5ED0A350100B03E1A35041
:101EA000200B03E00201010EFF6F7FD825E0020145
:101EB000FF5122E008018F51901119E09651020B59
:101EC00001E0010E146E156AE850151010E18DC87E
:101ED000E9FF8EC8EAFF8D2B000E8E23EF50E66ED1
:101EE000A5DFE55208018F07000E905BE3D78F5105
:101EF000901102E18D6B8E6B120008018D6B8E6B61
:101F0000D6EF0EF022D8E652A350200B03E1A350E7
:101F1000100B03E00201010EFF6F0201FF5113E0FD
:101F200008019CB110D03CD868DFE552E552DFCF04
:101F3000E6FFB6EC19F0E552000905E131D84BDFB8
:101F4000E552E552EDD7E55205D0D9CFE6FFE1CF16
:101F5000D9FF1200E552E7CFD9FF1200FD0EDBCF0B
:101F6000E6FFFE0EDBCFE6FF1200E552E552E5523A
:101F7000E5521200E66E3BECB6F0146E050EE15E23
:101F800014501200E66E55ECB6F0E552E552E552FB
:101F90001200FD0EDBCF8DF8FE0EDBCF8EF81200A7
:101FA000D9CFE6FFDACFE6FF120008018D518E117E
:021FB00012001D
:0E1FB200056A046A036A026A200EE76ED89080
:101FC0000636073608360936023603360436053635
:101FD0000B50025C0C5003580D5004580E5005581D
:101FE00009E30B50025E0C50035A0D50045A0E5078
:0A1FF000055A062AE72EE4D7120076
:021FFA000000E5
:041FFC00020054008B
:10200000303030007878005000303031000000016E
:102010005000303032007878025000303033007891
:102020007803500030303400787804500030303578
:10203000007878055000303036007878065000304F
:102040003037007878075000303038004040085072
:102050000030303900787809500030313000A0A0CD
:102060000A50003031310078780B500030313200A6
:1020700000000C50003031330078780D50003031C2
:10208000340078780E50003031350078780F5000E9
:1020900030313600787810500030313700787811C0
:1020A0005000303138007878125000303139004813
:1020B00048135000303230007878145000303231FC
:1020C00000A0A01550003032320078781650003051
:1020D0003233007878175000303234007878185056
:1020E0000030323500787819500030323600787878
:1020F0001A50003032370078781B500030323800E8
:10210000E8E81C50003032390078781D5000303338
:10211000300048481E50003033310078781F50009E
:1021200030333200A8A820500030333300787821B3
:102130005000303334007878225000303335007846
:10214000782350003033360078782450003033370D
:1021500000787825500030333800787826500030E9
:10216000333900F0F02750003034300078782850B0
:10217000003034310050502950003034320078782B
:102180002A50003034330078782B5000303434003B
:1021900078782C50003034350078782D5000303469
:1021A000360078782E50003034370078782F500081
:1021B00030343800A0A03050003034390078783105
:1021C0005000343730000000325000343739007886
:1021D0007833500034374100787834500034393740
:1021E000005050355000343938007878365000347B
:1021F000394100787837500036303100989838509F
:102200000036303200787839500036303300787834
:102210003A500036303400E8E83B500036303500A4
:1022200078783C50003630360078783D50003630B3
:10223000370030303E50003631300078783F500063
:1022400036323000787840500036333000787841AC
:1022500050003634300078784250003635300078FF
:102260007843500036363000C8C844500036373006
:102270000078784550003631410078784650003675
:1022800032410010104750003633410078784850F2
:1022900000363441007878495000363541005858AE
:1022A0004A50003636410078784B500036374100AE
:1022B00078784C50003637330078784D50003637F8
:1022C000340078784E50003734300078784F500022
:1022D00037343100787850500037343200787851F4
:1022E000500037343300787852500037353000785A
:1022F00078535000373531007878545000373532F4
:1023000000787855500037353300787856500037CC
:102310003534007878575000373535007878585084
:1023200000373536007878595000373537007878DF
:102330005A500037383900A8A85B500038303800B0
:1023400078785C50003830390078785D5000383942
:102350004400F0F05E50003934310078785F50006E
:1023600039343200787860500039343300404061AD
:1023700050003630410078786250003035420078A5
:102380007863500030353000888864500030353133
:102390000078786550003035410078786650003418
:1023A000363000D0D0675000393730007878685028
:1023B00000393731007878695000393732002020F1
:1023C0006A50003937330078786B50003937340061
:1023D00078786C50003937350068686D50003937AF
:1023E000360078786E50003937370078786F5000B3
:1023F00031393800B0B07050003435390078787118
:102400005000383732007878725000383930000088
:1024100000735000383938007878745000363142F3
:1024200000787875500036324200484876500036C1
:10243000334200787877500036344200787878500C
:102440000036354200909079500036364200787858
:102450007A50003637420078787B500036303800AA
:10246000E0E07C50003638300078787D5000363817
:10247000410078787E50003638420028287F50008E
:1024800036304200787880500038353200787881D4
:102490005000323430007070825000323431007895
:1024A0007883500039393930000184500039393986
:1024B000310001855000656E640078780000006589
:1024C0006E64007878000000656E64007878000023
:1024D00000656E64007878000000656E64007878AE
:1024E000000000656E64007878000000656E64008E
:1024F0007878000000656E64007878000000656EF2
:102500006400787800000000000000000000000077
:1025100000000000000000000000000000000000BB
:1025200000000000000000000000000000000000AB
:10253000000000000000000000000000000000009B
:10254000000000000000000000000000000000008B
:102900000600FC1F0000FB080000040000006472C9
:102910000100FB0500000500000041720100FF02FC
:102920000000010000005A720100000900000A00C6
:10293000000050720100F10800000A000000FA1FB8
:0A2940000000F20700000200000092
:06294A0086DAE6526EDAA7
:1029500066ECABF0E552E552F350DF6EDF501E0837
:1029600002E21E0EDF6E07DB06E2A0DAF9DA86DA93
:10297000FEE1010E69DA5ADADFCFE6FFF1DA7EDA3C
:10298000FEE1020E61DAE5526CD266DA040EE1264F
:1029900094DAEF500EE091DAEFCF16F0176A16BE18
:1029A0001768D4DA06E0FD0EDB2AFE0EF1E3DB2A1F
:1029B000EFD78ADA42DAEFCF16F0176A16BE176839
:1029C000CADA08E0C0DA06E0020EDB2A030EF2E300
:1029D000DB2AF0D7B8DA04E094DA01E3DB2A58DA2C
:1029E000C3DA0BE2B0DA09E094DADECFE6FFDDCF3E
:1029F000E6FFABDFE55294DA01D0010E146E040E4F
:102A0000E15C02E2E16AE552E16E14502AD224DA76
:102A1000040EE12652DAEF500EE04FDAEFCF16F057
:102A2000176A16BE176892DA06E0FD0EDB2AFE0E64
:102A3000F1E3DB2AEFD748DA00DAEFCF16F0176AB6
:102A400016BE176888DA08E07EDA06E0020EDB2A96
:102A5000030EF2E3DB2AF0D776DA04E052DA01E380
:102A6000DB2A16DA81DA10E26EDA0EE052DA5FEC77
:102A7000B2F0E552E552F350E66EDECFE6FFDDCF71
:102A8000E6FF3CD84DDA01D0010E146E040EE15C75
:102A900002E2E16AE552E16E1450E3D14CDA1EE243
:102AA0004EDAECD9FEE1010EB2D9DF5009E0BED911
:102AB000DFCFE6FFB4D9050EE1D9FEE1020EA7D9BA
:102AC000DF50E76EFB0EDBCFE9FFFC0EDBCFEAFF4A
:102AD000E750E926000EEA22EF6A0DD02C0EE66ED2
:102AE000620EE66E010EE66EA1D94DECABF0146EEF
:102AF000050EE15E1450000EE552B3D1ADD93BDABC
:102B00000DE2D950FC0FE66EFF0EDA20E66E010EE4
:102B1000E66E26DAB3D9FEE1000E96D9A2D10BDA21
:102B200014E20DDAABD9FEE1000E71D9DFCFE6FF7A
:102B3000E66A250EE66E620EE66E010EE66E76D948
:102B400037ECB7F0146E070E0BD0160EE66E620E61
:102B5000E66E010EE66E6AD916ECABF0146E050E49
:102B6000E15E1450000EE5527CD1E5D92EE2E7D9A2
:102B700085D9FEE1010E4BD9DF5027E0290EE66E24
:102B8000E6EC24F0E552000909E10601FE2BDFCF57
:102B9000E6FFAFEC24F0E552000902E0010E16D08A
:102BA000000EE66E070EE66EDFCFE6FF38D9050EA3
:102BB00065D9FEE1020E2BD939D9010EE66E2FD967
:102BC000050E5CD9FEE1000E22D9000EE55249D176
:102BD00043D9E652DF6AFE0EDB50290826E10601E2
:102BE000FE5123E0FE07FE511EE1FF51040A12E0F0
:102BF000070A0CE0010A06E0030A13E1B8D9BBECAE
:102C000029F00ED0B4D9D2EC29F00AD0B0D9E9EC31
:102C100029F006D0020EE66EAAD900EC2AF0E552A1
:102C2000E5520601FF6B010EDF6EDF50E55219D150
:102C300013D9E652DF6A0601FE5128E001017851FE
:102C4000791124E04ED9250816E1010EDF6E0AEC59
:102C500023F047D908E045D9290805E00701642B8E
:102C6000000E6523F6D73DD92908ECE10701642B56
:102C7000000E6523E7D7010E0101AD1507E0DF5017
:102C800005E0AEC1E6FFB1EC23F0E552E552E9D034
:102C9000E3D8C5D8000E145C500E155817E3D95070
:102CA000FD0FE96EFF0EDA20EA6E8F0ED880EE542B
:102CB000510EED540BE3BAD8B2D8000E145E500E8C
:102CC000155A5CD952DFE5522BD901D0010EC9D07B
:102CD000C3D8020EE126DE6ADD6A46D915E2E66A4D
:102CE000200EE66EE66A03D9050EC8D8FEE1000E96
:102CF0001CD9E6EC9BF0166E060EE15E1650DF2A3C
:102D0000010EEBE3DB2AE9D7146E020EE15C02E26E
:102D1000E16AE552E16E1450A4D09ED8020EE1267D
:102D2000FD0EDBCFDEFFDBCFDDFFE1D8F80EDBCF22
:102D300018F0F90EDBCF19F0FD0EDB501824166EDB
:102D4000FE0EDB501920176E1650145C17501558E4
:102D500055E2DECF1AF0DDCF1BF01C6A050ED890CD
:102D60001A361B361C36E806FAE1D950FA0FE96E1E
:102D7000FF0EDA20EA6EEE501A24176EEE501B207A
:102D8000186EEE501C20196EFD0EDBCF1DF0FE0EEE
:102D9000DBCF1EF01F6A050ED8901D361E361F367B
:102DA000E806FAE11D50175C146E1E501858156E97
:102DB0001F501958166EE2D8E66E200EE66EE66ACF
:102DC000DECF20F0DDCF21F0050ED8902036213661
:102DD000E806FBE1000E2026040E212220C0E6FFBB
:102DE00021C0E6FFE66AB2EC9BF0226E080EE15EBF
:102DF0002250DF2A010E99E3DB2A97D7146E020EC8
:102E0000E15C02E2E16AE552E16E14502AD08DD80D
:102E100094EC9CF0166E060EE15E16501200FD0E4C
:102E2000DBCF14F0FE0EDBCF15F01200FB0EDBCF74
:102E3000E6FFFC0EDBCFE6FF1200020EDBCFE9FF60
:102E4000030EDBCFEAFF120070D88DEC9BF0166EFC
:102E5000070EE15E16501200D9CFE6FFE1CFD9FF91
:102E60001200E552E7CFD9FF1200E552E552F3CF49
:102E700014F0F4CF15F0F350F4101200D89014367B
:102E80001536E8061200900E145C010E155812005B
:102E9000EF6A6DD8FE0EDBCFE6FFD4ECB2F0E55260
:102EA000E55206C0DEFF07C0DDFF1200D9CFE6FF06
:102EB000DACFE6FF010EE66E1200FD0EDBCFE9FF72
:102EC000FE0EDBCFEAFF1200FD0EDBCF08F0FE0E98
:102ED000DBCF09F0020E08C0DBFF030E09C0DBFFE9
:102EE000120064C7E9FF65C7EAFFEF501200DECFAA
:102EF00014F0DDCF15F0120016C0E6FF17C0E6FF94
:102F00001200020EDBCFE9FFDB2A030EDBCFEAFF64
:102F10001200020EDBCFE6FF030EDBCFE6FF12004E
:102F2000E552E552E552000E12001426040E152259
:102F300025D8E66A120090DFE652BBEF17F0B6DF45
:102F40006EDF050E120079DFEF501200D5DFD5ECF1
:102F500017F035EF17F0D0DFC3EC17F035EF17F0AF
:102F6000E66A5DDF050E1200C2DF43EF17F0FD0ECB
:102F7000DBCFE6FF120053DF43EF17F014C0E6FF8C
:062F800015C0E6FF12007F
:0A2F8600F36AF46AFF0EE124E96E1D
:102F9000FF0EE220EA6EED6607D02F0EEF6404D03C
:102FA0003A0EEF6001D0F32A1200F36AF46AFF0EC2
:102FB000E124E96EFF0EE220EA6EED660AD0200EF3
:102FC000EF5C06E0080EEF6404D00E0EEF6001D057
:102FD000F32A1200FF0EE124E96EFF0EE220EA6EF2
:102FE000EDCFF4FFEFCFF3FFF46607D0600EF3648C
:0C2FF00004D07B0EF36001D0F39A1200B5
:022FFC001200C1
:022FFE001200BF
:1030000000000000000000000000000000000000C0
:1030100000000000000000000000000000000000B0
:1030200000000000000000000000000000000000A0
:103030000000000000000000000000000000000090
:103040000000000000000000000000000000000080
:103050000000000000000000000000000000000070
:103060000000000000000000000000000000000060
:103070000000000000000000000000000000000050
:103080000000000000000000000000000000000040
:103090000000000000000000000000000000000030
:1030A0000000000000000000000000000000000020
:1030B0000000000000000000000000000000000010
:1030C0000000000000000000000000000000000000
:1030D00000000000000000000000000000000000F0
:1030E00000000000000000000000000000000000E0
:1030F00000000000000000000000000000000000D0
:1031000000000000000000000000000000000000BF
:1031100000000000000000000000000000000000AF
:10312000000000000000000000000000000000009F
:10313000000000000000000000000000000000008F
:10314000000000000000000000000000000000007F
:10315000000000000000000000000000000000006F
:10316000000000000000000000000000000000005F
:10317000000000000000000000000000000000004F
:10318000D9CFE6FFE1CFD9FFDD52DD52DF50E84471
:10319000DF10E844DF10E844DF10E844DE14DE52BC
:1031A000E552E7CFD9FF1200000C99EC8DF00D012C
:1031B0003D69FD0EDB50DF6E0D013D5109E0B8ECBD
:1031C00087F0010EE66E48EC87F0F9EC93F0F1E140
:1031D000010EDB50E0EC8BF002E2E16AE552E16EB9
:1031E0001450C8EF85F0CDEC8DF00D013D690D0157
:1031F0003D5110E0FA0EDBCFE6FF78EC86F0FDECF7
:1032000093F025EC91F030EC9DF006EC8EF0DF6E43
:10321000DF50EDE1DF50E552C8EF85F09FEC94F010
:1032200092EC91F031EF93F09FEC94F0F4EC8BF092
:1032300031EF93F09FEC94F0FAEC8BF031EF93F0D8
:10324000E1EC8EF00D013D69010EF36E040EF3CF3B
:10325000DBFF0D013D512CE0040EDB5029E0FD0E9B
:10326000DB500BE0FD0EDB50BDEC87F0D950030FB7
:103270006AEC91F002EC89F002D0040EDB6ADB50BC
:10328000E8E1020EF36EDB6EB8EC87F0E0EC93F051
:1032900037EC94F002EC89F0020EDB0403E1FF0E40
:1032A000DE1604D0020EDB50D4E1DE6ADD6AD1D72F
:1032B000040EDB5003E0F368F46A06D0ECEC86F011
:1032C00014C0F3FF15C0F4FF050EE15C02E2E16AF1
:1032D000E552E16EC8EF85F001EC8EF00D013D691D
:1032E000010E1EEC8AF00D013D5119E0020EDB507B
:1032F00016E0FD0EDB505AEC86F0D950010F6AEC57
:1033000091F062EC90F0EFE1500EDF6E78EC86F019
:10331000B8EC87F037EC94F0D5EC86F0E4D7020EE9
:10332000DB5002E0FF0E01D0000E2DEC8AF002E22D
:10333000E16AE552E16E1450C8EF85F069EC90F057
:103340000F0E9BEF93F069EC90F0100E9BEF93F053
:1033500098EC91F014BE1568CDEC89F00101080ECF
:10336000AE6F010EA76F000EC8EF85F098EC91F0DC
:1033700014BE1568CDEC89F00101ADB302D0080E82
:10338000AE6FC8EF85F0CDEC8DF0FE0EDB98DB9ACA
:10339000DB9CDB9EDB5002E1440E07D00A0E24ECDE
:1033A00086F005E2FE0EDB50300FDF6E1AD0FE0E07
:1033B000DB500F0A14E0010A10E0030A0CE0010AD6
:1033C00008E0070A04E0010A0CE1300E09D02A0ED9
:1033D00007D0230E05D0410E03D0420E01D0430E7C
:1033E000DF6EDF50E552C8EF85F045EC8EF000C18E
:1033F000DFFFDF5001E1A9D068EC8FF081EC89F0AC
:10340000020EEFCFDBFF01010C510DE0010EF36E58
:10341000DB5003E02FEC87F0FDE1F3500101B11523
:1034200002E1020EDB8836EC90F0BDEC87F0DB5059
:1034300029E1020EDB1C100B05E163EC87F031C1C2
:10344000EFFF30D054EC8CF00B0808E054EC8CF01B
:103450000C0804E028EC87F0EF500CE063EC87F0F8
:10346000EFCF14F03051D880145404E263EC87F0AD
:1034700030C1EFFF63EC87F0EF5014E153EC86F0BE
:10348000EF8810D0020EDB1C100B05E063EC87F018
:1034900032C1EFFF07D063EC87F0EF5003E153EC4C
:1034A00086F0EF98030EDB5016E036EC90F013E058
:1034B000020EDB1C100B0FE0A3EC94F00F0B146E4C
:1034C00054EC8CF0145C07E053EC86F0EF9863EC5E
:1034D00087F030C1EFFF36EC90F015E0020EDB1CF8
:1034E000100B11E0A3EC94F0200B0DE154EC8CF0E8
:1034F000146EA3EC94F0F00B1410E66E53EC86F00F
:10350000E552E750EF6E030EDB501DE036EC90F015
:103510001AE153EC86F0EF8A0BA515D03C0ECFECE8
:103520008AF0010EDB50300FCFEC8AF03A0ECFEC70
:103530008AF0A3EC94F0E66E26DFE552CFEC8AF039
:103540003E0ECFEC8AF0DF0654D7040EE15C02E2B7
:10355000E16AE552E16EC8EF85F02AEC91F0E4EC07
:103560008BF004E0010E0801BB1502E1000E01D052
:10357000010E3AEC90F00101BCEC88F003E0C5ECE0
:1035800089F0FDE1CEEC94F0DF5001E1BDD068ECB4
:103590008FF0AEEC86F0EF5014E0010EAEEC86F04A
:1035A00058EC8CF0AEEC86F0EFCF15F0010E81EC0C
:1035B00089F0EF1C1514145C04E152EC93F0EF80D9
:1035C00003D052EC93F0EF90010E81EC89F0EF1CE8
:1035D000400B04E0020EDB50B11303D0020EDB1CE3
:1035E000B117CBEC93F0030B020A21E0010A12E0C1
:1035F000020A08E0010A22E1ECEC8FF04D0FE96EBF
:10360000010E0DD0F6EC89F0EF5018E152EC93F07A
:10361000EF8214D0ECEC8FF0550FE96E010EEA2228
:10362000EF50E66EF6EC89F08EEC87F007D0F6EC02
:1036300089F0EF5003E152EC93F0EF92050EDB506E
:1036400004E1CBEC93F0020B25E1010EDB5093EC8F
:103650008BF0EF5003E0050EDB5042E0020EDB5032
:103660000801B31505E0AEC8E6FFAFC8E6FF08D015
:10367000020EDB50B41509E0B0C8E6FFB1C8E6FFA2
:10368000010E7FEC87F0A7EC90F0020EDB1C01012D
:10369000A81726D0010EDB5093EC8BF0B2C8EFFFD9
:1036A00068EC8CF0A00E1626000EA7EC94F06CECE3
:1036B00093F016E1020EDB500801B31103E0AE51A6
:1036C000AF1107E1020EDB50B4110AE0B051B111A5
:1036D00007E0050EDB5004E1020EDB500101A813E8
:1036E000CBEC93F0020B09E0020EDB500101A815B0
:1036F00004E1020EDB50AF1304D0020EDB1C01010B
:10370000AF1705EC94F040D7060EE15C02E2E16AE7
:10371000E552E16EC8EF85F0BBEC92F003E02FECD0
:1037200087F0FDE1F350DF6E010192519311E81C27
:10373000146E0BEC8EF0CDEC92F00315A51514145D
:103740001BE0DF50011509E0040E0D1506E146EC03
:103750008FF0D10EE926060E0BD0DF5002150CE0DB
:10376000080E0D1509E146EC8FF0B90EE926060E9C
:10377000FDEC89F038EC88F0DF50010101152BE0F9
:103780000BEC8EF0CDEC92F0021525E0DF50921597
:1037900006E046EC8FF0000EE926080E21D0DF503F
:1037A000931506E046EC8FF0A10EE926060E18D020
:1037B0000FEC8EF0C8EC27F0E552000906E046EC6D
:1037C0008FF0300EE926080E0BD046EC8FF0180E65
:1037D000E926080E05D046EC8FF0480EE926080EC3
:1037E000FDEC89F038EC88F0E552C8EF85F0CDECBF
:1037F0008DF0070E98EC93F071EC90F004E1155009
:1038000002E1D2DCDF6ADF5002E0000E01D0010EDF
:10381000E552C8EF85F001EC8EF031EC8AF007E15B
:1038200001010A5104E0010E1EEC8AF009D0BCEC43
:1038300086F003E02FEC87F0FDE1F350D5EC86F045
:1038400000C1DFFFDF501FE068EC8FF094EC8AF0DE
:103850000FE001010A5110E052EC87F049EC8EF0C4
:10386000C2EC94F009E049EC8EF0EE52EF0404E172
:103870004DEC8EF0EF8A05D0A35103E14DEC8EF0B4
:10388000EF9ADF06DFD731EC8AF004E0020E010187
:103890000B1551E00D01F951010196190EE10D01D1
:1038A000FA510101971909E1510EE66EE66A0C0E14
:1038B000E66E620EE66E010E2ED008017551010112
:1038C00096190EE1080176510101971909E1510E8F
:1038D000E66EE66A000EE66E620EE66E010E1BD024
:1038E00008017251010196190EE10801735101019D
:1038F000971909E1510EE66EE66AF00EE66E610E6A
:10390000E66E010E08D0510EE66EE66AEB0EE66E2C
:10391000610EE66E010EE66EAD0EE66E040E05EC6F
:103920008AF09BEC8AF0E552E5528BEC8EF003E3D3
:1039300001010A510BE098C1E6FF96C1E6FF97C16D
:10394000E6FFD6EC00F0E552E552E552030EE15CED
:1039500002E2E16AE552E16EC8EF85F091EC04F015
:10396000000904E12FECADF0000901E0000C010CAE
:1039700001EC8EF031EC8AF007E101010A5104E01C
:10398000010E1EEC8AF009D0BCEC86F003E02FECAF
:1039900087F0FDE1F350D5EC86F000C1DFFFDF508A
:1039A00042E068EC8FF094EC8AF031E001010A51BA
:1039B0000CE052EC87F049EC8EF0C2EC94F005E09C
:1039C00049EC8EF0EE52EF0422E0A95124E00151BF
:1039D0000211146E010EF36EDB5003E02FEC87F042
:1039E000FDE1F350141417E049EC8EF0080EF4ECEE
:1039F00085F0EFCF15F052EC87F031EC8AF002E061
:103A0000000E01D0010EE552E710151404E04DEC54
:103A10008EF0EF8A06D00101A35103E14DEC8EF048
:103A2000EF9ADF06BCD731EC8AF004E0020E010108
:103A30000B151CE04F0EE66EE66A3EEC92F02FECA2
:103A400091F034EC91F02FEC91F029EC93F0500EC2
:103A5000F35C000EF45806E26FEC8CF02FEC91F062
:103A60005EEC94F09BEC8AF0E552E5528BEC8EF024
:103A700005E30101AC5108E10A5106E03EEC92F089
:103A80004AEC03F0E552E552030EE15C02E2E16A22
:103A9000E552E16EC8EF85F0C5EC03F0000904E1E2
:103AA0002FECADF0000901E0000C010CC3EC85F037
:103AB0000BEC8EF0AFEC93F09F0B07E10BEC8EF06C
:103AC000050E77EC8DF0010B02E0010E01D0000E27
:103AD000C8EF85F043DF000904E0DEDF000901E004
:103AE000000C010C3FEC90F0060EDB6A0101BCEC0F
:103AF00088F003E0C5EC89F0FDE1CEEC94F0DF50F6
:103B000001E1ABD02DEC93F0800B06E076EC8CF06D
:103B100003E0BFEC92F0EF9E010E010109150BE0EE
:103B2000020EDB50AF1507E02DEC93F0400B03E0E5
:103B300079EC90F0EF8A040E09150BE0B8EC94F0E4
:103B4000010B07E02DEC93F0400B03E0BFEC92F08B
:103B5000EF9C2DEC93F0620B69E0200A32E0220A20
:103B600019E0420A71E19FEC8AF0EF5073E1020E16
:103B7000091504E0B8EC94F0010B6CE12DEC93F026
:103B80009F0B68E179EC90F0EF82DF04E66EC4DD14
:103B9000E55260D076EC8CF05DE0020EDB50010166
:103BA000AF150BE052EC87F0E8EC85F0C2EC94F036
:103BB00004E0BFEC92F0EF9243D0BFEC92F0EF92B2
:103BC00049D0020EDB50AF1545E1BFEC92F0EF9A01
:103BD000020EDB50A8150AE0060EDBCFE7FF020E4F
:103BE000DB50E712060EE7CFDBFF34D0020EDB50CE
:103BF00001150CE156EC8DF02DE0E8EC85F0CDECF4
:103C000092F0A51527E0080E0D1524E1BFEC92F007
:103C1000EF8C56EC8DF005E09FEC8AF034C1EFFF9D
:103C200019D09FEC8AF033C1EFFF14D052EC87F02B
:103C30006E1D146E6D1DAF151414E552E7140AE0E5
:103C4000BFEC92F0EF8A06D09D0E146EBFEC92F09E
:103C50001450EF1605EC94F052D717EC8DF0F3CF1B
:103C6000DBFF5AEC8DF02CE2DF50DCEC85F0AFECA2
:103C700093F0620B22E1060EDBCFE6FFDF50DCECB7
:103C800085F0C2EC94F019E0010E0E1504E0020E6E
:103C9000DB50011506E1020E0E150FE056EC8DF01B
:103CA0000CE0FBC6E6FFFCC6E6FFFDC6E6FF35EC12
:103CB0008BF0DF50D0EC93F0EF82A6EC8AF0CFD7F8
:103CC000060EDB6A050EDB6A17EC8DF0F3CFDBFF27
:103CD0000051DF5C1FE2EA6ADF346DEC91F0EE52D6
:103CE000EF50800B11E1020EDB50BA1509E0050E12
:103CF000DBCFE7FF020EDB50E712050EE7CFDBFF5D
:103D0000020EDB1CBA1703D0020EDB50BA13A6EC6E
:103D10008AF0DCD7D950030FEBEC8EF0000EEE6E7C
:103D2000040EED6E17EC8DF0F3CFDBFF5AEC8DF047
:103D300046E22DEC93F0620B37E12B1DA511146EBA
:103D4000050EDBCFE6FFE8EC85F0C2EC94F003153E
:103D500014142AE0010E0D1504E0020EDB500115CB
:103D600006E1020E0D1520E056EC8DF01DE0020E6E
:103D7000DB50011506E066EC90F0D10EE926060E48
:103D800008D056EC8DF009E066EC90F0B90EE9260B
:103D9000060EFDEC89F035EC8BF0020EDB1C2AECF4
:103DA00089F0BFEC92F0EF82D950030FEBEC8EF06C
:103DB0000B0EEE26000EEF22A6EC8AF0B5D7B2511C
:103DC000400A68E0C00A66E0A00A4AE0300A2CE037
:103DD000180A22E00C0A19E0060A0BE0030A01E0C7
:103DE00097D0755117E0040EB26F080E765D07E3A9
:103DF00009D0755116E0080EB26F765D03E243C13B
:103E000040FD86D044C140FD83D00D01405101E00A
:103E10007FD00101100E06D00D01405101E078D095
:103E20000101200EB26F74D002EC8CF071E101013F
:103E3000400EB26F080E765D04E29DEC91F0EF84C7
:103E400004D00A5102E0040104850101756B76C1BA
:103E5000E6FFE1DCE5526FEC86F03BEC8BF058D0EE
:103E600002EC8CF055E10101800EB26F080E765D18
:103E700004E29DEC91F0EF8606D00A5104E0AC51CB
:103E800002E1040104870101756B76C1E6FF70DD74
:103E9000E5523ED01FDE000907E10101B26BA96BBC
:103EA00077EC8FF035E132D0400E0101B25D30E1A8
:103EB0003AC114F0156A166A176A3AC1E6FF15C0CE
:103EC000E6FFFFEC86F06FEC86F07DEC8CF084EC86
:103ED0008CF001017F51065C186E80510758196EF5
:103EE000815108581A6E825109581B6E1850145C83
:103EF000195015581A5016581B50175809E272ECF1
:103F000004F00101B26B77EC8FF002E1AEEC3AF015
:103F1000070EE15C02E2E16AE552E16EC8EF85F06E
:103F2000C3EC85F0010E62EC94F0050E43EC92F0C8
:103F3000C8EF85F0CDEC8DF0020E98EC93F071ECAB
:103F400090F005E1155003E1D4EC18F0DF6ADF5082
:103F500002E0000E01D0010EE552C8EF85F0C3EC7F
:103F600085F0180E62EC94F066EC94F0C8EF85F0E2
:103F7000A3EC92F008E048EC92F041E094EC8FF072
:103F800021EC8DF01BD072EC93F01BE01BEC93F056
:103F900036E001016A5102E135EC8EF0ECEC86F07E
:103FA00014503B5D15503C592AE36A5102E035EC50
:103FB0008EF03BC1E6FF3CC1E6FF020E39EC93F008
:103FC0001DD01BEC93F010E04CEC92F015E0E9EC06
:103FD00094F015E12DEC93F0DF0B11E1ECEC86F0A1
:103FE00026EC8DF00CE308D001016A5108E1ECECFD
:103FF00086F026EC8DF003E34FEC92F0E552050ECF
:10400000E15C02E2E16AE552E16EC8EF85F0A3EC03
:1040100092F00BE048EC92F028E035EC8EF021ECC9
:104020008DF0020E39EC93F01CD01BEC93F01BE0EA
:1040300072EC93F011E0ECEC86F0010126EC8DF0CF
:1040400008E33BC1E6FF3CC1E6FF020E39EC93F00A
:10405000E55235EC8EF009D04CEC92F006E14FECD5
:1040600092F0E55202D094EC8FF0050EE15C02E292
:10407000E16AE552E16EC8EF85F0A3EC92F013E03F
:104080001BEC93F00AE135EC8EF0030E0101695D43
:1040900038E052EC87F063DF30D048EC92F031E04A
:1040A00035EC8EF025D01BEC93F029E0E9EC94F090
:1040B00026E072EC93F012E0ECEC86F04151145CD7
:1040C0004251155808E241C1E6FF42C1E6FF020E27
:1040D00039EC93F0E55235EC8EF013D04CEC92F0C5
:1040E00010E14FEC92F0E552030E0101695D09E128
:1040F00021EC8DF0020E39EC93F0E55202D094ECF5
:104100008FF0050EE15C02E2E16AE552E16EC8EF74
:1041100085F0C3EC85F0050E75EC93F0BCEC88F0EF
:1041200003E0C5EC89F0FDE153EC92F0DF5041E093
:1041300068EC8FF001016E1D146EC1EC88F06D1DEE
:10414000E552E71414146C152DE003EC86F060ECD6
:104150008CF005E1690519E0695124E01AD003ECFF
:1041600086F0EE52EF0408E003EC86F0EE52EF50DA
:10417000040814E16B0504E104EC87F0F9DE0CD0CF
:10418000020E6B5D0BE1690504E104EC87F03FDF93
:1041900003D004EC87F071DFE55204D003EC86F025
:1041A00066EC94F0040EB1EC86F058EC92F0DF0669
:1041B000BDD7050EE15C02E2E16AE552E16EC8EFAF
:1041C00085F0C3EC85F0C5EC88F0FE0E39EC93F079
:1041D000E552C8EF85F0C3EC85F00AEC8CF0DF50B7
:1041E0000EE0A0EC91F006E0DF500101005DE66E0C
:1041F000E8DFE552010E8DEC88F0DF06F0D7020E05
:10420000E15C02E2E16AE552E16EC8EF85F0C3ECE1
:1042100085F00AEC8CF0DF500FE0A0EC91F001018A
:10422000011505E0DF50005DE66ECBDFE552010EC3
:104230008DEC88F0DF06EFD7020EE15C02E2E16A66
:10424000E552E16EC8EF85F0CDEC8DF0C1EC8BF05E
:1042500003E02FEC87F0FDE1F350DF6EFE0EDB5044
:1042600005E0DF5001018B13DF5002D0DF50010168
:104270008C13E552C8EF85F0C3EC85F00BEC8EF0A3
:10428000070E43EC92F0C8EF85F0C3EC85F00FEC1D
:104290008EF0E66A2BEC8DF0C8EF85F0C3EC85F06C
:1042A0000101105105E00FEC8EF0010EE66E03D017
:1042B0000FEC8EF0E66A2BEC8DF0C8EF85F099ECF0
:1042C0008DF0BCEC86F003E02FEC87F0FDE1F350BD
:1042D0005AEC86F0DF6A050EDF5C07E2B0EC90F086
:1042E00002E0DF5003D0DF2AF6D7FF0EE0EC8BF0C0
:1042F00002E2E16AE552E16E1450C8EF85F0C3ECCA
:1043000085F0060E75EC93F0BCEC88F003E0C5EC8C
:1043100089F0FDE153EC92F0DF5001E18ED068ECC2
:104320008FF003EC86F0070E77EC8DF001E07BD088
:10433000010117050DE1040EDB50AB1509E0B11DBD
:104340001F15E81C146EC6EC94F0AF15141425D09C
:1043500003EC86F060EC8CF00FE0C1EC88F00351C8
:104360001515146E045116151410E552E71404E1E6
:10437000040EDB50AB1506E0B11D1F15E81C156ED1
:104380008B1D05D0B11D1F15E81C156E8C1D146EFC
:10439000C6EC94F0AF15141415143AEC90F003EC3D
:1043A00086F0EE52EF0422E1040EDB5092150DE090
:1043B000040EDB50AF1509E0050EDBCFE7FF040E5E
:1043C000DB50E716050EE7CFDBFF040EDB5093153D
:1043D0000DE0C1EC88F0C6EC94F00115E552E71051
:1043E000AF1504E0015193152AEC89F0C6EC94F066
:1043F0009415AF1511E0C1EC88F0C6EC94F0E552CD
:10440000E710AF15E66EC0EC18F0E552000904E0C5
:104410000101941D2AEC89F0010E11EC86F0050EC5
:10442000DBCFEFFF04D0010E11EC86F0EF6A58EC01
:1044300092F0040EF0EC8FF06FD7060EE15C02E212
:10444000E16AE552E16EC8EF85F0BBEC92F003E063
:104450002FEC87F0FDE1F350DF6EDF1C01018B17BD
:10446000DF1C8C174CDFE552C8EF85F0AAEC94F006
:1044700075EC93F000C1DFFFDF5009E003EC86F03C
:10448000070ECAEC94F058EC92F0DF06F5D737DF50
:10449000040EE15C02E2E16AE552E16EC8EF85F0EC
:1044A000E1EC8EF0BCEC86F003E02FEC87F0FDE150
:1044B000F350DF6E0FEC8EF075EC91F002E3020E1C
:1044C000DB6A0101C6EC8BF0020E57EC93F014147A
:1044D0001514BDEC87F0020E57EC93F0DF1405E1E4
:1044E000DF50011505E01C5103E0010EDB6A03D02B
:1044F000DE52020EDD6E020EE7EC8DF0040EF4ECDF
:1045000085F0040EEFCFDBFF1B5130E122EC89F088
:10451000EB50DF142BE12EEC86F0011527E02EEC9A
:1045200086F0146E075102E0000E01D0010E140255
:10453000F3501CE1040EDB50DF1410E1010EF36EAA
:10454000020EDB5003E02FEC87F0FDE1F350010198
:10455000951504E0040EDB1C071508E1040EDB5082
:10456000DF1407E0040EDB50071503E0010EDB94B7
:1045700002D0010EDB84DB50146E050EE15C02E21A
:10458000E16AE552E16E1450C8EF85F0CDEC8DF094
:104590008BEC8CF0DF6EF0CDE6FFF1CDE6FFF2CDD7
:1045A000E6FF38EC88F0DFA207D0F3CDE6FFF4CDCC
:1045B000E6FFF5CDE6FF08D0DFA40DD0F6CDE6FF8F
:1045C000F7CDE6FFF8CDE6FF0FEC8EF0A3EC19F087
:1045D000D9EC8DF0E5520BEC8EF0040E5CEC92F011
:1045E000E552C8EF85F0C3EC85F01C0E14EC87F0A3
:1045F0001D0E62EC94F0AFEC93F0100B04E00BECAA
:104600008EF0ECEC92F0C8EF85F090EC8CF00601A7
:10461000FE6B120001EC8EF064C7E9FF65C7EAFF8C
:10462000EFCFDFFF010E64C7DBFF020E65C7DBFFC4
:10463000010EE76EDBCFE9FF020EDBCFEAFFE750AA
:1046400077EC8DF0E66E5DEC86F08EEC87F006E0A0
:10465000010EDB2A020EECE3DB2AEAD7DF502DEC59
:104660008AF002E2E16AE552E16E1450C8EF85F08B
:1046700099EC8DF08BEC8CF05AEC86F00101B06F68
:104680006FEC86F006C0BBF107C0BCF108C0BDF1FD
:1046900009C0BEF10101A35107E100C1DFFFDF50F6
:1046A00003E061EC92F0FBD73CEC94F05CEC92F010
:1046B000EFCDE6FFEDCDE6FFEECDE6FFD6EC00F068
:1046C000D9EC8DF00101A35117E1010EDBA207D057
:1046D000F5CDE6FFF3CDE6FFF4CDE6FF08D0DBA491
:1046E0000BD0F8CDE6FFF6CDE6FFF7CDE6FF2FECD9
:1046F00001F0E552E552E552020EE15C02E2E16AA8
:10470000E552E16EC8EF85F099EC8DF00101B051F2
:1047100020E0B06B72EC04F00101A35102E18AECDD
:1047200004F000C1DFFFDF5014E068EC8FF00101FE
:10473000A35103E14DEC8EF0EF9A49EC8EF0AFEC13
:1047400093F0100B04E049EC8EF0ECEC92F0DF06F5
:10475000EAD7020EE15C02E2E16AE552E16EC8EFDF
:1047600085F0CDEC8DF00101A35107E100C1DFFF21
:10477000DF5003E061EC92F0FBD78BEC8EF010E29F
:104780003CEC94F0F4EC85F0040EEF6E65C8E6FFA7
:1047900063C8E6FF64C8E6FFD6EC00F0E5520DD032
:1047A000E60EE66E610EE66E010EE66EAD0EE66E8C
:1047B000040E6FEC87F09BEC8AF0D9EC8DF0C8EF1B
:1047C00085F0E1EC8EF091EC04F0000904E15BEC83
:1047D00005F0000924E0D950040F1CEC8EF0E0EC49
:1047E00093F015EC01F0D6EC94F072EC04F000C1FB
:1047F000DFFFDF5014E068EC8FF00101A35103E10B
:104800004DEC8EF0EF9A49EC8EF0AFEC93F0040B88
:1048100004E049EC8EF0ECEC92F0DF06EAD7050EEE
:10482000E15C02E2E16AE552E16EC8EF85F0AAECD4
:1048300094F05CEC8CF024EC86F015E21F0EDF6E39
:10484000010E5DC1DBFF020E5EC1DBFF030E5FC127
:10485000DBFFD950010F04EC95F049EC86F01F0EF8
:10486000EEEC87F019D031EC8AF016E1010EA36F5F
:104870005DC1E6FF5EC1E6FFB9EC02F0E552E5522C
:10488000F3CF16FDF4CF17FD5FC11CFD9D900D0108
:1048900011899D80A0EC3AF0040EE15C02E2E16A2D
:1048A000E552E16EC8EF85F0C3EC85F031EC8AF09B
:1048B0000BE10101A35108E0A36B9D900D0111993B
:1048C0009D80AEEC3AF006D04AEC8FF003E21E0E6B
:1048D00014EC87F0C8EF85F0C3EC85F069EC94F038
:1048E000B1EC89F0F3CFE6FFF4CFE6FFF4EC94F0FF
:1048F0007DEC8CF01650F324146E1750F420156ED6
:10490000640E66EC91F007E2F8EC85F0000EE66EBE
:10491000070E0AEC8AF0C8EF85F0C3EC85F049EC8D
:1049200090F0F4EC8EF01426000E1522640E66EC66
:1049300091F009E20FEC8EF049EC90F07FEC05F07D
:10494000E552E552E552C8EF85F069EC94F0320E7D
:10495000D880F354000EF45401E2010C000C99ECE1
:104960008DF069EC94F0F350DF6EFE0EDB50DF2427
:10497000010F146E640E145C1FE2010EDFCFDBFF2B
:10498000DB5012E0010EDB5099EC8BF0EF50E66E3D
:1049900066EC92F0DB50E552E72499EC8BF08EEC5C
:1049A00087F0010EDB06ECD7FE0EDB5099EC8BF0A6
:1049B00000C7EFFF000E01D0010EE0EC8BF002E229
:1049C000E16AE552E16E1450C8EF85F0EFEC92F029
:1049D000DB500BE0010EE66EC2DFE552000905E197
:1049E000FE0EDBCF00F7000E01D0010EC8EF85F000
:1049F000C3EC85F097EC8CF0EFCF14F0B8EC8FF0AF
:104A0000145C0DE1B8EC8FF00AE0FB0EDB2AFC0E23
:104A100001E3DB2AE7EC89F0EDE3DB2AEBD7B8EC26
:104A20008FF002E0000E07D097EC8CF0EF5002E020
:104A3000010E01D0020EC8EF85F03FEC90F00101AD
:104A4000B05118E06FEC86F00101BB51065C146EAA
:104A5000BC510758156EBD510858166EBE51095805
:104A6000176E45C118F0196A1A6A1B6A44EC8BF07C
:104A700001E24ADE25EC93F09EEC8CF0BCEC88F071
:104A800003E0C5EC89F0FDE153EC92F0DF5001E169
:104A9000F9D168EC8FF0D9EC94F006E0E4EC8BF0FF
:104AA00003E10AEC93F0EF6A53EC86F0020EEFCFCD
:104AB000DBFFC1EC88F0010103510411E552E7145A
:104AC0001DE0C1EC88F004511215146E035111154C
:104AD0001410E552E71412E1020EDBA805D004EC35
:104AE00087F0E66E2BEC8DF0020EDBAA07D053ECBC
:104AF00086F0EF9A69EC92F0020EDB6A020EDBA8F8
:104B000053D069EC92F03DEC91F0040804E03DECE8
:104B100091F0080813E1C1EC88F00101045114156B
:104B2000146E035113151410E552E71407E104EC59
:104B300087F0E66E24EC21F0E5520CD001010FB1B4
:104B400007D0020E0F1507E054EC8CF00B0803E0C1
:104B500042EC91F0E552D9EC94F004E00101B0513F
:104B600001E0D2DD54EC8CF00B080FE13DEC91F04C
:104B7000010B05E004EC87F04EEC21F005D00101BB
:104B80000FA503D042EC91F0E552020EDB50230852
:104B90000BE123EC8AF005E18A5103E0010EAD152B
:104BA00003E142EC91F0E552020EDBAAACD0DBCF80
:104BB000E6FFC3EC19F0E552D5EC86F053EC86F035
:104BC000EF9AD9EC94F005E00101B05102E09CDDD0
:104BD0000CD0C3EC92F0200B08E00AEC93F0EF6AE3
:104BE000AAEC8FF002E0E0EC90F0020EDB502A0815
:104BF00011E13DEC91F0010B07E0D9EC94F03FE0BE
:104C0000E4EC8BF06DE13BD0D9EC94F063E0010172
:104C1000AD9360D0C3EC92F0080836E152EC87F017
:104C2000F4EC8FF06DEC94F04EEC8FF0F4EC8FF030
:104C3000DFDED6EC94F0BDEC87F0DB501CE1010E1A
:104C4000DB50050DB1EC89F0CA0E1626070EA7EC55
:104C500094F029EC93F0F3CFE6FFF4CFE6FF4EECAF
:104C60008FF0C1EC86F084EC8CF09FEC8BF0145C40
:104C7000F45015582FE2030EDB50020831E17DECB1
:104C80008EF05CEC92F02CD0020EDB50230828E171
:104C900023EC8AF005E18A5103E0010EAD1520E115
:104CA00042EC91F0E55223EC8AF004E1020EAD15DE
:104CB00001E0AD93AAEC8FF00DE00AEC93F0080E42
:104CC000EF6E010EDB50050D4EEC90F0CA0EE9269A
:104CD000070E04D07DEC8EF0E926000EEA22EF6A82
:104CE000D9EC94F010E052EC87F017DEE55230EC8E
:104CF0008DF003E0A8EC88F0FDE10101AF1502E0C2
:104D0000899101D08981C3EC92F0100B2CE023EC47
:104D10008AF00BE0010EAD1515E1B05113E107016A
:104D2000005110E14DEC8BF00DE1DCEC94F0AD8323
:104D3000AAEC8FF058E0010EAD1555E107010051C6
:104D400052E14DD00AEC93F0200EEF6EAAEC8FF0FA
:104D500001E185D004EC87F019DCE55228EC87F0FE
:104D600038C1EFFF7CD0C3EC92F0200B4AE0010E7B
:104D70000101AD153CE1B0513AE10701005137E1C5
:104D80004DEC8BF034E1010EDB50AE5D1FE0080E00
:104D9000AE5D1CE2AE51DCEC85F008EC95F0020B48
:104DA00015E0AE51DCEC85F0020EF4EC85F0EF92EC
:104DB0004A0E176E440E186E000E196E010EDBCFF0
:104DC0001AF01B6A1C6A030ECCEC87F0DCEC94F042
:104DD0000101AD83AAEC8FF006E0E0EC90F004EC6A
:104DE00087F046DCE5522A0EE66E97DD37D028ECD8
:104DF00087F0EF5034E1AAEC8FF029E0E0EC90F07E
:104E000026D0D9EC94F01FE023EC8AF009E128ECDD
:104E100087F0EF500EE1B0510CE1010EAD1509E144
:104E20000AEC93F0EF6A010EDB50AE5D13E1AD9337
:104E300011D0B25103E1010EAD1511E039510FE06F
:104E400069EC92F00CD028EC87F0EF5008E10AEC06
:104E500093F0EF6A04EC87F025EC22F0E55223ECA6
:104E60008AF008E1010EAD1505E036EC90F002E0A5
:104E700047C141FDD950050F94EC86F0040EF0ECCB
:104E80008FF004D6070EE15C02E2E16AE552E16EC2
:104E9000C8EF85F045EC8EF00101BCEC88F003E032
:104EA000C5EC89F0FDE1EFEC94F0DF5010E06EEC22
:104EB00092F008E1030ED4EC8EF004E0E6EC90F002
:104EC00036C1EFFFEBEC90F0F0EC8FF0EED7040E74
:104ED000E15C02E2E16AE552E16EC8EF85F045EC83
:104EE0008EF00101BCEC88F003E0C5EC89F0FDE137
:104EF000EFEC94F0DF5017E06EEC92F00FE1030E50
:104F0000D4EC8EF00BE02BEC94F00101061DE55281
:104F1000E71404E0E6EC90F035C1EFFFEBEC90F025
:104F2000F0EC8FF0E7D7040EE15C02E2E16AE552B3
:104F3000E16EC8EF85F0C3EC85F0030E5CEC8CF0FD
:104F4000EFEC8DF066EC89F0DF501AE06EEC92F039
:104F500011E10101061D156EDF04146E010E1452DD
:104F600003E0C5EC89F0FDE1151404E0E6EC90F0F7
:104F700035C1EFFFD950010F94EC86F0DF06E4D77E
:104F8000030EE15C02E2E16AE552E16EC8EF85F0F2
:104F9000E1EC8EF0040EDB6A0FEC8EF0B7EC90F0D3
:104FA00002E3000E2BD0010E5EEC93F0010102151E
:104FB00062EC90F021E0010EF36E030EF3CFDBFF05
:104FC000DF6A0051DF5C18E22BEC94F0020EE8EC93
:104FD0008BF00DE0DF50DCEC85F0090E77EC8DF006
:104FE000355D05E1010EF36E040EF3CFDBFF030E1A
:104FF0008DEC88F0DF2AE5D7040EDB50146E050E29
:10500000E15C02E2E16AE552E16E1450C8EF85F01E
:1050100072EC92F0DF5004E1010E0101011506E08F
:10502000ADEC8AF0400EEF6E000E01D0010EE5529D
:10503000C8EF85F072EC92F0DF5004E1010E01013F
:10504000011506E0ADEC8AF0600EEF6E000E01D0A7
:10505000010EE552C8EF85F099EC8DF012EC8AF064
:10506000DF5004E1010E0101011518E0ADEC8AF0FA
:10507000EF50200BF9EC93F006E0DD0EE66E610ECA
:10508000E66E010E05D0D30EE66E610EE66E010EE1
:1050900098EC93F023DAD9EC8DF0E552020EE15C46
:1050A00002E2E16AE552E16EC8EF85F0F1EC90F0C2
:1050B000400EEF6EC8EF85F0F1EC90F0600EEF6EF1
:1050C000C8EF85F001EC8EF08BEC8EF043E253ECF0
:1050D0008FF0020EEFCFDBFF010EF36E020EDB50FE
:1050E00003E02FEC87F0FDE1F3505AEC86F0020E5E
:1050F000AEEC86F0EF50200BDF6EDF500CE0010EBF
:10510000ECEC8BF008E03FEC87F0C60EE66E610E2B
:10511000E66E010E1DD0DF5008E03FEC87F0B90EBF
:10512000E66E610EE66E010E13D0010EECEC8BF014
:1051300008E03FEC87F0AB0EE66E610EE66E010E06
:1051400007D03FEC87F09D0EE66E610EE66E010E15
:1051500046EC91F0030EE15C02E2E16AE552E16E99
:10516000C8EF85F0F1EC90F0EF5063EC8AF0156A2F
:10517000940F146E020EFCEC85F0D8EC85F0C8EFAD
:1051800085F0E1EC8EF0010E9DEC87F0DF6E020EF3
:105190009DEC87F05AEC86F0030E9DEC87F0D5EC81
:1051A00086F0040E9DEC87F0D880DF54BDEC87F0CC
:1051B000050E9DEC87F002EC89F00101875108E0B3
:1051C0008EEC8EF0880EE66E610EE66E010E07D054
:1051D0008EEC8EF0740EE66E610EE66E010E05EC3E
:1051E00093F0146E110EE15E145071EC94F0050E04
:1051F000E15C02E2E16AE552E16EC8EF85F02AEC7B
:1052000091F00A0E9DEC87F0DE6EDD6A0B0EF4EC79
:1052100090F0F1EC86F01450EE121550ED120C0ED9
:105220009DEC87F0E66E80EC93F076EC92F00D0E3C
:10523000F4EC90F0D950020F12EC8CF00E0E9DECB5
:1052400087F0E66ED950040FEBEC8EF076EC92F01E
:105250000F0EF4EC90F0D950040F12EC8CF0C1EC6E
:1052600088F0050EDBCFE6FF7AEC91F0660EE66E75
:10527000610EE66E010E3FEC89F0DAEC86F0060E68
:10528000E15C02E2E16AE552E16EC8EF85F099EC7B
:105290008DF076EC7BF010EC90F05B0EE66E610E1C
:1052A000E66E010E16EC90F002E2E16AE552E16E64
:1052B000C8EF85F099EC8DF07FEC7BF010EC90F06E
:1052C000500EE66E610EE66E010E16EC90F002E2F4
:1052D000E16AE552E16EC8EF85F099EC8DF086EC5D
:1052E0007BF010EC90F0450EE66E610EE66E010E5E
:1052F00016EC90F002E2E16AE552E16EC8EF85F04B
:10530000C3EC85F0020E5CEC8CF08FEC89F01AE2B5
:10531000210EE66EFDEC93F020EC19F088EC89F09C
:1053200043EC87F0FD0EDBCFE6FFE66A380EE66E53
:10533000610EE66E010EE66EEAEC8DF093EC89F0FC
:1053400071EC94F0020EE15C02E2E16AE552E16E7A
:10535000C8EF85F0C3EC85F001010051E66EE66A06
:10536000330EE66E610EE66E010E4DEC86F0DAEC61
:1053700086F0C8EF85F010EC8FF00FE10601FE51CA
:1053800003E00101775109E1FFEC87F060C896F175
:1053900061C897F162C898F103D00601010EFF6F52
:1053A000C8EF85F010EC8FF00FE10601FE5103E02D
:1053B0000101775109E1FFEC87F06CC896F16DC8E7
:1053C00097F16EC898F103D00601020EFF6FC8EF87
:1053D00085F010EC8FF00FE10601FE5103E00101B2
:1053E000775109E1FFEC87F06FC896F170C897F12B
:1053F00071C898F103D00601030EFF6FC8EF85F066
:1054000010EC8FF015E10601FE5103E00101775128
:105410000FE1FFEC87F0FD0EDB50060B07E0F9CD46
:1054200096F1FACD97F1FBCD98F10CD0B26B0AD082
:10543000FD0EDB50060B04E00601040EFF6F02D0E8
:105440000601FF69C8EF85F010EC8FF00FE106014F
:10545000FE5103E00101775109E1FFEC87F072C8CA
:1054600096F173C897F174C898F103D00601050E40
:10547000FF6FC8EF85F010EC8FF00FE10601FE51D1
:1054800003E00101775109E1FFEC87F075C896F15F
:1054900076C897F177C898F103D00601060EFF6F22
:1054A000C8EF85F0C3EC85F0FFEC87F0FC0EDBCF96
:1054B00096F1FD0EDBCF97F15FC198F1C8EF85F053
:1054C00010EC8FF009E14F0E6BEC89F03EEC92F09E
:1054D00034EC91F0A5EC8CF0C8EF85F010EC8FF077
:1054E0000AE14F0E35EC8AF0000EE66E050E05EC73
:1054F0008AF0A5EC8CF0C8EF85F0C3EC85F0FB0ECC
:10550000DBCFE9FFDB2AFC0EDBCFEAFF01E3DB2A7E
:10551000EF50E66E70EC88F001E3DB2A8EEC87F04A
:10552000EEE1C8EF85F02FEC94F0ADB106D0CEECF3
:1055300086F0EF6AC26B56EC87F00D01415103E132
:10554000E1EC23F069D00101C1516BE01BEC87F065
:10555000EF5067E051EC8AF003E146C141FD02D013
:1055600047C141FD4AEC91F02A0EDF5C55E0230E65
:10557000DF5C52E00AEC23F00101C25113E0C26B80
:10558000DF50390A0DE00E0A09E0760A0EE0030A40
:105590000CE0010A0AE0070A3FE107D02A0E22D0F8
:1055A000230E20D084EC93F003E0DFCFE6FF1BD086
:1055B000DF50430A24E0020A1DE0030A0BE0620AFE
:1055C00009E0290A07E04D0A11E04E0A0FE0070A38
:1055D00023E10CD0CEEC86F0EF5020E0FB0EDB5048
:1055E00005E1200EE66EA2EC87F018D00101010E55
:1055F000C16F14D00101410EC26FC12B0FD0FE0E3E
:10560000DB500101C15D08E2FE0EDB28C16FCEEC6C
:1056100086F0300EEF6E02D0FF0E05D00101C107FB
:1056200092D70101C151E552C8EF85F02FEC94F0FB
:10563000ADB107D0CEEC86F0EF6A010EAA6F56EC42
:1056400087F00D01415106E1E1EC23F00101AA6B65
:10565000FF0E52D00101C1513DE01BEC87F0EF502D
:1056600039E051EC8AF003E146C141FD02D047C167
:1056700041FD4AEC91F00AEC23F001017251DF5C2C
:1056800002E12A0E1ED07351DF5C02E1230E19D015
:10569000FB0EDB50DF5C0DE084EC93F014E1DF5097
:1056A000200A0AE0290A08E0030A02E0070A0BE1DF
:1056B0000101010EC16F0BD0CEEC86F0EF5007E078
:1056C000200EE66E02D0DFCFE6FFA2EC87F00101EC
:1056D000C107C0D7FB0EDB500AE130EC8DF003E0D0
:1056E000A8EC88F0FDE10101AF1501E1C16B0101FA
:1056F000C15101E1AA6BC151E552C8EF85F03FEC01
:1057000090F0FE0EDB50146E156A060ED88014540D
:10571000000E155405E2060EF36EFE0EF3CFDBFF0E
:10572000010EE66EF90EE66E010E98EC93F0FBDECC
:10573000E552A1EC89F03CE1D950050FEBEC8EF07D
:10574000F90EEE6E010EED6EDF680AEC86F0EF509A
:1057500025E00AEC86F0EBEC89F016BE1768E6EC63
:1057600092F001E0DF6A0AEC86F0EBEC89F016BEFD
:105770001768E6EC92F00CE10AEC86F0EFCF1AF035
:105780001B6A1ABE1B687DEC90F002E1FF0E11D07F
:10579000050EDB2A060ED9E3DB2AD7D7F90EE66E13
:1057A000010EE66EE4EC93F006C0BFF107C0C0F155
:1057B000DF50146E070EE15C02E2E16AE552E16E31
:1057C0001450C8EF85F0CDEC8DF0E66AFAEC90F05D
:1057D000AADEE552A1EC89F002E0DF5020D0CEEC49
:1057E00086F0EF501BE0CEEC86F0EBEC89F016BEB5
:1057F0001768E6EC92F00CE1CEEC86F0EFCF1AF0F1
:105800001B6A1ABE1B687DEC90F002E1FF0E07D008
:10581000FC0EDB2AFD0EE3E3DB2AE1D7000EE552A6
:10582000C8EF85F02FEC94F0ADB106D0CEEC86F049
:10583000EF6AC36B56EC87F00D01415103E1E1ECD7
:1058400023F072D00101C15101E17BD01BEC87F044
:10585000EF5001E176D051EC8AF003E146C141FD01
:1058600002D047C141FD4AEC91F084EC93F033E063
:105870000101C35105E1300EDF5C010FC36F56D04B
:105880002C0E176E710E186E010E196EC3051A6E6E
:105890001B6A1C6A1AAE02D01B681C68050ECCEC91
:1058A00087F0300EDF5C1D6E1E6A1F6A14501D24C7
:1058B000F36E15501E20F46E16501F20F86EF4CFB4
:1058C000F7FFF3CFF6FF0800F550E66EA2EC87F085
:1058D0000101C36B2BD0440EDF5C06E00D0EDF5CD4
:1058E00003E00A0EDF5C04E10101010EC16F1ED06E
:1058F0002A0EDF5C19E0430EDF5C09E1FE0EDB28B7
:105900000101C16FCEEC86F0300EEF6E0FD00101B9
:10591000C35108E1200EDF5C03E0090EDF5C02E109
:10592000C12B04D00AEC23F0FF0E0DD00AEC23F0BB
:105930000101C35104E0440EDF5C01E083D7C107DD
:1059400081D70101C151E552C8EF85F02FEC94F0E9
:10595000ADB105D0CEEC86F0EF6A56EC87F00D01C4
:10596000415103E1E1EC23F020D00101C15128E0D5
:105970001BEC87F0EF5024E051EC8AF003E146C1C4
:1059800041FD02D047C141FD4AEC91F00D0EDF5CB4
:1059900003E00A0EDF5C04E10101010EC16F0BD0D0
:1059A000210EDF5C04E10AEC23F0FF0E0BD0DFCF09
:1059B000E6FFA2EC87F00AEC23F00101C107D5D77E
:1059C0000101C151E552C8EF85F045EC8EF0C60EDD
:1059D000E66E010EE66E080EE66E7BEC92F040E19C
:1059E000D950010FEBEC8EF0C60EEE6E010EED6E8F
:1059F0000101C56B5DEC86F0EF5032E05DEC86F0A6
:105A0000EBEC89F016BE1768E6EC92F023E0090E85
:105A1000186E5DEC86F0EF50D00FBDEC87F0DB50D8
:105A2000D880185417E2FE0EDB5009E0030EDB505D
:105A3000A7EC91F00DE0C5EC89F0FDE109D0010E75
:105A4000F36E030EDB5003E02FEC87F0FDE1F35023
:105A50000101C513010EDB2A020ECCE3DB2ACAD7F3
:105A6000DF506BEC8AF002E2E16AE552E16E14501D
:105A7000C8EF85F09FEC94F0FD0F7FEC92F0FF0EE5
:105A8000D880EE54350EED5438E3ACEC8CF0E40ED7
:105A9000145C010E15580BE3FD0EDBCF16F0FE0E65
:105AA000DBCF17F0700E165C010E175826E3FD0EC3
:105AB000DBCF18F0FE0EDBCF19F0010E185C000EE4
:105AC000195808E3E9EC88F0040ED880EE54000E73
:105AD000ED5413E2E9EC88F0A00EEE1802E1020E9C
:105AE000ED180BE0E9EC88F09F0EEE1808E1020ECD
:105AF000ED1805E101018E5102E1000E01D0010E09
:105B0000C8EF85F0FCEC8EF00CE0BDEC90F002E606
:105B1000DEEC8FF006E347EC89F002E6AEEC91F0A4
:105B200002E2010E04D07FEC91F0B4EC91F0146E1F
:105B3000080EE15C02E2E16AE552E16E1450C8EF42
:105B400085F0FCEC8EF010E0BDEC90F002E6DEECAF
:105B50008FF00AE347EC89F006E6D880FF0E075481
:105B6000FF0E5DEC8AF002E2010E04D056EC8BF0E1
:105B7000B4EC91F0146E080EE15C02E2E16AE552C9
:105B8000E16E1450C8EF85F0C3EC85F0100EE126ED
:105B900094EC88F0F8EC85F04BEC88F0D9500A0FC3
:105BA000A6EC89F074E00A0EDBCFE9FF0B0EDBCF29
:105BB000EAFFEF506CE073EC8AF0F4EC87F032EC23
:105BC0008FF002E6DEEC8FF062E3D9EC89F009E6B3
:105BD000D880000E0754000E0854010E0954000E20
:105BE0000A5455E332EC8FF005E6200EEE5CA20E6F
:105BF0003EEC88F00AE2D9EC89F006E6D880FF0E88
:105C00000754350E5DEC8AF042E326EC8FF04BEC46
:105C100088F0040EDB6A050EDB6AD9500A0FA6EC89
:105C200089F04AE0EDEC88F0D890155004E6100EAB
:105C3000145C000E155840E273EC8AF00C0E06C09E
:105C4000DBFF0D0E07C0DBFF0E0E08C0DBFF0F0EE3
:105C500009C0DBFFD9500C0FEBEC8EF075EC94F023
:105C600002E6DEEC8FF013E30C0EDBCF07F00D0E37
:105C7000DBCF08F00E0EDBCF09F00F0EDBCF0AF002
:105C80000A34000E0A1802E6AEEC91F002E2010EB0
:105C900023D115EC86F0CF0EE926010EEA220C0E78
:105CA000DBCFEFFF040EDB2A050E01E3DB2A26EC37
:105CB0008FF04BEC88F0B1D7080EDB6A090EDB6A77
:105CC000A5EC8BF0040EDBCF1CF0050EDBCF1DF036
:105CD0001E6A1F6A1DAE02D01E681F6856EC88F04F
:105CE000F1EC86F0030EEBCFF3FF1750F318E8AE9C
:105CF00002D0F33408D0EE50145CEE501558EE503C
:105D00001658EE50175808E2A5EC8BF0F1EC86F02F
:105D100063EC88F0F4EC88F032EC8FF005E6EB0EE3
:105D2000EE5C010E3EEC88F001E392D0EDEC88F0E1
:105D3000166A176A15AE02D01668176833EC94F02D
:105D40001426EE501522EE501622EE50172217346C
:105D5000000E171804E6D880E40E18EC8CF001E36E
:105D600077D0040EDBCF08F0050EDBCF09F0060E6E
:105D700008C0DBFF070E09C0DBFF32EC8FF005E641
:105D8000E40EEE5C010E3EEC88F024E2E40E87ECBB
:105D900090F0F4EC88F0060EDBCF16F0070EDBCFA8
:105DA00017F0040EDB50165C146E050EDB5017580E
:105DB000156E070E145E000E155A060E14C0DBFF9A
:105DC000070E15C0DBFF1DEC90F00001800E1514CE
:105DD00043E03ED0040EDBCF18F0050EDBCF19F008
:105DE0001A6A1B6A19AE02D01A681B68EB0E206E85
:105DF000010E216E226A236A33EC94F0205C1C6E43
:105E0000EE5021581D6EEE5022581E6EEE50235853
:105E10001F6E56EC88F0F4EC88F0EB0E87EC90F0F7
:105E2000080E14C0DBFF090E15C0DBFFEDEC88F097
:105E30000001800E151404E0040EDB6A050EDB6A17
:105E4000EB0EDE6E010EDE6EDE6ADD6ADD52DD52C5
:105E5000060EDB6A070EDB6AD950040FA6EC89F048
:105E600010E0080EDBCF14F0090EDBCF15F0CF0EDB
:105E70001426010EFCEC85F0C1EC88F0050E90ECC8
:105E800090F0EDEC88F0070E1426000E1522166A2D
:105E9000176A15AE02D0166817681450DE26155022
:105EA000DE221650DE221750DD22DD52DD52D9509F
:105EB000060FA6EC89F00FE0EDEC88F0CF0E14266B
:105EC000010E1522070EE9EC93F0060EDBCFE6FF7C
:105ED000070E90EC90F0000E146E100EE15C02E2E2
:105EE000E16AE552E16E1450C8EF85F001EC8EF0E6
:105EF00081EC8FF002E1010E10D07FEC91F09CEC70
:105F00008FF052EC87F0E66A43EC87F01F0EE66EE6
:105F1000610EE66E010EBBEC91F02DEC8AF002E210
:105F2000E16AE552E16E1450C8EF85F045EC8EF061
:105F300081EC8FF002E1010E0DD056EC8BF09CEC61
:105F40008FF07AEC91F0160EE66E610EE66E010EA1
:105F5000BBEC91F06BEC8AF002E2E16AE552E16E93
:105F60001450C8EF85F04FEC91F0BAEC93F0ECECE4
:105F700086F0166AD8901650000A06E6200E145CC9
:105F8000A20E1558000E165808E2F1EC86F0FF0E2E
:105F9000D880EE54350EED540BE326EC8FF032EC46
:105FA00086F0C0EC91F0D950020FA6EC89F002E126
:105FB000010EDBD080EC93F0100ED880EE54000E72
:105FC000ED5405E2100E1EEC8AF0030EDB6A43EC82
:105FD00087F0110EE66E610EE66E010EAEEC94F0E7
:105FE00037ECB7F057EC8FF0ECEC86F0166A176AD6
:105FF0001C6A1D6A010E1E6E1F6A020EDBCF20F0A6
:10600000030EDBCF21F0226A236A20501C5C186E3D
:1060100021501D58196E22501E581A6E23501F58B9
:106020001B6EE8501718E8AE02D0173402D044ECCB
:106030008BF00CE2A5EC8BF0DECF1CF0DDCF1DF079
:106040001E6A1F6A56EC88F0CDEC8EF0DF0EE66E0D
:10605000010EE66E52EC87F09CEC8FF0ECEC86F0D3
:10606000EA0ED8801454010E15544BE3020EDBCF18
:1060700018F0030EDBCF19F0DE501824166EDD5039
:106080001920176E1606000E175AE40ED880165403
:10609000010E175436E2ECEC86F0E40ED88014546E
:1060A000010E155411E3ECEC86F0E40ED880145682
:1060B000010E1556080E14C0DBFFDB50070FE76E0C
:1060C000090EE7CFDBFF0ED0080EDB6AECEC86F0A2
:1060D000E40E145E010E155A070ECBEC8BF0090E80
:1060E00014C0DBFF090EDB50B3EC8CF00AE2100E9B
:1060F000B3EC8CF006E21CEC8CF0EF6A080EDB2AA5
:10610000F1D7080EDB6ADBCF14F0020EDBCF15F0FF
:10611000030EDBCF16F01550145C000E165424E26B
:106120001CEC8CF0EF50E66EE66A0D0EE66E610E2A
:10613000E66E010E05EC93F057EC8FF0F8EC94F05E
:10614000500ECBEC8BF01406155A53EC90F0EAECA1
:106150008DF0F8EC85F099ECABF0166E060EE15E72
:106160001650080EDB2ACFD7000E146E0A0EE15C23
:1061700002E2E16AE552E16E1450C8EF85F0C3EC2B
:1061800085F0010100518FEC89F00CE2EAEC8DF012
:106190000C0EE66EFDEC93F06CEC19F0D6EC94F07E
:1061A00071EC94F0C8EF85F0CDEC8DF0DF6A080E4D
:1061B000DF5C0BE2DF50F6EC86F0EF50F36EFE0E84
:1061C000DB50F35C02E0DF2AF2D7DF50E552C8EF84
:1061D00085F0C3EC85F0140EE12653EC8FF0EFCF81
:1061E000DFFFDFCFE6FFB2EC93F03AEC90F0DB504C
:1061F0009BEC88F004E1155002E1050EDB6A010E0C
:10620000DF5205E0DFCFF3FFC9EC89F0FDE1D5EC0B
:1062100086F0DBCFE6FF050E57EC93F0E552E7146E
:106220005AEC86F0020EDB500101021506E00B0E5F
:10623000E66E610EE66E010E19D0020EDB500415FB
:1062400006E0090EE66E610EE66E010E0FD0020E3C
:10625000DB50031506E0060EE66E610EE66E010EDB
:1062600005D0040EE66E610EE66E010EE66ED950A4
:10627000110F04EC95F06FEC87F0FD0EDB5010E091
:10628000DF5091EC8DF042EC94F0FA0EE66E600E69
:10629000E66E010E5BEC8BF00B0EE15E16500CD03F
:1062A00042EC94F0F30EE66E600EE66E010EE66EC2
:1062B000EAEC8DF093EC89F0010EDB5027E0020E42
:1062C000DB1C146E050E57EC93F0141435EC8DF0B6
:1062D000080EDB6A070EDB6A080EF36E070EE6ECAB
:1062E0008EF00EE2060EDBA005D0070EDB50300F5D
:1062F000EFEC89F0070EDB2A060EB1EC86F0ECD746
:10630000080EDB5003E0200EEFEC89F0020EDB50AC
:1063100001016D1502E1000E01D0010EBDEC87F008
:10632000020EDB506E1502E1000E01D0010E020DCF
:106330005FEC8BF0020EDB50701502E1000E01D015
:10634000010E040D5FEC8BF0DB50030B13E0030E2A
:10635000DBA207D0EC0EE66E600EE66E010EC6EC18
:1063600086F0030EDBA02ED0E70EE66E600EE66E22
:10637000010E26D0010EDB501EE0E30EE66E600E2D
:10638000E66E010EC6EC86F0FD0EDB501BE0080E3B
:10639000DB5018E0DF0EE66E600EE66E010EC6EC16
:1063A00086F0D950080F1CEC8EF0970EE66E050EA5
:1063B0000AEC8AF007D0DA0EE66E600EE66E010E89
:1063C000C6EC86F0030EDBA407D0D30EE66E600E9B
:1063D000E66E010EC6EC86F0D10EE66E600EE66E3D
:1063E000010EC6EC86F0EAEC8DF074EC87F0010E3D
:1063F000146E140EE15C02E2E16AE552E16E1450A3
:10640000C8EF85F07AEC94F03AE27EEC94F005E087
:10641000DFCFF3FFC9EC89F0FDE1F9EC93F0010166
:106420006D1506EC8FF00BE0020EDB5008E03FEC40
:1064300087F0C70EE66E600EE66E010E1DD0030EED
:10644000DB5008E03FEC87F0BC0EE66E600EE66EB7
:10645000010E12D0020EDB5008E03FEC87F0B30EC5
:10646000E66E600EE66E010E07D03FEC87F0AA0ED6
:10647000E66E600EE66E010E46EC91F001D0000E65
:106480006BEC8AF002E2E16AE552E16E1450C8EF6B
:1064900085F07AEC94F03AE27EEC94F005E0DFCF00
:1064A000F3FFC9EC89F0FDE1F9EC93F001016E1501
:1064B00006EC8FF00BE0020EDB5008E03FEC87F0BB
:1064C0009E0EE66E600EE66E010E1DD0030EDB50D2
:1064D00008E03FEC87F0910EE66E600EE66E010E6E
:1064E00012D0020EDB5008E03FEC87F0860EE66E1D
:1064F000600EE66E010E07D03FEC87F07B0EE66E75
:10650000600EE66E010E46EC91F001D0000E6BECD1
:106510008AF002E2E16AE552E16E1450C8EF85F0BC
:106520007AEC94F03AE27EEC94F005E0DFCFF3FFF2
:10653000C9EC89F0FDE1F9EC93F00101701506EC6E
:106540008FF00BE0020EDB5008E03FEC87F0720E9C
:10655000E66E600EE66E010E1DD0030EDB5008E005
:106560003FEC87F0680EE66E600EE66E010E12D00C
:10657000020EDB5008E03FEC87F05D0EE66E600E29
:10658000E66E010E07D03FEC87F0520EE66E600E0D
:10659000E66E010E46EC91F001D0000E6BEC8AF035
:1065A00002E2E16AE552E16E1450C8EF85F0EDECCD
:1065B00093F013E2BCEC86F003E02FEC87F0FDE1F2
:1065C000B4EC88F087EC93F0DF5001016D1525ECF9
:1065D0008EF03CEC89F0D8EC85F0020EE15C02E232
:1065E000E16AE552E16EC8EF85F0EDEC93F015E25B
:1065F000BCEC86F003E02FEC87F0FDE1B4EC88F012
:10660000D0EC8BF0D4EC85F0DF5001016E1525EC59
:106610008EF0D0EC8BF0D8EC85F0020EE15C02E25B
:10662000E16AE552E16EC8EF85F0EDEC93F013E21C
:10663000BCEC86F003E02FEC87F0FDE1B4EC88F0D1
:106640004A0E88EC8DF0DF5001016F1525EC8EF0BD
:106650004A0E7BEC8DF0020EE15C02E2E16AE5524B
:10666000E16EC8EF85F0EDEC93F015E2BCEC86F03E
:1066700003E02FEC87F0FDE1B4EC88F0D3EC8BF075
:10668000D4EC85F0DF500101701525EC8EF0D3ECD1
:106690008BF0D8EC85F0020EE15C02E2E16AE55293
:1066A000E16EC8EF85F001017051E66EE66A6E5149
:1066B000E66EE66A6D51E66EE66A470EE66E600EBD
:1066C000E66E010E3FEC89F074EF87F03DEC93F03D
:1066D000080EABEC89F010E20101011D146E090EE9
:1066E000D4EC8EF0141402E0A0EC8EF0080EDB2A3D
:1066F000090E8DEC88F0ECD70A0EE15C02E2E16A4B
:10670000E552E16EC8EF85F03DEC93F0080EABEC7E
:1067100089F00EE2090ED4EC8EF00101011502E0C1
:10672000A0EC8EF0080EDB2A090E8DEC88F0EED777
:106730000A0EE15C02E2E16AE552E16EC8EF85F023
:1067400026EC89F0EB5001010715166E010EEB5097
:10675000156E071D1514161020EC8EF022EC89F032
:10676000F4EC85F00151EF1601EC94F06FEC89F038
:1067700028EF86F0E5DFB6EC89F003E0A8EC88F0BE
:10678000FDE1E81C0101951701EC94F028EC8AF07A
:1067900021B19CDF010121A302D06FEC27F028EF8B
:1067A00086F0E1EC8EF0DF6A8BEC8EF03AE20BECD7
:1067B0008EF0EE52EF0404E1FE0EDB50DF6E31D0BE
:1067C0000FEC8EF0B7EC90F002E3010EDB6A010EE5
:1067D000FCEC94F062EC90F024E0030EDB6A040E13
:1067E000DB6A79EC8AF016E252EC87F0C7EC91F0A4
:1067F000EF50166E010E165204E0E846FE0B160628
:10680000FCE1E552E71406E1030EDB2A040EE9E39E
:10681000DB2AE7D779EC8AF004E2C7EC91F0EFCFFE
:10682000DFFFDF50146E050EE15C02E2E16AE55223
:10683000E16E1450C8EF85F045EC8EF0FD0EDB5094
:106840001CE00FEC8EF02DEC88F004E3020EDB6A06
:10685000030EDB6A44EC88F037E1B451151834E1DB
:1068600003EC86F020EC88F0EF500115F9EC93F082
:106870009313010EDB1C921729D012EC8AF0DF5023
:1068800004E1010E010101151FE0DFCFE6FF2DEC51
:1068900088F004E3020EDB6A030EDB6A44EC88F046
:1068A00013E1B451151810E1010EDF5205E0DFCFFE
:1068B000F3FFC9EC89F0FDE1F9EC93F001019213CB
:1068C000010EDB1C931702D0010E0ED0B6EC89F03E
:1068D00003E0A8EC88F0FDE101019513B3EC8EF024
:1068E000FCEC85F0FFEC90F06BEC8AF002E2E16AE0
:1068F000E552E16E1450C8EF85F001EC8EF012EC19
:106900008AF0010EDF5205E0DFCFF3FFC9EC89F01A
:10691000FDE15AEC86F0DFCFE6FF75EC91F002E383
:10692000020EDB6A020EDB507BEC93F015220101B4
:10693000B351141802E1B451151802E0010E13D03E
:10694000010EDB50931507E0020E5EEC93F09315F9
:10695000E81C931703D0010EDB1C9217020EA6EC65
:106960008DF0FFEC90F02DEC8AF002E2E16AE55246
:10697000E16E1450C8EF85F0CDEC8DF0010122B12D
:10698000C3DE010122A302D06FEC27F0CEEC91F020
:10699000011D2CEC8CF00115151020EC8EF0011D62
:1069A000156E22EC89F0EB50151401110CEC89F0F6
:1069B0000BEC95F08BEC8FF028EC86F0E552C8EFED
:1069C00085F099EC8DF001018D6B8E6B8F6B010E54
:1069D000776F996B9E6BDF6A5AEC8DF003E2B7EC30
:1069E0008CF0FAD7080EE66E54EC24F0E552010163
:1069F00023B18ADE010123A302D06FEC27F001014D
:106A000023A523D001EC94F028EC8AF0071D2CEC90
:106A10008CF00715151020EC8EF0071D166E22EC79
:106A200089F0EB501614156E015148EC94F0A5173F
:106A30008BEC93F087EC93F0010EDB1C146E2EECC4
:106A400086F0ABEC8BF028EC86F00101AB6B020E0C
:106A5000E15C02E2E16AE552E16EC8EF85F0EFEC3D
:106A600092F0DBA602D06CDE18D026EC89F0EB5059
:106A7000166E01010151041103111614156E010E59
:106A8000EB500215151020EC8EF0021D146E22EC56
:106A900089F0F4EC85F01450EF1601EC94F001014C
:106AA0006FEC89F0FE0EDBB011DEFE0EDBA202D031
:106AB0006FEC27F0FE0EDBA402D0CEEC91F028ECB8
:106AC00086F0C8EF85F0BEEC8CF0176E0101071D53
:106AD000166EEF5016141714156E020EEB500715B4
:106AE000151020EC8EF0071D0115156E22EC89F0B3
:106AF000EB5048EC94F028EC8AF0B6EC89F003E017
:106B0000A8EC88F0FDE10101951325B1DFDD01015D
:106B100025A302D06FEC27F00101996B9E6B28EF43
:106B200086F0B6EC89F003E0A8EC88F0FDE1E81C03
:106B30000101951728EF86F0B6EC89F003E0A8EC88
:106B400088F0FDE10101951328EF86F0E3EC8FF06A
:106B500005E0DFCFF3FFC9EC89F0FDE154EC91F0E3
:106B600009E0F4EC8DF0010EDB5001016D1382ECB5
:106B700094F001D0010E6BEC8AF002E2E16AE5527A
:106B8000E16E1450C8EF85F0E3EC8FF005E0DFCF45
:106B9000F3FFC9EC89F0FDE154EC91F00BE0F4EC6B
:106BA0008DF0010EDB1C01016D1703EC86F099ECF2
:106BB00090F001D0010E6BEC8AF002E2E16AE5523E
:106BC000E16E1450C8EF85F0C3EC85F0050E92EC31
:106BD00087F005E0DFCFF3FFC9EC89F0FDE15AEC67
:106BE00086F0040EDB6A080EF36E040EE6EC8EF0FF
:106BF0000AE2040EDB50F6EC86F0EF50DF5C03E0B7
:106C0000040EDB2AF0D7010EECEC8BF046E0F4EC3E
:106C10008DF0010EDB5001016E1508E014EC93F0CD
:106C2000330EE66E600EE66E010E31D0010EDB50C3
:106C30006D1509E104EC87F003EC86F077EC8DF03C
:106C4000E552E71008E114EC93F0260EE66E600EB4
:106C5000E66E010E1CD004EC87F003EC86F008EC25
:106C600095F002E0000E01D0010EE552E71408E0B5
:106C700014EC93F0180EE66E600EE66E010E07D06F
:106C800014EC93F00C0EE66E600EE66E010E5BECFB
:106C90008BF0090EE15E165009D0050EE66E600E0F
:106CA000E66E010E05EC93F006EC8EF0EAEC8DF04A
:106CB00074EC87F0050EE15C02E2E16AE552E16EF8
:106CC000C8EF85F0E3EC8FF005E0DFCFF3FFC9EC10
:106CD00089F0FDE154EC91F00DE0F4EC8DF0010E43
:106CE000DB1C146E03EC86F058EC90F0EF1682EC8F
:106CF00094F001D0010E6BEC8AF002E2E16AE552F9
:106D0000E16E1450C8EF85F0E3EC8FF005E0DFCFC3
:106D1000F3FFC9EC89F0FDE154EC91F00FE0F4ECE5
:106D20008DF003EC86F0F4EC85F0010EDB50EF12F1
:106D300003EC86F0020E99EC90F001D0010E6BECA2
:106D40008AF002E2E16AE552E16E1450C8EF85F084
:106D5000BBEC92F003E02FEC87F0FDE152EC8EF0FB
:106D60000EE04AEC8FF00BE22EEC86F0DF14146E8E
:106D700058EC91F0EF1228EC86F0000E01D0010ED5
:106D8000E552C8EF85F0BBEC92F003E02FEC87F002
:106D9000FDE152EC8EF00FE04AEC8FF00CE22EECAD
:106DA00086F0DF14E81C146E58EC91F0EF1628EC16
:106DB00086F0000E01D0010EE552C8EF85F0CDEC53
:106DC0008DF0DF6A050EDF5C14E2F3EC92F0030E47
:106DD000F4EC85F001010151EF160EEC95F0011570
:106DE000146EF3EC92F058EC91F0EF126AEC8DF027
:106DF000E9D7E552C8EF85F0BBEC92F003E02FEC49
:106E000087F0FDE152EC8EF012E04AEC8FF00FE2D9
:106E1000DF50AB13BCC8E6FFBDC8E6FF420EE66E0E
:106E20000D0EE66E85EC87F0E552000E01D0010EE6
:106E3000E552C8EF85F0CDEC8DF048DC65DC6FECF9
:106E400027F0BEEC8CF020EC8EF02EEC86F00101E9
:106E50000115E66E2EEC8FF028EC8AF08BEC8FF0AB
:106E6000EF50E81C6FEC89F0AB6BB6EC89F003E0F7
:106E7000A8EC88F0FDE101012615146EB6EC89F04E
:106E800003E0A8EC88F0FDE1E81C01019515141061
:106E9000956F28EC86F095DDE552C8EF85F0CDECD6
:106EA0008DF0C9EC88F0E4EC85F09BEC27F0010153
:106EB000926B936B2DEC82F0B8EC87F087EC93F03B
:106EC000DF1C01010115E81C6D17A56B0CEC94F09B
:106ED000010127510315946F26C195F1DF6A050E54
:106EE000DF5C06E2ABEC8DF028EC86F0DF2AF7D70A
:106EF0000101010E776F996B9E6BAB6BDF6A5AECE9
:106F00008DF003E2B7EC8CF0FAD7080EE66E54EC85
:106F100024F0E55256DDE552C8EF85F0F1EC93F030
:106F20000FE2FD0EDB501F0B146E44EC90F0EF509F
:106F3000A00B1410E66E44EC90F08EEC87F02CD091
:106F400031EC8AF029E1FD0EDBA002D08E8801D061
:106F50008E98DBA202D08E8A01D08E9ADBA402D05A
:106F60008E8C01D08E9CDBA602D08E8E01D08E9EA0
:106F7000DBA802D08F8001D08F90DBAA02D08D8059
:106F800001D08D90DBAC02D08D8201D08D92DBAE32
:106F900002D0908601D09096C8EF85F0CDEC8DF0B0
:106FA0008BEC8EF030E2050E8FEC89F02CE2C1EC18
:106FB0008BF003E02FEC87F0FDE1F350DF6EFC0E69
:106FC000DB500CE0C1EC8BF003E02FEC87F0FDE12F
:106FD000F350E76EFC0EE7CFDBFF02D0FC0EDB6A5E
:106FE000DBCFE6FFFE0E11EC86F0EECF14F0EFCF14
:106FF00015F0DF1C1514E552E710E66E44EC90F036
:107000008EEC87F077D031EC8AF001E073D0080E77
:107010008FEC89F06FE2FC0EDB5006E0010EF36EA0
:10702000FC0EF3CFDBFF02D0FC0EDB6AC1EC8BF071
:1070300003E02FEC87F0FDE1F35001012A150AE08F
:10704000FC0EDB5002E0000E01D0010EE76EFC0EDC
:10705000E7CFDBFFFD0EDB50070A46E0010A3CE00C
:10706000030A32E0010A28E0070A1EE0010A14E0E0
:10707000030A0AE0010A3EE1FC0EDB50E8B08E880C
:10708000E8B038D08E9836D0FC0EDB50E8B08E8A4F
:10709000E8B030D08E9A2ED0FC0EDB50E8B08E8C4B
:1070A000E8B028D08E9C26D0FC0EDB50E8B08E8E47
:1070B000E8B020D08E9E1ED0FC0EDB50E8B08F8052
:1070C000E8B018D08F9016D0FC0EDB50E8B08D8061
:1070D000E8B010D08D900ED0FC0EDB50E8B08D8261
:1070E000E8B008D08D9206D0FC0EDB50E8B0908658
:1070F000E8A09096E552C8EF85F0C3EC85F04AEC25
:107100008FF010E203010D0EC66FFD0EDBCFC7F34B
:10711000FC0EDBCFC8F38EEC91F0D0EC92F00D0EAC
:10712000EEEC87F0C8EF85F0EFEC92F04EEC94F0C7
:10713000D5EC93F0FC0EDBCFEFFF010E63EC8AF091
:10714000040DD2EC91F0FD0EDB50C5EC90F063EC39
:107150008AF0040DC2EC8CF0FD0EDB5057EC89F088
:10716000C8EF85F0C3EC85F0FAEC90F0DDDFD9ECE8
:107170008DF031EC8AF005E136EC8FF013EC6AF01B
:1071800004D0FAEC90F0B9DFE552E552E552C8EFD1
:1071900085F0C3EC85F031EC8AF007E11DEC8FF04F
:1071A000FDEC93F013EC6AF006D01DEC8FF0F8ECD8
:1071B00085F0A3DFE552E552E552C8EF85F099EC82
:1071C0008DF00101ADA1F46BF45139E1F10EE66EE1
:1071D000010ED0EC92F07BEC92F029E1F10EE66E1C
:1071E000010EE66EC1EC86F0F4CF15F0020EF31836
:1071F0001EE115501CE10101010EF46F300EF15D2E
:10720000EF6F300EF25DF06F000EEF5D43E3EF5174
:10721000080840E3000EF05D3DE3F05103083AE357
:10722000DBEC8EF0EFCFF5F146C141FD92D0B1EC31
:1072300094F001E08ED0155001E08BD02AD00D01E2
:10724000415104E113EC94F019E01DD00101785193
:10725000791101E17ED01BEC87F0D9EC8AF001E1D5
:1072600078D046C141FD010EDB502A0804E0010E32
:10727000DB50230812E113EC94F005E1DBEC8EF017
:10728000C9EC8CF004D0DBEC8EF0E8EC8AF0E5522F
:10729000E5520101786B796B5CD0010EDB50440A3A
:1072A00031E07D0A28E00A0A1FE00B0A19E00D0A06
:1072B00012E0070A0CE0050A06E0060A38E1FCECD9
:1072C0008DF0EF2A34D0FCEC8DF0EF0630D0FCECE2
:1072D0008DF0EF682CD0FCEC8DF07F0EEF6E27D098
:1072E000FCEC8DF0EF6A23D00A0E166EFCEC8DF0EC
:1072F0001650EF261CD00A0E166EFCEC8DF01650C0
:10730000EF5E15D0010EE66E6FEC8AF0D2EC91F0D4
:10731000F051C5EC90F0E66E040E0101EF03C2ECF3
:107320008CF0F051000157EC89F068EC8BF00AEC1E
:1073300023F0080E0101EF5D05E1DBEC8EF0C9ECF6
:107340008CF004D0DBEC8EF0E8EC8AF0E552E552EC
:1073500082D7020EE15C02E2E16AE552E16EC8EF1B
:1073600085F099EC8DF00101ADB102D00001F46B14
:107370000001F45139E1F10EE66E000E3EEC86F0AC
:107380007BEC92F029E1F10EE66E000EE66EF4EC75
:107390008EF0F31821E115501FE10001010EF46F8A
:1073A000300EF15DF06F000EF05D41E3080EF05D10
:1073B0003EE2F051F6EC86F0EFCFF0F062EC8DF0AB
:1073C000E66A370EA3EC8FF00001F56FF66BF76BF2
:1073D000F86B46C141FDACD0B1EC94F001E0A8D00F
:1073E000155001E0A5D023D00D01415120E001014D
:1073F0007851791101E19CD01BEC87F0D9EC8AF02F
:1074000001E196D046C141FD010EDB502A0804E09F
:10741000010EDB5023080FE1F5C0E6FFF6C0E6FFE2
:10742000F7C0E6FFF8C0E6FF340EA3EC8FF00101D1
:10743000786B796B7DD0010EDB50440A69E0710AEC
:107440005EE0010A52E0020A46E0010A3BE0060A59
:1074500030E0090A1CE00A0A11E00B0A0BE00A0AF4
:1074600059E10001E051F927E151FA23E251FB23F0
:10747000E35139D0E00EE96E000E0CD00001E4516A
:10748000F927E551FA23E651FB23E7512CD0E40E0E
:10749000E96E000EEA6EEE500001F95D146EEE50DA
:1074A000FA59156EEE50FB59166EEE50FC59176ED8
:1074B00031D00001E851F927E951FA23EA51FB23C1
:1074C000EB5111D00001E851F95FE951FA5BEA5143
:1074D000FB5BEB5112D00001EC51F927ED51FA237F
:1074E000EE51FB23EF51FC2315D00001EC51F95F65
:1074F000ED51FA5BEE51FB5BEF51FC5B0BD0F5C03D
:10750000F9F0F6C0FAF0F7C0FBF0F8C0FCF002D0DA
:1075100068EC8BF0F9C0E6FFFAC0E6FFFBC0E6FFBF
:10752000FCC0E6FF340EA3EC8FF00AEC23F064D726
:10753000020EE15C02E2E16AE552E16EC8EF85F01D
:10754000CDEC8DF0080EDF6EDF5005E008EC87F023
:10755000EF8ADF06F9D7E552C8EF85F0CDEC8DF064
:10756000080EDF6EDF5003E061EC92F0FBD7E552CE
:10757000C8EF85F054EC94F0F1EC86F001018351F2
:10758000EE5C146E8451EE58156E8551EE58166EF1
:107590008651EE58D2EC88F00BE3DFCF83F1010E79
:1075A000DBCF84F1020EDBCF85F1030EDBCF86F15A
:1075B000040EE15C02E2E16AE552E16EC8EF85F09B
:1075C000AEC191F1AEC1E6FFB2EC93F00101B56F2F
:1075D000050EB55D01E3B56BB551CFEC8CF0B3276B
:1075E000060EB423120001019151AE5D11E16FEC62
:1075F00086F001018351065C146E84510758156EA4
:1076000085510858166E86510958D2EC88F001E26F
:10761000D7DF1200C3EC85F0AEC191F1050E24EC6A
:1076200086F002E3010E0FD0FE0EDBCFB5F1DB508A
:10763000CFEC8CF00101B327060EB4236FEC86F07B
:1076400071EC8BF0000EC8EF85F0F1EC93F002E3E3
:10765000FE0EDB6A53EC8FF0EF50E66EB2EC93F067
:10766000E66ED8DFE552C8EF85F02FEC94F0ADB1AF
:1076700016D0F66BE9EC88F0770EEE1802E1030EF7
:10768000ED1808E0E9EC88F0710EEE1808E1370E0D
:10769000ED1805E1A388A38A0201010EFF6F010125
:1076A000F6513FE1FBEC88F0610E081802E1370E5D
:1076B00009181BE0710E081802E1370E091815E0D1
:1076C000760E081802E1030E091806E0770E081876
:1076D00015E1030E091812E1E66A78EC86F04B0E0C
:1076E000E66E93EC2AF0E55206D078EC86F04B0E6D
:1076F000E66EA6EC2CF0D9EC8DF0DF6EDF500AE1DF
:107700000101010EF66F6FEC8CF078EC86F05EEC08
:1077100094F057D0B1EC94F054E1155052E1FF0EC3
:1077200051D0F60529E1FBEC88F0770E081802E14C
:10773000030E091817E0710E081802E1370E091838
:1077400011E0760E081802E1030E091806E0610E3A
:1077500008180EE1370E09180BE178EC86F08FEC73
:10776000ADF004D078EC86F02BEC0FF0E552E5524A
:107770000101020EF66F25D0FBEC88F0770E081899
:1077800002E1030E091817E0710E081802E1370E26
:10779000091811E0760E081802E1030E091806E038
:1077A000610E08180EE1370E09180BE133ECADF04D
:1077B000000907E004D0CFEC0EF0000902E0000E53
:1077C00001D0010EE552C8EF85F02FEC94F0ADA189
:1077D000F76BF7511CE1060EE66E7FEC2BF0E552DD
:1077E000DF6EDF500EE10101FF0ED880BF55000EA5
:1077F000C05502E2BF69C06BBFC13FFD010EF76F0C
:107800000CD0B1EC94F009E1155007E103D00D0163
:107810003F5103E10101786B796BE552C8EF85F0C8
:10782000D9CFE6FFE1CFD9FF130EE12601018D513B
:1078300001018E1128E0450EE66E0D0EE66EA6ECF7
:1078400000F0E552E55201017B51065C146E010126
:107850007C510758156E01017D510858166E0101C3
:107860007E510958176ED8802C0E1454010E1554F1
:10787000000E1654000E175406E201018D6B010133
:107880008E6B01018F6B040EDB6A0601FE5102E173
:107890000F015D6B0701005101E06CDE010E01017B
:1078A000AD1502E07AEF41F00101B25102E07AEF4A
:1078B00041F00701005102E17AEF41F000C7DFFF1C
:1078C0000AEC23F0DF6E2A0EDF5C0EE0DFCFE6FF6E
:1078D000E66AD5EC17F0E552E552F3CF14F0F4CF99
:1078E00015F01450151006E00101786B796B0F014B
:1078F000006B80D3AEC1E6FFDFCFE6FFE8EC15F00A
:10790000E552E55200090BE00101786B796B0F013C
:10791000006B0601FE5102E10F015D6B6BD3DFCFFF
:10792000E6FF000EE66E0F0EE66E7FEC05F0E55208
:10793000E552E55201018D5101018E110BE001016B
:10794000AE510101905D06E001018D6B01018E6B6E
:1079500001018F6BD950080FE66E000EDA20E66E3B
:10796000000EE66E0F0EE66E070EE66E140EE66E65
:10797000610EE66E0D0EE66EEAEC83F0146E080EF4
:10798000E15E1450E76E050EE7CFDBFF050EDB501E
:10799000020850E1010EF36E040EF3CFDBFF0F017E
:1079A000006B0101786B796B080EDBCF14F0090EC8
:1079B000DBCF15F0153404E214500108000E155405
:1079C00008E20101010E8D6F01018E6B01018F6BC9
:1079D00011D00101010E8E6FD950080FE96EDACF78
:1079E000EAFFEE50ED1003E10101010E8F6F01017E
:1079F000010E8D6F450EE66E0D0EE66EA6EC00F0E4
:107A0000E552E55206C07BF107C07CF108C07DF16C
:107A100009C07EF1AEC190F1080E0101AE5D09E131
:107A2000010E01010B1505E0AEC1E6FFBBEC29F02C
:107A3000E552E0D2050EDB0409E1010EF36E040EFF
:107A4000F3CFDBFF0101786B796BD4D2D950060FED
:107A5000E66E000EDA20E66E000EE66E0F0EE66EA3
:107A6000040EE66E010EE66E0E0EE66E3E0EE66E3D
:107A7000010EE66E53EC83F0146E090EE15E1450B5
:107A8000E76E050EE7CFDBFF110EDB6A050EDB505C
:107A900001E0A8D0D950060FE66E000EDA20E66E9F
:107AA000000EE66E0F0EE66EFA0EE66EE66A000E49
:107AB000E66E200EE66E000EE66E53EC83F0146E5A
:107AC000090EE15E1450E76E050EE7CFDBFF010EF5
:107AD000F36E110EF3CFDBFF050EDB50020801E061
:107AE00081D0000E166E200E176E000E186E060E58
:107AF000DBCF19F0070EDBCF1AF01B6A1ABE1B682A
:107B0000090E0C6E0D6A0E6A19C007F01AC008F053
:107B10001BC009F02FECB5F004C019F005C01AF035
:107B200006C01BF016501924F36E17501A20F46E7D
:107B300018501B20F86EF4CFF7FFF3CFF6FF060EB8
:107B4000F626000EF722000EF8220900F5CF14F0F9
:107B50000800F5CF15F0150E141802E1010E1518E6
:107B60003FE0000E1E6E200E1F6E000E206E060EF1
:107B7000DBCF21F0070EDBCF22F0236A22BE236881
:107B8000090E0C6E0D6A0E6A21C007F022C008F0C3
:107B900023C009F02FECB5F004C021F005C022F09D
:107BA00006C023F01E502124F36E1F502220F46ED5
:107BB00020502320F86EF4CFF7FFF3CFF6FF060E28
:107BC000F626000EF722000EF8220900F5CF1CF071
:107BD0000800F5CF1DF01C5002E1010E1D1802E156
:107BE000050EDB6A050EDB500AE10101786B796B4B
:107BF0000101AD6B0F01006B05EC23F0FBD1050E0D
:107C0000DB50020801E0EED1040EDB6A0F01006BCD
:107C1000110EDB5001E0F3D00E0E146E3E0E156E09
:107C2000010E166E060EDBCF17F0070EDBCF18F035
:107C3000196A18BE1968090E0C6E0D6A0E6A17C013
:107C400007F018C008F019C009F02FECB5F004C017
:107C500017F005C018F006C019F014501724F36E81
:107C600015501820F46E16501920F86EF4CFF7FF57
:107C7000F3CFF6FF060EF626000EF722000EF822CE
:107C80000900F5CF78F10A00F5CF79F10601FE5130
:107C900038E10E0E146E3E0E156E010E166E060EB7
:107CA000DBCF17F0070EDBCF18F0196A18BE196882
:107CB000090E0C6E0D6A0E6A17C007F018C008F0A6
:107CC00019C009F02FECB5F004C017F005C018F08A
:107CD00006C019F014501724F36E15501820F46ED6
:107CE00016501920F86EF4CFF7FFF3CFF6FF080E09
:107CF000F626000EF722000EF8220800F5CF0CFF42
:107D000005D00601FE0502E108CF0CFF0E0E156E30
:107D10003E0E166E010E176E060EDBCF18F0070E24
:107D2000DBCF19F01A6A19BE1A68090E0C6E0D6ABB
:107D30000E6A18C007F019C008F01AC009F02FEC3D
:107D4000B5F004C018F005C019F006C01AF01550BF
:107D50001824F36E16501920F46E17501A20F86E7E
:107D6000F4CFF7FFF3CFF6FF080EF626000EF7224A
:107D7000000EF8220800F5500F010C15146E800E4D
:107D800014140F010A6F0E0E146E3E0E156E010EC6
:107D9000166E060EDBCF17F0070EDBCF18F0196A50
:107DA00018BE1968090E0C6E0D6A0E6A17C007F02E
:107DB00018C008F019C009F02FECB5F004C017F096
:107DC00005C018F006C019F014501724F36E1550B2
:107DD0001820F46E16501920F86EF4CFF7FFF3CF89
:107DE000F6FF080EF626000EF722000EF822080015
:107DF000F5500F010C11100B0F010B6FF2D0000E9C
:107E0000146E200E156E000E166E060EDBCF17F0E8
:107E1000070EDBCF18F0196A18BE1968090E0C6E30
:107E20000D6A0E6A17C007F018C008F019C009F0F3
:107E30002FECB5F004C017F005C018F006C019F01B
:107E400014501724F36E15501820F46E1650192094
:107E5000F86EF4CFF7FFF3CFF6FF060EF626000E0E
:107E6000F722000EF8220900F5CF78F10A00F5CFCD
:107E700079F10601FE5138E1000E146E200E156EE8
:107E8000000E166E060EDBCF17F0070EDBCF18F0D4
:107E9000196A18BE1968090E0C6E0D6A0E6A17C0B1
:107EA00007F018C008F019C009F02FECB5F004C0B5
:107EB00017F005C018F006C019F014501724F36E1F
:107EC00015501820F46E16501920F86EF4CFF7FFF5
:107ED000F3CFF6FF080EF626000EF722000EF8226A
:107EE0000800F5CF0CFF05D00601FE0502E108CF22
:107EF0000CFF000E156E200E166E000E176E060E8D
:107F0000DBCF18F0070EDBCF19F01A6A19BE1A681A
:107F1000090E0C6E0D6A0E6A18C007F019C008F041
:107F20001AC009F02FECB5F004C018F005C019F024
:107F300006C01AF015501824F36E16501920F46E6E
:107F400017501A20F86EF4CFF7FFF3CFF6FF080EA4
:107F5000F626000EF722000EF8220800F5500F0159
:107F60000C15146E800E14140F010A6F000E146E9F
:107F7000200E156E000E166E060EDBCF17F0070EE4
:107F8000DBCF18F0196A18BE1968090E0C6E0D6A5D
:107F90000E6A17C007F018C008F019C009F02FECDE
:107FA000B5F004C017F005C018F006C019F0145061
:107FB0001724F36E15501820F46E16501920F86E21
:107FC000F4CFF7FFF3CFF6FF080EF626000EF722E8
:107FD000000EF8220800F5500F010C11100B0F01D4
:107FE0000B6F08D0010EF36E040EF3CFDBFF01011F
:107FF000786B796B01017851791101E17BD1010135
:10800000781D01E1791D04E10101786B796B62D182
:10801000080E0101AE5D21E10101896B01018D5165
:1080200003E00101899702D00101898701018E5186
:1080300003E00101899902D0010189890F010C51E6
:108040000F010B11010189150F01096F0F01095172
:1080500003E00101786B796B3DD1010EAEC1E7FF02
:10806000E75204E0E846FE0BE706FCE1E76E0A0E85
:10807000E7CFDBFF0A0EDBCFE6FFB3C1E9FFB4C1F8
:10808000EAFF020EEB50E552E71408E10A0EDB505E
:108090000101011506E001011C5103E00101899372
:1080A00002D00101898301016E1D156E01016D1D54
:1080B000146EB3C1E9FFB4C1EAFF020EEB50141411
:1080C0001514E76E120EE7CFDBFFB3C114F0B4C195
:1080D00015F0880E145E060E155A050E0D6E0E6A0A
:1080E00014C008F015C009F009ECB5F008C014F090
:1080F00009C015F00B0E14C0DBFFB3C1E9FFB4C11A
:10810000EAFF040EEB50E76E0C0EE7CFDBFF010138
:108110001B5143E10A0EDBCFE6FFB3C1E9FFB4C157
:10812000EAFF030EEB50E552E71437E1B3C1E9FF74
:10813000B4C1EAFFEF50010101152FE0B3C1E9FF1F
:10814000B4C1EAFFEF500101071527E00C0EDBCFA9
:10815000E6FF0A0EDB50E552E71412E1010EF36E62
:108160000B0EDB5004E0D890F336E806FCE1F35048
:108170000101951505E00C0EDB1C010107150DE151
:108180000C0EDBCFE6FF0A0EDB50E552E71408E0E9
:108190000C0EDB500101071503E00101899502D0A7
:1081A0000101898501018D5103E00101899702D008
:1081B0000101898701018E5103E00101899902D0F3
:1081C000010189890F010C510F010B110101891562
:1081D0000F01096F0A0EDB5001016D1503E00F015D
:1081E000098B02D00F01099B0A0EDB5001016E15AD
:1081F00003E00F01098D02D00F01099D0F015D51B0
:1082000003E0400E0F0109170101000E785D500ECA
:1082100079590AE301018F0ED8807855510E7955AE
:1082200003E39F0E0F01091701011D510EE001012B
:108230008D5101018E1109E0500E0F010917010146
:108240008E5103E0100E0F0109170601FE5106E0E2
:108250000F01095103E10F01010E5D6F01017A5118
:108260000EE00101030E781901E1795104E1180EC5
:108270000F01091503E00101786B796B2BD00F0119
:1082800009511BE0800E0F010C150F010A15146E29
:10829000156A1450151011E10101AD810101AD9372
:1082A00005EC23F009CFE6FFAEC1E6FF00EC2AF0B3
:1082B000E552E5520101786B796B0A0EDB50010142
:1082C000701508E001018D5101018E1103E10101DA
:1082D000786B796B080E0101AE5D0AE10101010EB8
:1082E000781901E1795104E10101010EAC6F02D06E
:1082F0000101AC6B01017851791102E12BEF67F0BC
:10830000F3EC3AF0450EE66E0D0EE66EA6EC00F0CC
:10831000E552E55206C07BF107C07CF108C07DF153
:1083200009C07EF10101781D01E1791D02E006011D
:10833000FF6B040EDB5018E1080EE66E0F0EE66EC2
:1083400078C1E6FF79C1E6FF48EC16F0E552E55248
:10835000E552E552000908E1010EF36E040EF3CF79
:10836000DBFF0101786B796B18EC16F0040EDB5023
:1083700001E0C6D3010EF36E040EF3CFDBFF210E36
:108380000101781902E1030E791901E1F3D2230EFC
:108390000101781902E1030E791901E1EBD2240EF3
:1083A0000101781902E1030E791901E1E3D2020E0D
:1083B0000101781902E1030E791901E1DBD2030E04
:1083C0000101781902E1030E791901E1D3D2050EFA
:1083D0000101781902E1030E791901E1CBD2070EF0
:1083E0000101781902E1030E791901E1C3D20101FB
:1083F000785102E1030E791901E1BCD2010E0101AD
:10840000781902E1030E791901E17DD2040E010110
:10841000781902E1030E791901E175D2580E0101B4
:10842000781902E1030E791901E16DD2590E0101AB
:10843000781902E1030E791901E165D2060E0101F6
:10844000781902E1030E791901E137D2080E010112
:10845000781902E1030E791901E122D2330E0101EC
:10846000781902E1030E791901E1D2D13B0E010125
:10847000781902E1030E791901E1CAD1380E010120
:10848000781902E1030E791901E17BD13A0E01015D
:10849000781902E1030E791901E173D1360E010159
:1084A000781902E1030E791901E140D1370E01017B
:1084B000781902E1030E791901E138D1310E010179
:1084C000781902E1030E791901E1A9D0320E0101F8
:1084D000781902E1030E791901E1A1D0390E0101E9
:1084E000781902E1030E791901E199D0300E0101EA
:1084F000781902E1030E79195BE0210E0101781968
:1085000001E1795126E0010E0101781901E179516B
:108510000CE0E8680101781902E1E868791901E0E6
:10852000ECD20101786B796BEBD20101AD81F90ED0
:10853000E66E5F0EE66E010EE66EAEC1E6FF6EEC15
:108540002AF0E552E552E552E5520101786B796B6C
:10855000D7D2010EE66E7FEC2BF0E552E76E050EEA
:10856000E7CFDBFF050EDB5016E101010051146E71
:10857000156A01011450BF5D1550C05908E2BFC112
:10858000E6FFAEC1E6FFBFEC30F0E552E552010177
:10859000786B796B0CD0050EDB50146E156AFF0EEC
:1085A000141801E1155003E10101786B796BA8D231
:1085B000010EE66E7FEC2BF0E552E76E050EE7CF7D
:1085C000DBFF050EDB501EE10101080EBF5D000E52
:1085D000C05914E20A0E0101BF25E96E090E01011E
:1085E000C021EA6EEF50E66EBBEC7FF0E552000969
:1085F00005E0AEC1E6FFBBEC29F0E5520101786B66
:10860000796B0CD0050EDB50146E156AFF0E141832
:1086100001E1155003E10101786B796B71D2010E14
:10862000E66E7FEC2BF0E552E76E050EE7CFDBFF41
:10863000050EDB506EE10101080EBF5D000EC05952
:1086400064E20F01095117E00F010C51146E156A15
:108650001450800B4EE0F80E0F0109154AE10A0E86
:108660000101BF25E96E090E0101C021EA6EEF503C
:108670000101AE5D3EE10F01010E5D6F310E0101A2
:10868000781902E1030E791915E10A0E0101BF25DF
:10869000E96E090E0101C021EA6EEF50E66E9DEC15
:1086A0007FF0E552000905E0AEC1E6FFBBEC29F022
:1086B000E5521ED0320E0101781902E1030E79193C
:1086C00008E1E66ABFC1E6FFE9EC30F0E552E552A9
:1086D0000FD0390E0101781902E1030E791908E172
:1086E000010EE66EBFC1E6FFE9EC30F0E552E5525F
:1086F0000CD00101AD9305EC23F009CFE6FFAEC12C
:10870000E6FF00EC2AF0E552E5520101786B796B47
:108710000CD0050EDB50146E156AFF0E141801E123
:10872000155003E10101786B796BEAD10101AD814C
:10873000010100510101AE5D20E2370E01017819FF
:1087400002E1030E79190EE0360E0101781902E1FB
:10875000030E791901E00CD0AEC1E6FFBBEC7FF04F
:10876000E55206D0AEC1E6FF9DEC7FF0E55200D0A9
:10877000AEC1E6FFBBEC29F0E5520101786B796BE5
:10878000BFD10101AD810B0EDB6A0B0EDB50EA6A33
:108790000A0FE96E090EEA22EF500101AE5D0CE00E
:1087A000080EF36E0B0EDBCFF4FFF350F45C04E223
:1087B00000D00B0EDB2AE9D7080EF36E0B0EDBCFD1
:1087C000F4FFF350F45C20E2380E0101781902E165
:1087D000030E791909E1E66A0B0EDBCFE6FFE9EC3F
:1087E00030F0E552E55210D03A0E0101781902E15D
:1087F000030E791909E1010EE66E0B0EDBCFE6FFE1
:10880000E9EC30F0E552E5520101786B796B78D1F3
:108810000D0EE66E0F0EE66E4F0EE66EE3EC2BF0DD
:10882000E552E552E552E76E050EE7CFDBFF050E98
:10883000DB5029E1330E0101781902E1030E7919A9
:108840000DE10D0EE66E0F0EE66E3BEC82F0E5528A
:10885000E552E66EE5EC7FF0E5520CD00D0EE66ECB
:108860000F0EE66E3BEC82F0E552E552E66EF9EC57
:108870007FF0E552AEC1E6FFBBEC29F0E552010105
:10888000786B796B0CD0050EDB50146E156AFF0EF9
:10889000141801E1155003E10101786B796B30D1B7
:1088A0000101AD81D8EC7FF0AEC1E6FFBBEC29F051
:1088B000E5520101786B796B23D1010EE66E7FECF6
:1088C0002BF0E552E76E050EE7CFDBFF050EDB5020
:1088D00019E1050EDB50146E156AD890155004E6A8
:1088E000FF0E145C000E15580AE2BFC1E6FF2FEC24
:1088F00035F0E552AEC1E6FFBBEC29F0E5520101CF
:10890000786B796BFDD00101AD81590E01017819A9
:1089100002E1030E791922E0580E0101781902E1F3
:10892000030E791918E0040E0101781902E1030E13
:1089300079190BE0010E0101781902E1030E791992
:1089400001E00FD0BAEC33F00CD024C1E6FF2FECDD
:1089500035F0E55206D066EC33F003D084EC33F00A
:1089600000D0AEC1E6FFBBEC29F0E5520101786B07
:10897000796BC6D00101AD81D9500B0FE66E000EA8
:10898000DA20E66E9E0EE66E020EE66EC1EC6AF02E
:10899000E552E552E552E5520F01095127E0180E64
:1089A0000F01091501E099D001018E5105E1400E3A
:1089B0000F01091501E091D00B0EDB1C146E0A0E9D
:1089C000DB5001016D15141401E187D0070E010180
:1089D000AE150B0DF3CFE9FFF4CFEAFF000EE92649
:1089E000040EEA22EE52EF0401E077D00F01010EEF
:1089F0005D6F0B0EDB6A0101785102E1030E7919FC
:108A000054E0070E0101781902E1030E79194AE0DA
:108A1000050E0101781902E1030E791940E0030EF9
:108A20000101781902E1030E791936E0020E010105
:108A3000781902E1030E79192CE0240E010178194E
:108A400002E1030E79191DE0230E0101781902E1FC
:108A5000030E79190FE0210E0101781902E1030ECE
:108A6000791901E025D0C4EC35F0E76E0B0EE7CFA5
:108A7000DBFF1ED084EC36F0E76E0B0EE7CFDBFF9A
:108A800017D0E4EC35F0010EF36E0B0EF3CFDBFFE5
:108A90000FD063EC35F00CD0E1EC34F009D0BCEC35
:108AA00034F006D01BEC37F003D04FEC37F000D099
:108AB0000B0EDB5011E10101785102E1030E79192F
:108AC00006E1AEC1E6FFE9EC29F0E55205D0AEC102
:108AD000E6FFBBEC29F0E5520CD00101AD9305ECAB
:108AE00023F009CFE6FFAEC1E6FF00EC2AF0E55225
:108AF000E5520101786B796B03D0040EDB6A00D07C
:108B0000040EDB5002E020EF51F0010EF36E040E74
:108B1000F3CFDBFF060E0101781902E1040E79198B
:108B200002E11AEF51F00101785102E1040E7919C6
:108B300001E1D7D3010E0101781902E1040E791980
:108B400001E1CFD3020E0101781902E1040E791977
:108B500001E1C7D3030E0101781902E1040E79196E
:108B600001E1BFD3040E0101781902E1040E791965
:108B700001E1B7D3050E0101781902E1040E79195C
:108B800001E1AFD3070E0101781902E1040E791952
:108B900001E1A7D3080E0101781902E1040E791949
:108BA00001E19FD3100E0101781902E1040E791939
:108BB00001E197D3090E0101781902E1040E791938
:108BC00001E18FD3110E0101781902E1040E791928
:108BD00001E187D30A0E0101781902E1040E791927
:108BE00001E17FD3D20E0101781902E1400E79191B
:108BF00001E177D30B0E0101781902E1040E791916
:108C000001E16FD3D30E0101781902E1400E791909
:108C100001E167D30C0E0101781902E1040E791904
:108C200001E15FD3D00E0101781902E1400E7919FC
:108C300001E157D3D10E0101781902E1400E7919F3
:108C400001E14FD3140E0101781902E1040E7919E4
:108C500001E147D3150E0101781902E1040E7919DB
:108C600001E13FD3160E0101781902E1040E7919D2
:108C700001E137D3190E0101781902E1040E7919C7
:108C800001E12FD31A0E0101781902E1040E7919BE
:108C900001E127D31B0E0101781902E1040E7919B5
:108CA00001E11FD31C0E0101781902E1040E7919AC
:108CB00001E117D31D0E0101781902E1040E7919A3
:108CC00001E10FD3200E0101781902E1040E791998
:108CD00001E107D3210E0101781902E1040E79198F
:108CE00001E1FFD2220E0101781902E1040E791987
:108CF00001E1F7D2230E0101781902E1040E79197E
:108D000001E1EFD2240E0101781902E1040E791974
:108D100001E1E7D2250E0101781902E1040E79196B
:108D200001E1DFD2200E0101781902E1030E791969
:108D300001E1ADD2220E0101781902E1030E791989
:108D400001E1A5D2820E0101781902E1030E791921
:108D500001E18FD2800E0101781902E1030E791929
:108D600001E1F5D1810E0101781902E1030E7919B3
:108D700001E1EDD1170E0101781902E1040E791914
:108D800001E1E5D1180E0101781902E1040E79190B
:108D900001E1DDD1570E0101781902E1030E7919C5
:108DA00001E19FD1550E0101781902E1030E7919F5
:108DB00001E161D1540E0101781902E1030E791924
:108DC00001E1E3D0560E0101781902E1030E791991
:108DD00001E1DBD0510E0101781902E1030E79198E
:108DE00001E1C3D0500E0101781902E1030E791997
:108DF00066E0520E0101781902E1030E79195FE075
:108E0000130E0101781902E1030E791946E0120EE2
:108E10000101781902E1030E79192DE0110E01010B
:108E2000781902E1030E79191FE0100E010178197B
:108E300002E1030E791911E0A00E0101781902E197
:108E4000020E791902E01DEF51F00101786B796B88
:108E50000101010EA96F20EF51F00101786B796BD0
:108E6000EBEC20F020EF51F00101786B796B07EC0F
:108E700021F020EF51F00101AD81580EE66E040E95
:108E8000E66EAEC1E6FF60EC2AF0E552E552E5522F
:108E90000101786B796B20EF51F00101AD81800EFB
:108EA000E66E040EE66EAEC1E6FF60EC2AF0E55217
:108EB000E552E5520101786B796B20EF51F0010129
:108EC000AD810F0109511AE00F010C51146E156AA2
:108ED0001450800B39E0F80E0F01091535E1070E2B
:108EE0000101AE150B0DF3CFE9FFF4CFEAFF000E41
:108EF000E926040EEA22EE52EF0426E10F01010EEC
:108F00005D6F520E0101781902E1030E791912E02A
:108F1000500E0101781902E1030E791901E013D016
:108F200008EC28F0000905E1AEC1E6FFBBEC29F032
:108F3000E55209D0AEC1E6FF2CEC28F0E552010164
:108F4000786B796B00D00CD00101AD9305EC23F068
:108F500009CFE6FFAEC1E6FF00EC2AF0E552E5528C
:108F60000101786B796B20EF51F00101AD811AECB2
:108F700028F0000905E1AEC1E6FFBBEC29F0E5529F
:108F80000101786B796B20EF51F0010EE66E7FECFA
:108F90002BF0E552E76E050EE7CFDBFF050EDB5049
:108FA0005CE10101080EBF5D000EC05952E20F01E5
:108FB000095117E00F010C51146E156A1450800B03
:108FC0003CE0F80E0F01091538E10A0E0101BF253A
:108FD000E96E090E0101C021EA6EEF500101AE5D9C
:108FE0002CE10F01010E5D6F560E0101781902E1AF
:108FF000030E79191BE0540E0101781902E1030EEA
:10900000791901E019D00A0E0101BF25E96E090E98
:109010000101C021EA6EEF50E66E56EC28F0E552F1
:10902000AEC1E6FFBBEC29F0E55206D0BFC1E6FFBA
:1090300062EC28F0E55200D00CD00101AD9305ECB4
:1090400023F009CFE6FFAEC1E6FF00EC2AF0E552BF
:10905000E5520101786B796B0CD0050EDB50146E74
:10906000156AFF0E141801E1155003E10101786B38
:10907000796B20EF51F0010EE66E7FEC2BF0E5529C
:10908000E76E050EE7CFDBFF050EDB501CE10101AB
:10909000080EBF5D000EC05912E20A0E0101BF2585
:1090A000E96E090E0101C021EA6EEF50E66E5CEC3C
:1090B00028F0E552AEC1E6FFBBEC29F0E552010114
:1090C000786B796B0CD0050EDB50146E156AFF0EB1
:1090D000141801E1155003E10101786B796B20EF61
:1090E00051F0010EE66E7FEC2BF0E552E76E050EB7
:1090F000E7CFDBFF050EDB501CE10101080EBF5D71
:10910000000EC0590DE20A0E0101BF25E96E090EDD
:109110000101C021EA6EEF50E66EB2EC28F0E55294
:10912000AEC1E6FFD2EC29F0E5520101786B796B14
:109130000CD0050EDB50146E156AFF0E141801E1F9
:10914000155003E10101786B796B20EF51F0010EAE
:10915000E66E7FEC2BF0E552E76E050EE7CFDBFF06
:10916000050EDB5001E077D00101080EBF5D000E57
:10917000C05965E2180E0101781902E1040E79194F
:109180004CE0170E0101781902E1040E791933E061
:10919000810E0101781902E1030E79191AE0800E9F
:1091A0000101781902E1030E791901E048D00A0E95
:1091B0000101BF25E96E090E0101C021EA6EEF50E1
:1091C000E66E2BEC80F0E552E76E050EE7CFDBFF95
:1091D00036D00A0E0101BF25E96E090E0101C0213A
:1091E000EA6EEF50E66E46EC80F0E552E76E050E53
:1091F000E7CFDBFF24D00A0E0101BF25E96E090E7F
:109200000101C021EA6EEF50E66E5AEC80F0E552A3
:10921000E76E050EE7CFDBFF12D00A0E0101BF2576
:10922000E96E090E0101C021EA6EEF50E66E6CECAA
:1092300080F0E552E76E050EE7CFDBFF00D0050EAC
:10924000DB5005E1AEC1E6FFBBEC29F0E5520101C0
:10925000786B796B0CD0050EDB50146E156AFF0E1F
:10926000141801E1155003E10101786B796B20EFCF
:1092700051F00101AD817EEC80F00101786B796BDA
:10928000AEC1E6FFBBEC29F0E55220EF51F0010141
:10929000AD81220E0101781902E1030E791912E065
:1092A000200E0101781902E1030E791901E014D0B2
:1092B000A6EC35F0000905E1AEC1E6FFBBEC29F0F4
:1092C000E5520AD062EC36F0000905E1AEC1E6FFD6
:1092D000BBEC29F0E55200D00101786B796B20EFEF
:1092E00051F00101ADB102D00F015E6B0F015E5173
:1092F000040A02E196EF50F0070A02E180EF50F015
:10930000010A02E116EF4FF0030A01E17ED1010AE2
:1093100002E013EF51F0090E0101781902E1040E89
:10932000791901E14BD1110E0101781902E1040E06
:10933000791901E143D10A0E0101781902E1040E05
:10934000791901E13BD1D20E0101781902E1400EF9
:10935000791901E133D10B0E0101781902E1040EF4
:10936000791901E12BD1D30E0101781902E1400EE8
:10937000791901E123D10C0E0101781902E1040EE3
:10938000791901E11BD1D00E0101781902E1400EDB
:10939000791901E113D1D10E0101781902E1400ED2
:1093A000791901E10BD11B0E0101781902E1040EBC
:1093B000791901E103D11C0E0101781902E1040EB3
:1093C000791901E1FBD0230E0101781902E1040EA5
:1093D000791901E1F3D0240E0101781902E1040E9C
:1093E000791901E1EBD0250E0101781902E1040E93
:1093F000791901E1E3D0080E0101781902E1040EA8
:10940000791901E1CBD0050E0101781902E1040EB2
:10941000791901E1B3D0040E0101781902E1040EBB
:10942000791901E19BD0140E0101781902E1040EB3
:10943000791901E193D0150E0101781902E1040EAA
:10944000791901E18BD0030E0101781902E1040EB4
:10945000791974E0020E0101781902E1040E7919FC
:109460005DE00101785102E1040E791947E0010E37
:109470000101781902E1040E791940E0070E01019B
:10948000781902E1040E791939E0160E01017819F4
:1094900002E1040E791932E0100E0101781902E19F
:1094A000040E79192BE0190E0101781902E1040E5E
:1094B000791924E01A0E0101781902E1040E7919D4
:1094C0001DE01D0E0101781902E1040E791916E064
:1094D000200E0101781902E1040E79190FE0210E26
:1094E0000101781902E1040E791908E0220E010148
:1094F000781902E1040E791901E070D00D0EE66EC4
:109500000F0EE66E050EE66EE3EC2BF0E552E5522B
:10951000E552E76E050EE7CFDBFF60D00D0EE66E7D
:109520000F0EE66E070EE66EE3EC2BF0E552E55209
:10953000E552E76E050EE7CFDBFF50D00D0EE66E6D
:109540000F0EE66E0A0EE66EE3EC2BF0E552E552E6
:10955000E552E76E050EE7CFDBFF40D00D0EE66E5D
:109560000F0EE66E0C0EE66EE3EC2BF0E552E552C4
:10957000E552E76E050EE7CFDBFF30D00D0EE66E4D
:109580000F0EE66E060EE66EE3EC2BF0E552E552AA
:10959000E552E76E050EE7CFDBFF20D00D0EE66E3D
:1095A0000F0EE66E070EE66EE3EC2BF0E552E55289
:1095B000E552E76E050EE7CFDBFF10D00D0EE66E2D
:1095C0000F0EE66E010EE66EE3EC2BF0E552E5526F
:1095D000E552E76E050EE7CFDBFF00D0050EDB504E
:1095E00004E10F01010E5E6F0ED0050EDB50146E0C
:1095F000156AFF0E141801E1155005E105EC23F082
:109600000101786B796B19EF51F0300E0F010D5D90
:109610000F015F6F080E0F015F5D09E20F015F51DF
:10962000EA6A0A0FE96E090EEA22EFCF5FFF010135
:1096300000510F015F5D01E3F6D30E0EE66E0F0ED3
:10964000E66ED4ECB2F0E552E5520D0E06C0DBFF3B
:109650000E0E07C0DBFF0F0E08C0DBFF100E09C0A7
:10966000DBFF0101785102E1040E79195CE0010E83
:109670000101781902E1040E791955E0020E010189
:10968000781902E1040E79194EE0030E01017819F0
:1096900002E1040E791947E0040E0101781902E194
:1096A000040E791940E0050E0101781902E1040E5B
:1096B000791939E0070E0101781902E1040E7919D0
:1096C00032E0080E0101781902E1040E79192BE04D
:1096D000140E0101781902E1040E791924E0150E27
:1096E0000101781902E1040E79191DE0160E01013D
:1096F000781902E1040E791916E0210E010178199A
:1097000002E1040E79190FE0250E0101781902E13A
:10971000040E791908E0240E0101781902E1040E03
:10972000791901E00AD05FCFE6FF46EC80F0E55200
:10973000E76E050EE7CFDBFF00D0240E010178199C
:1097400002E1040E791901E151D3250E01017819C6
:1097500002E1040E791901E136D3230E01017819D3
:1097600002E1040E791901E11BD3220E01017819DF
:1097700002E1040E791901E1F7D2210E01017819F5
:1097800002E1040E791901E1D3D20A0E0101781920
:1097900002E1040E791901E1B8D2D20E0101781963
:1097A00002E1400E791901E1B0D20B0E01017819E6
:1097B00002E1040E791901E1A8D2D30E0101781952
:1097C00002E1400E791901E1A0D20C0E01017819D5
:1097D00002E1040E791901E198D2D00E0101781945
:1097E00002E1400E791901E190D2D10E0101781900
:1097F00002E1400E791901E188D2200E01017819A9
:1098000002E1040E791901E164D21D0E01017819FB
:1098100002E1040E791901E140D21C0E0101781910
:1098200002E1040E791901E125D21B0E010178191C
:1098300002E1040E791901E10AD21A0E0101781928
:1098400002E1040E791901E1F4D1190E0101781930
:1098500002E1040E791901E1D0D1160E0101781947
:1098600002E1040E791901E1BAD1150E010178194E
:1098700002E1040E791901E198D1140E0101781961
:1098800002E1040E791901E176D1110E0101781976
:1098900002E1040E791901E15BD1090E0101781989
:1098A00002E1040E791901E140D1100E010178198D
:1098B00002E1040E791901E11CD1080E01017819A9
:1098C00002E1040E791901E1F8D0070E01017819BF
:1098D00002E1040E791901E1D4D0050E01017819D5
:1098E00002E1040E791901E1B0D0040E01017819EA
:1098F00002E1040E791901E18CD0030E01017819FF
:1099000002E1040E791969E0020E0101781902E101
:10991000040E791946E0010E0101781902E1040EE6
:10992000791923E00101785102E1040E791901E06F
:1099300070D2D9500D0FE96EDACFEAFFEECFE6FF15
:10994000EECFE6FFEECFE6FFEFCFE6FF300EE66E9E
:109950005FCFE6FF1AEC19F0146E060EE15E1450AC
:10996000E76E050EE7CFDBFF54D2D9500D0FE96E3D
:10997000DACFEAFFEECFE6FFEECFE6FFEECFE6FF6F
:10998000EFCFE6FF310EE66E5FCFE6FF1AEC19F07F
:10999000146E060EE15E1450E76E050EE7CFDBFF96
:1099A00038D2D9500D0FE96EDACFEAFFEECFE6FFDD
:1099B000EECFE6FFEECFE6FFEFCFE6FF320EE66E2C
:1099C0005FCFE6FF1AEC19F0146E060EE15E14503C
:1099D000E76E050EE7CFDBFF1CD2D9500D0FE96E05
:1099E000DACFEAFFEECFE6FFEECFE6FFEECFE6FFFF
:1099F000EFCFE6FF330EE66E5FCFE6FF1AEC19F00D
:109A0000146E060EE15E1450E76E050EE7CFDBFF25
:109A100000D2D9500D0FE96EDACFEAFFEECFE6FFA4
:109A2000EECFE6FFEECFE6FFEFCFE6FF340EE66EB9
:109A30005FCFE6FF1AEC19F0146E060EE15E1450CB
:109A4000E76E050EE7CFDBFFE4D1D9500D0FE96ECD
:109A5000DACFEAFFEECFE6FFEECFE6FFEECFE6FF8E
:109A6000EFCFE6FF350EE66E5FCFE6FF1AEC19F09A
:109A7000146E060EE15E1450E76E050EE7CFDBFFB5
:109A8000C8D1D9500D0FE96EDACFEAFFEECFE6FF6D
:109A9000EECFE6FFEECFE6FFEFCFE6FF380EE66E45
:109AA0005FCFE6FF1AEC19F0146E060EE15E14505B
:109AB000E76E050EE7CFDBFFACD1D9500D0FE96E95
:109AC000DACFEAFFEECFE6FFEECFE6FFEECFE6FF1E
:109AD000EFCFE6FF390EE66E5FCFE6FF1AEC19F026
:109AE000146E060EE15E1450E76E050EE7CFDBFF45
:109AF00090D1D9500D0FE96EDACFEAFFEECFE6FF35
:109B0000EECFE6FFEECFE6FFEFCFE6FF430EE66EC9
:109B10005FCFE6FF1AEC19F0146E060EE15E1450EA
:109B2000E76E050EE7CFDBFF74D1E66AE66AE66A08
:109B3000E66A3A0EE66E5FCFE6FF1AEC19F0146E95
:109B4000060EE15E1450E76E050EE7CFDBFF61D134
:109B5000E66AE66AE66AE66A3B0EE66E5FCFE6FF15
:109B60001AEC19F0146E060EE15E1450E76E050E45
:109B7000E7CFDBFF4ED1D9500D0FE96EDACFEAFF08
:109B8000EECFE6FFEECFE6FFEECFE6FFEFCFE6FF4C
:109B90005FCFE6FFACECA9F0146E050EE15E145049
:109BA000E76E050EE7CFDBFF34D1D9500D0FE96E1C
:109BB000DACFEAFFEECFE6FFEECFE6FFEECFE6FF2D
:109BC000EFCFE6FF5FCFE6FFB2ECA9F0146E050E13
:109BD000E15E1450E76E050EE7CFDBFF1AD10D0EE4
:109BE000DBCFE6FF5FCFE6FFB8ECA9F0E552E55228
:109BF000E76E050EE7CFDBFF0CD1D9500D0FE96EF4
:109C0000DACFEAFFEECFE6FFEECFE6FFEECFE6FFDC
:109C1000EFCFE6FF440EE66E5FCFE6FF1AEC19F0D9
:109C2000146E060EE15E1450E76E050EE7CFDBFF03
:109C3000F0D00D0EDBCFE6FF5FCFE6FFBFECA9F063
:109C4000E552E552E76E050EE7CFDBFFE2D0E66AAC
:109C5000E66AE66AE66A450EE66E5FCFE6FF1AEC54
:109C600019F0146E060EE15E1450E76E050EE7CF94
:109C7000DBFFCFD0E66AE66AE66AE66A460EE66E83
:109C80005FCFE6FF1AEC19F0146E060EE15E145079
:109C9000E76E050EE7CFDBFFBCD0D9500D0FE96EA4
:109CA000DACFEAFFEECFE6FFEECFE6FFEECFE6FF3C
:109CB000EFCFE6FF470EE66E5FCFE6FF1AEC19F036
:109CC000146E060EE15E1450E76E050EE7CFDBFF63
:109CD000A0D0D9500D0FE96EDACFEAFFEECFE6FF44
:109CE000EECFE6FFEECFE6FFEFCFE6FF480EE66EE3
:109CF0005FCFE6FF1AEC19F0146E060EE15E145009
:109D0000E76E050EE7CFDBFF84D0E66AE66AE66A17
:109D1000E66A370EE66E5FCFE6FF1AEC19F0146EB6
:109D2000060EE15E1450E76E050EE7CFDBFF71D043
:109D3000D9500D0FE96EDACFEAFFEECFE6FFEECF96
:109D4000E6FFEECFE6FFEFCFE6FF490EE66E5FCF10
:109D5000E6FF1AEC19F0146E060EE15E1450E76E81
:109D6000050EE7CFDBFF55D0D9500D0FE96EDACFE6
:109D7000EAFFEECFE6FFEECFE6FFEECFE6FFEFCF56
:109D8000E6FF4A0EE66E5FCFE6FF1AEC19F0146E9E
:109D9000060EE15E1450E76E050EE7CFDBFF39D00B
:109DA000E66AE66AE66AE66A4B0EE66E5FCFE6FFB3
:109DB0001AEC19F0146E060EE15E1450E76E050EF3
:109DC000E7CFDBFF26D0E66AE66AE66AE66A4C0E73
:109DD000E66E5FCFE6FF1AEC19F0146E060EE15E38
:109DE0001450E76E050EE7CFDBFF13D0E66AE66A94
:109DF000E66AE66A4D0EE66E5FCFE6FF1AEC19F0F2
:109E0000146E060EE15E1450E76E050EE7CFDBFF21
:109E100000D0050EDB5004E10F01020E5E6F02D090
:109E20000F015E6902D00F015E6903D2D9500D0F98
:109E3000E66E000EDA20E66E5FCFE6FFADECA8F02E
:109E4000E552E552E552E76E050EE7CFDBFF050E62
:109E5000DB5001E154D10101785102E1040E79197E
:109E600047E0020E0101781902E1040E791940E081
:109E7000030E0101781902E1040E791939E0040E8C
:109E80000101781902E1040E791932E0050E010191
:109E9000781902E1040E79192BE0070E01017819F7
:109EA00002E1040E791924E0080E0101781902E19B
:109EB000040E79191DE0210E0101781902E1040E4A
:109EC000791916E0230E0101781902E1040E7919BF
:109ED0000FE0240E0101781902E1040E791908E05F
:109EE000250E0101781902E1040E791901E01CD058
:109EF000050EDB040CE1010E5FCFE7FFE75204E043
:109F0000E846FE0BE706FCE10101A6130CD0010EAA
:109F10005FCFE7FFE75204E0E846FE0BE706FCE10F
:109F2000E81C0101A61700D0050EDB50030A01E171
:109F3000CDD0010A09E0030A01E0D0D0AEC1E6FFAE
:109F4000BBEC29F0E552D2D0D10E0101781902E123
:109F5000400E79194CE0D00E0101781902E1400E53
:109F600079193FE00C0E0101781902E1040E79190C
:109F700032E0D30E0101781902E1400E791925E093
:109F80000B0E0101781902E1040E791918E0D20EC6
:109F90000101781902E1400E79190BE00A0E010166
:109FA000781902E1040E791901E027D00B0EDB6A63
:109FB00027D0200EF36E0B0EF3CFDBFF21D0080E5F
:109FC000F36E0B0EF3CFDBFF1BD0280EF36E0B0EE0
:109FD000F3CFDBFF15D0090EF36E0B0EF3CFDBFFD3
:109FE0000FD00A0EF36E0B0EF3CFDBFF09D0190E64
:109FF000F36E0B0EF3CFDBFF03D00B0EDB6A00D04A
:10A00000D20E0101781902E1400E79192EE0D30E2B
:10A010000101781902E1400E791927E00A0E0101C9
:10A02000781902E1040E79191DE00B0E010178196F
:10A0300002E1040E791916E00C0E0101781902E113
:10A04000040E79190FE0D00E0101781902E1400EDB
:10A05000791908E0D10E0101781902E1400E791951
:10A0600001E02DD00F01030E5E6FD9500D0FE96E88
:10A07000DACFEAFFEECFE6FFEECFE6FFEECFE6FF68
:10A08000EFCFE6FF0B0EDBCFE6FF0D0EE66E0F0EF9
:10A09000E66EE4ECA8F0146E070EE15E1450030EB9
:10A0A0000F015E5D0BE20D0EE66E0F0EE66EAEC1A9
:10A0B000E6FF60EC2AF0E552E552E55206D0AEC16B
:10A0C000E6FFBBEC29F0E55200D010D005EC23F000
:10A0D000AEC1E6FF24EC2AF0E55208D005EC23F0EF
:10A0E000AEC1E6FF3BEC2AF0E55200D0030E0F01B3
:10A0F0005E5D05E20101786B796B0F015E6B99D0B3
:10A100004E0EE66E5FCFE6FFD5EC18F0E552E55255
:10A11000E76E050EE7CFDBFF050EDB5004E10F0114
:10A12000040E5E6F02D00F015E6983D0D9500D0F0F
:10A13000E66E000EDA20E66E5FCFE6FFADECA8F02B
:10A14000E552E552E552E76E050EE7CFDBFF050E5F
:10A15000DB5002085BE1D9500D0FE96EDACFEAFF60
:10A16000010EEE1805E1EE5003E1EE5001E1EE5074
:10A170000EE0D9500D0FE96EDACFEAFF030EEE18AC
:10A1800005E1EE5003E1EE5001E1EE500CE16D0E01
:10A19000E66E0D0EE66E0F0EE66E7FEC05F0E552F4
:10A1A000E552E55227D0D9500D0FE96EDACFEAFF1C
:10A1B000020EEE1805E1EE5003E1EE5001E1EE5023
:10A1C0000EE0D9500D0FE96EDACFEAFF040EEE185B
:10A1D00005E1EE5003E1EE5001E1EE500BE1700EAF
:10A1E000E66E0D0EE66E0F0EE66E7FEC05F0E552A4
:10A1F000E552E5520D0EE66E0F0EE66EAEC1E6FFBD
:10A2000060EC2AF0E552E552E55207D005EC23F068
:10A21000AEC1E6FF3BEC2AF0E5520101786B796BA9
:10A220000F015E6B06D00101786B796B0F015E6BDD
:10A2300000D006D0B1EC39F003D0040EDB6A00D0B8
:10A24000040EDB5002E0B5EF5DF0010EF36E040E7C
:10A25000F3CFDBFF160E0101781902E1020E791926
:10A2600002E1A7EF5DF0150E0101781902E1020E7F
:10A27000791902E16EEF5DF0140E0101781902E127
:10A28000020E791902E141EF5DF0810E01017819AA
:10A2900002E1210E791902E1F4EF5CF0800E010178
:10A2A000781902E1210E791902E1F4EF5CF0100E49
:10A2B0000101781902E1020E791902E1A0EF5CF0C8
:10A2C000110E0101781902E1020E791902E1A0EFE5
:10A2D0005CF0130E0101781902E1020E791902E116
:10A2E00093EF5CF0170E0101781902E1020E791963
:10A2F00002E15CEF5CF0120E0101781902E1020E3E
:10A30000791902E125EF5CF06C0E0101781902E188
:10A31000030E791902E11DEF5CF0610E010178195D
:10A3200002E1030E791902E116EF5BF0650E0101FF
:10A33000781902E1030E791902E116EF5BF0690E5C
:10A340000101781902E1030E791902E116EF5BF0C1
:10A35000620E0101781902E1030E791902E116EF8C
:10A360005BF0660E0101781902E1030E791902E132
:10A3700016EF5BF06B0E0101781902E1030E7919FB
:10A3800002E116EF5BF0600E0101781902E1030EA5
:10A39000791902E1F3EF59F0640E0101781902E135
:10A3A000030E791902E1F3EF59F06D0E01017819EE
:10A3B00002E1030E791902E1F3EF59F06E0E01018B
:10A3C000781902E1030E791902E1F3EF59F0680EF2
:10A3D0000101781902E1030E791902E1F3EF59F056
:10A3E000630E0101781902E1030E791902E1F3EF1E
:10A3F00059F0670E0101781902E1030E791902E1A3
:10A40000F3EF59F06A0E0101781902E1030E791990
:10A4100002E1F3EF59F0330E0101781902E1010E68
:10A42000791902E1A9EF59F0320E0101781902E120
:10A43000010E791902E176EF59F0310E0101781918
:10A4400002E1010E791902E12BEF59F0300E010102
:10A45000781902E1010E791902E19CEF58F001012F
:10A46000785102E1130E791902E19CEF58F0260EA3
:10A470000101781902E1010E791902E19CEF58F00F
:10A48000600E0101781902E1120E791902E19CEFC8
:10A4900058F0120E0101781902E1010E791902E15A
:10A4A00064EF58F0100E0101781902E1010E7919DC
:10A4B00002E167EF57F0150E0101781902E1010E74
:10A4C000791902E167EF57F0140E0101781902E1E2
:10A4D000010E791902E167EF57F0110E01017819A9
:10A4E00002E1010E791902E167EF57F0130E010145
:10A4F000781902E1010E791902E167EF57F00D0EAC
:10A500000101781902E1010E791902E157EF57F0C4
:10A510000C0E0101781902E1010E791902E147EFF1
:10A5200057F0070E0101781902E1010E791902E1D5
:10A53000D8EF56F0090E0101781902E1010E7919E0
:10A5400002E1D8EF56F00B0E0101781902E1010E7D
:10A55000791902E1D8EF56F0060E0101781902E1EF
:10A56000010E791901E1BBD3080E0101781902E14E
:10A57000010E791901E1B3D30A0E0101781902E144
:10A58000010E791901E1ABD3300E0101781902E116
:10A59000020E791901E150D3310E0101781902E15F
:10A5A000020E791901E148D3320E0101781902E156
:10A5B000020E791901E140D3330E0101781902E14D
:10A5C000020E791901E138D3340E0101781902E144
:10A5D000020E791901E130D3350E0101781902E13B
:10A5E000020E791901E128D3360E0101781902E132
:10A5F000020E791901E120D3270E0101781902E139
:10A60000020E791901E108D32A0E0101781902E13D
:10A61000020E791901E1DBD2250E0101781902E160
:10A62000020E791901E1C3D2260E0101781902E167
:10A63000020E791901E19FD2210E0101781902E180
:10A64000010E791901E130D2170E0101781902E1EA
:10A65000010E791901E128D2190E0101781902E1E0
:10A66000010E791901E120D2230E0101781902E1CE
:10A67000010E791901E118D2250E0101781902E1C4
:10A68000010E791901E110D20101785102E1120E97
:10A69000791901E18AD1600E0101781902E1110EE8
:10A6A000791901E182D1800E0101781902E1110EC0
:10A6B000791901E17AD1200E0101781902E1120E17
:10A6C000791901E172D1400E0101781902E1120EEF
:10A6D000791901E16AD1200E0101781902E1010E18
:10A6E000791901E1E2D0160E0101781902E1010E9B
:10A6F000791901E1DAD0180E0101781902E1010E91
:10A70000791901E1D2D0220E0101781902E1010E7E
:10A71000791901E1CAD0240E0101781902E1010E74
:10A72000791901E1C2D00101785102E1020E7919D3
:10A7300001E188D0010E0101781902E1020E7919B8
:10A740001EE0020E0101781902E1020E791917E0EC
:10A75000030E0101781902E1020E791910E0040ECE
:10A760000101781902E1020E791909E0050E0101D3
:10A77000781902E1020E791902E0B2EF5DF0E66AA3
:10A78000E5EC2CF0E552E76E050EE7CFDBFF050E9A
:10A79000DB504AE1010E0101781902E1020E79193C
:10A7A00006E1C5C1E6FFA5EC6CF0E55234D0020E1F
:10A7B0000101781902E1020E79190AE10101C51DB2
:10A7C00001010517C5C1E6FFC5EC6CF0E55223D0C9
:10A7D000030E0101781902E1020E791906E1C5C1E3
:10A7E000E6FFE9EC6CF0E55216D0040E0101781991
:10A7F00002E1020E791906E1C5C1E6FF0DEC6DF02C
:10A80000E55209D00101C55101010513C5C1E6FF9B
:10A81000C5EC6CF0E552AEC1E6FFD2EC29F0E55292
:10A820000101786B796B0CD0050EDB50146E156A44
:10A83000FF0E141801E1155003E10101786B796BEB
:10A84000B5EF5DF00D0EE66E0F0EE66E080EE66ECD
:10A85000E3EC2BF0E552E552E552E76E050EE7CF4B
:10A86000DBFF050EDB5013E10D0EE66E0F0EE66EFC
:10A870005CEC6BF0E552E552000905E1AEC1E6FF84
:10A88000D2EC29F0E5520101786B796B0CD0050E02
:10A89000DB50146E156AFF0E141801E1155003E128
:10A8A0000101786B796BB5EF5DF00D0EE66E0F0E62
:10A8B000E66E4F0EE66E12EC2CF0E552E552E552D4
:10A8C000E76E050EE7CFDBFF050EDB5060E1240EDF
:10A8D0000101781902E1010E791941E0220E01010E
:10A8E000781902E1010E791931E0180E0101781989
:10A8F00002E1010E791921E0160E0101781902E139
:10A90000010E791911E0200E0101781902E1010E02
:10A91000791901E02DD00D0EE66E0F0EE66EBAEC41
:10A920006DF0E552E55224D00D0EE66E0F0EE66E88
:10A9300040EC6DF0E552E5521BD00D0EE66E0F0EA9
:10A94000E66E60EC6DF0E552E55212D00D0EE66E4B
:10A950000F0EE66E7AEC6DF0E552E55209D00D0E61
:10A96000E66E0F0EE66E9AEC6DF0E552E55200D001
:10A970000D0EE66E0F0EE66EAEC1E6FF60EC2AF03D
:10A98000E552E552E5520101786B796B0CD0050E6A
:10A99000DB50146E156AFF0E141801E1155003E127
:10A9A0000101786B796BB5EF5DF00D0EE66E0F0E61
:10A9B000E66E4F0EE66EA6EC2CF0E552E552E5523F
:10A9C000E76E050EE7CFDBFF050EDB505FE1400EC3
:10A9D0000101781902E1120E791940E0200E0101FF
:10A9E000781902E1120E791930E0800E0101781910
:10A9F00002E1110E791920E0600E0101781902E1DF
:10AA0000110E791910E00101785102E1120E791945
:10AA100001E02DD00D0EE66E0F0EE66EBAEC6DF075
:10AA2000E552E55224D00D0EE66E0F0EE66E40ECB8
:10AA30006DF0E552E5521BD00D0EE66E0F0EE66E80
:10AA400060EC6DF0E552E55212D00D0EE66E0F0E81
:10AA5000E66E7AEC6DF0E552E55209D00D0EE66E29
:10AA60000F0EE66E9AEC6DF0E552E55200D00D0E39
:10AA7000E66E0F0EE66EAEC1E6FF60EC2AF0E55220
:10AA8000E552E5520101786B796B0CD0050EDB5075
:10AA9000146E156AFF0E141801E1155003E101014F
:10AAA000786B796BB5EF5DF00101AD81250E010189
:10AAB000781902E1010E79194DE0230E0101781990
:10AAC00002E1010E79193AE0190E0101781902E14B
:10AAD000010E791927E0170E0101781902E1010E24
:10AAE000791914E0210E0101781902E1010E79199A
:10AAF00001E03CD0A80EE66E040EE66EAEC1E6FFA5
:10AB000060EC2AF0E552E552E55230D0580EE66E80
:10AB1000040EE66EAEC1E6FF60EC2AF0E552E552A7
:10AB2000E55224D06C0EE66E040EE66EAEC1E6FF72
:10AB300060EC2AF0E552E552E55218D0800EE66E40
:10AB4000040EE66EAEC1E6FF60EC2AF0E552E55277
:10AB5000E5520CD0940EE66E040EE66EAEC1E6FF32
:10AB600060EC2AF0E552E552E55200D00101786B25
:10AB7000796BB5EF5DF00101AD810101010E0A6F46
:10AB8000440EE66E010EE66E430EE66EE66AC1EC1A
:10AB90006AF0E552E552E552E552AEC1E6FFBBEC84
:10ABA00029F0E5520101786B796BB5EF5DF0010199
:10ABB000AD8101010A6B0101446BAEC1E6FFBBEC44
:10ABC00029F0E5520101786B796BB5EF5DF0030E6A
:10ABD000E66E7FEC2BF0E552E76E050EE7CFDBFF6C
:10ABE000050EDB500BE1BFC10BF1AEC1E6FFBBECC4
:10ABF00029F0E5520101786B796B0CD0050EDB5022
:10AC0000146E156AFF0E141801E1155003E10101DD
:10AC1000786B796BB5EF5DF00101AD81E668E7EC2B
:10AC200075F0E552AEC1E6FFD2EC29F0E552010124
:10AC3000786B796BB5EF5DF00101AD81360E0101E6
:10AC4000781902E1020E79193DE0350E01017819FB
:10AC500002E1020E791933E0340E0101781902E1A4
:10AC6000020E791929E0330E0101781902E1020E72
:10AC700079191FE0320E0101781902E1020E7919EB
:10AC800015E0310E0101781902E1020E79190BE08D
:10AC9000300E0101781902E1020E791901E015D098
:10ACA000B9EC6EF012D0D3EC6EF00FD0F6EC6EF083
:10ACB0000CD019EC6FF009D03CEC6FF006D05FECD3
:10ACC0006FF003D082EC6FF000D0AEC1E6FFD2ECA3
:10ACD00029F0E5520101786B796BB5EF5DF00D0E4F
:10ACE000E66E0F0EE66E4F0EE66EE3EC2BF0E552CD
:10ACF000E552E552E76E050EE7CFDBFF050EDB50B0
:10AD000049E10A0E0101781902E1010E791929E0E1
:10AD1000080E0101781902E1010E791915E0060EFD
:10AD20000101781902E1010E791901E027D00D0E19
:10AD3000E66E0F0EE66E82EC2DF0E552E552E76E00
:10AD4000050EE7CFDBFF1AD00D0EE66E0F0EE66E96
:10AD5000A1EC2DF0E552E552E76E050EE7CFDBFFE3
:10AD60000DD00D0EE66E0F0EE66EC4EC2DF0E55222
:10AD7000E552E76E050EE7CFDBFF00D0050EDB5096
:10AD800005E1AEC1E6FFD2EC29F0E5520101786B96
:10AD9000796B0CD0050EDB50146E156AFF0E14187B
:10ADA00001E1155003E10101786B796BB5EF5DF0BE
:10ADB0000D0EE66E0F0EE66E4F0EE66EE3EC2BF018
:10ADC000E552E552E552E76E050EE7CFDBFF050ED3
:10ADD000DB504FE10B0E0101781902E1010E7919E8
:10ADE00029E0090E0101781902E1010E791915E037
:10ADF000070E0101781902E1010E791901E027D04F
:10AE00000D0EE66E0F0EE66E76EC2FF0E552E55273
:10AE1000E76E050EE7CFDBFF1AD00D0EE66E0F0EC4
:10AE2000E66E96EC2FF0E552E552E76E050EE7CFA1
:10AE3000DBFF0DD00D0EE66E0F0EE66EB3EC2FF0BD
:10AE4000E552E552E76E050EE7CFDBFF00D0050EB9
:10AE5000DB500BE10D0EE66E0F0EE66EAEC1E6FFA7
:10AE600060EC2AF0E552E552E5520101786B796B0E
:10AE70000CD0050EDB50146E156AFF0E141801E19C
:10AE8000155003E10101786B796BB5EF5DF00101BD
:10AE9000AD8141ECAEF0000905E1AEC1E6FFD2ECB8
:10AEA00029F0E5520101786B796BB5EF5DF0010196
:10AEB000AD81E4ECAEF0000905E1AEC1E6FFD2ECF5
:10AEC00029F0E5520101786B796BB5EF5DF00D0E5D
:10AED000E66E0F0EE66E070EE66EE3EC2BF0E55223
:10AEE000E552E552E76E050EE7CFDBFF050EDB50BE
:10AEF00001E0DCD00B0EDB6A0D0EE66E0F0EE66E87
:10AF000066ECABF0E552E5520C0EF3CFDBFF0C0E16
:10AF1000DB50F36E0B0EDBCFF4FFF350F45C20E25A
:10AF20000B0EDB50EA6A0D0FE96E0F0EEA22EFCF2F
:10AF300016F0176A16BE176816C0E6FF17C0E6FFC0
:10AF4000D5EC17F0E552E552F3CF14F0F4CF15F03D
:10AF50001450151002E0050EDB680B0EDB2AD7D764
:10AF6000050EDB50146E156AFF0E141801E1155022
:10AF700071E0130E0101781902E1010E79195DE00B
:10AF8000110E0101781902E1010E791949E0150E3F
:10AF90000101781902E1010E79192FE0140E010167
:10AFA000781902E1010E791915E0100E01017819E6
:10AFB00002E1010E791901E04DD00D0EE66E0F0E83
:10AFC000E66E64EC84F0E552E552E76E050EE7CFDD
:10AFD000DBFF40D0010100510DE10D0EE66E0F0EBA
:10AFE000E66EA5EC84F0E552E552E76E050EE7CF7C
:10AFF000DBFF02D0050EDB682DD001018F510DE083
:10B000000D0EE66E0F0EE66EA5EC84F0E552E552ED
:10B01000E76E050EE7CFDBFF02D0050EDB681AD026
:10B020000D0EE66E0F0EE66EEAEC84F0E552E55288
:10B03000E76E050EE7CFDBFF0DD00D0EE66E0F0EAF
:10B04000E66ECFEC84F0E552E552E76E050EE7CFF1
:10B05000DBFF00D0050EDB50146E156AFF0E1418CE
:10B0600001E115501FE0050EDBCFE6FFE66AF40EA6
:10B07000E66E5F0EE66E010EE66E0D0EE66E0F0ECC
:10B08000E66E37ECB7F0146E070EE15E14500D0E4D
:10B09000E66E0F0EE66EAEC1E6FF60EC2AF0E552FA
:10B0A000E552E5520101786B796B0CD0050EDB504F
:10B0B000146E156AFF0E141801E1155003E1010129
:10B0C000786B796BB5EF5DF00D0EE66E0F0EE66EE8
:10B0D000020EE66EE3EC2BF0E552E552E552E76E28
:10B0E000050EE7CFDBFF050EDB5018E10D0EE66E17
:10B0F0000F0EE66E5FECB2F0E552E552F350E66EED
:10B1000012EC85F0E552000905E0AEC1E6FFD2EC95
:10B1100029F0E5520101786B796B0CD0050EDB50FC
:10B12000146E156AFF0E141801E1155003E10101B8
:10B13000786B796BB5EF5DF00101785102E1130E88
:10B14000791926E0600E0101781902E1120E7919D1
:10B150001FE0300E0101781902E1010E791908E0B3
:10B16000260E0101781902E1010E791901E020D0C3
:10B170000D0EE66E0F0EE66E4F0EE66E12EC2CF024
:10B18000E552E552E552E76E050EE7CFDBFF10D042
:10B190000D0EE66E0F0EE66E4F0EE66EA6EC2CF070
:10B1A000E552E552E552E76E050EE7CFDBFF00D032
:10B1B000050EDB5042E1260E0101781902E1010E75
:10B1C000791922E0600E0101781902E1120E791955
:10B1D0001BE0300E0101781902E1010E791907E038
:10B1E0000101785102E1130E791901E01AD00D0E18
:10B1F000E66E0F0EE66EC5EC14F0E552E552E76E12
:10B20000050EE7CFDBFF0DD00D0EE66E0F0EE66EDE
:10B21000EDEC6DF0E552E552E76E050EE7CFDBFF92
:10B2200000D0050EDB5005E1AEC1E6FFD2EC29F0FF
:10B23000E5520101786B796B0CD0050EDB50146E72
:10B24000156AFF0E141801E1155003E10101786B36
:10B25000796BB5EF5DF00D0EE66E0F0EE66E030E28
:10B26000E66EE3EC2BF0E552E552E552E76E050E93
:10B27000E7CFDBFF050EDB502BE10D0EE66E0F0E68
:10B28000E66E0D0EE66E0F0EE66E5FECB2F0E55266
:10B29000E552F3CF14F0F4CF15F014C0E6FF15C05B
:10B2A000E6FF4EEC15F0E552E552E552E552000995
:10B2B0000BE10D0EE66E0F0EE66EAEC1E6FF60EC22
:10B2C0002AF0E552E552E5520101786B796B0CD01A
:10B2D000050EDB50146E156AFF0E141801E11550AF
:10B2E00003E10101786B796BB5EF5DF00D0EE66E51
:10B2F0000F0EE66E4F0EE66EE3EC2BF0E552E552D4
:10B30000E552E76E050EE7CFDBFF050EDB5013E1DC
:10B310000D0EE66E0F0EE66E07EC15F0E552E552E7
:10B32000000905E1AEC1E6FFD2EC29F0E5520101CA
:10B33000786B796B0CD0050EDB50146E156AFF0E1E
:10B34000141801E1155003E10101786B796BB5EF39
:10B350005DF00D0EE66E0F0EE66E4F0EE66EE3EC40
:10B360002BF0E552E552E552E76E050EE7CFDBFF25
:10B37000050EDB502BE10D0EE66E0F0EE66E0D0E88
:10B38000E66E0F0EE66E5FECB2F0E552E552F3CFDB
:10B3900014F0F4CF15F014C0E6FF15C0E6FF8FECF3
:10B3A00015F0E552E552E552E55200090BE10D0EAC
:10B3B000E66E0F0EE66EAEC1E6FF60EC2AF0E552D7
:10B3C000E552E5520101786B796B0CD0050EDB502C
:10B3D000146E156AFF0E141801E1155003E1010106
:10B3E000786B796BC2D3010EE66E7FEC2BF0E552E1
:10B3F000E76E050EE7CFDBFF050EDB5001E009D15C
:10B400000101080EBF5D000EC05901E3FED00A0E17
:10B410000101BF25E96E090E0101C021EA6EEF505E
:10B420000101BF6FC06B010EBFC1E7FFE75204E02F
:10B43000E846FE0BE706FCE1E76E0B0EE7CFDBFF0D
:10B44000BFC1E6FF5FEC21F0E552E76E0C0EE7CFDF
:10B45000DBFF6A0E0101781902E1030E791901E19F
:10B46000C9D0670E0101781902E1030E791901E1D3
:10B47000B1D0630E0101781902E1030E791901E1DF
:10B4800099D0680E0101781902E1030E791901E1E2
:10B4900087D0640E0101781902E1030E79194BE09F
:10B4A0006E0E0101781902E1030E791944E0600E75
:10B4B0000101781902E1030E791908E06D0E01010E
:10B4C000781902E1030E791901E09FD00B0EDB50D1
:10B4D00001016D13600E0101781902E1030E791963
:10B4E00005E10B0EDB1C01016F1704D00B0EDB50C6
:10B4F00001016F13050EF36E0C0EDBCFF4FFF3505A
:10B50000F45C13E20C0EDB50050DF3CF14F0F4CF16
:10B5100015F0880E1426060E152214C0E6FF15C07D
:10B52000E6FFE8EC7EF0E552E552AEC1E6FFBBEC8B
:10B5300029F0E5526AD00B0EDB5001016E13640E48
:10B540000101781902E1030E791905E10B0EDB1CEC
:10B5500001016F1704D00B0EDB5001016F13050EB4
:10B56000F36E0C0EDBCFF4FFF350F45C13E20C0E21
:10B57000DB50050DF3CF14F0F4CF15F0880E142630
:10B58000060E152214C0E6FF15C0E6FFE8EC7EF0BB
:10B59000E552E552AEC1E6FFBBEC29F0E55235D0ED
:10B5A0000B0EDB5001017013AEC1E6FFBBEC29F0BE
:10B5B000E5522BD0BFC1E6FFD7EC32F0E552BFC158
:10B5C000E6FF15EC33F0E552AEC1E6FFD2EC29F010
:10B5D000E5521BD0BFC1E6FFF5EC32F0E552BFC12A
:10B5E000E6FF15EC33F0E552AEC1E6FFD2EC29F0F0
:10B5F000E5520BD0BFC1E6FF33EC33F0E552AEC1EC
:10B60000E6FFD2EC29F0E55200D00101786B796BAE
:10B610000CD0050EDB50146E156AFF0E141801E1F4
:10B62000155003E10101786B796B9FD2010EE66E34
:10B630007FEC2BF0E552E76E050EE7CFDBFF050E42
:10B64000DB5001E0EDD00101080EBF5D000EC059D6
:10B6500001E3E2D00A0E0101BF25E96E090E0101E6
:10B66000C021EA6EEF500101BF6FC06B010EBFC178
:10B67000E7FFE75204E0E846FE0BE706FCE1E76E71
:10B680000B0EE7CFDBFFBFC1E6FF5FEC21F0E55219
:10B69000E76E0C0EE7CFDBFF0F0109511AE00F0137
:10B6A0000C51146E156A1450800B01E1A9D0980E4C
:10B6B0000F01091501E0A4D00A0E0101BF25E96EB2
:10B6C000090E0101C021EA6EEF500101AE5D01E0FB
:10B6D00097D00F01010E5D6F6B0E0101781902E129
:10B6E000030E791901E185D0660E0101781902E196
:10B6F000030E791901E177D0620E0101781902E198
:10B70000030E79196AE0690E0101781902E1030E4E
:10B71000791959E0650E0101781902E1030E7919D2
:10B720002DE0610E0101781902E1030E791901E0A3
:10B7300066D00B0EDB1C01016D17050EF36E0C0EAF
:10B74000DBCFF4FFF350F45C13E20C0EDB50050D7D
:10B75000F3CF14F0F4CF15F0880E1426060E152240
:10B7600014C0E6FF15C0E6FFE8EC7EF0E552E552B6
:10B77000AEC1E6FFBBEC29F0E55241D00B0EDB1C5D
:10B7800001016E17050EF36E0C0EDBCFF4FFF350C4
:10B79000F45C13E20C0EDB50050DF3CF14F0F4CF84
:10B7A00015F0880E1426060E152214C0E6FF15C0EB
:10B7B000E6FFE8EC7EF0E552E552AEC1E6FFBBECF9
:10B7C00029F0E5521CD00B0EDB1C01017017AEC135
:10B7D000E6FFBBEC29F0E55212D0BFC1E6FF02EC58
:10B7E00032F0E5520CD0BFC1E6FF49EC32F0E55231
:10B7F00006D0BFC1E6FF90EC32F0E55200D00CD08D
:10B8000009CFE6FFAEC1E6FF00EC2AF0E552E552B3
:10B810000101AD9305EC23F00101786B796B0CD03D
:10B82000050EDB50146E156AFF0E141801E1155059
:10B8300003E10101786B796B98D10101AD8153EC83
:10B8400033F00101786B796B90D10D0EE66E0F0E1F
:10B85000E66E080EE66EE3EC2BF0E552E552E5529B
:10B86000E76E050EE7CFDBFF050EDB5018E10D0E8E
:10B87000E66E0F0EE66E46EC81F0E552E552E76E9D
:10B88000050EE7CFDBFF050EDB5005E1AEC1E6FF9D
:10B89000BBEC29F0E5520101786B796B0CD0050EF9
:10B8A000DB50146E156AFF0E141801E1155003E108
:10B8B0000101786B796B59D10D0EE66E0F0EE66EB5
:10B8C0000A0EE66EE3EC2BF0E552E552E552E76E28
:10B8D000050EE7CFDBFF050EDB5018E10D0EE66E1F
:10B8E0000F0EE66EB0EC81F0E552E552E76E050E04
:10B8F000E7CFDBFF050EDB5005E1AEC1E6FFBBEC99
:10B9000029F0E5520101786B796B0CD0050EDB5004
:10B91000146E156AFF0E141801E1155003E10101C0
:10B92000786B796B22D10101AD812DEC82F0AEC133
:10B93000E6FFBBEC29F0E5520101786B796B15D17C
:10B940000D0EE66E0F0EE66E0A0EE66EE3EC2BF0C1
:10B95000E552E552E552E76E050EE7CFDBFF050E37
:10B96000DB5035E1110E0101781902E1020E79195F
:10B9700015E0100E0101781902E1020E791901E0BB
:10B980001AD00D0EE66E0F0EE66E6AEC82F0E552EE
:10B99000E552E76E050EE7CFDBFF0DD00D0EE66E2C
:10B9A0000F0EE66EC9EC82F0E552E552E76E050E29
:10B9B000E7CFDBFF00D0050EDB5005E1AEC1E6FFAF
:10B9C000D2EC29F0E5520101786B796B0CD0050EB1
:10B9D000DB50146E156AFF0E141801E1155003E1D7
:10B9E0000101786B796BC1D0010EE66E7FEC2BF014
:10B9F000E552E76E050EE7CFDBFF050EDB5034E1C5
:10BA0000800E0101781902E1210E791915E0810EED
:10BA10000101781902E1210E791901E019D0010E16
:10BA2000E66EBFC1E6FF03EC83F0E552E552E76E38
:10BA3000050EE7CFDBFF0CD0E66ABFC1E6FF03ECE3
:10BA400083F0E552E552E76E050EE7CFDBFF00D04D
:10BA5000050EDB5005E1AEC1E6FFBBEC29F0E55277
:10BA60000101786B796B0CD0050EDB50146E156AF2
:10BA7000FF0E141801E1155003E10101786B796B99
:10BA800074D0010EE66E7FEC2BF0E552E76E050EEA
:10BA9000E7CFDBFF050EDB5014E10101050EBF5DB2
:10BAA000000EC0590AE2BFC1E6FF0AEC3BF0E552C6
:10BAB000AEC1E6FFBBEC29F0E5520101786B796B72
:10BAC0000CD0050EDB50146E156AFF0E141801E140
:10BAD000155003E10101786B796B47D0010EE66EDA
:10BAE0007FEC2BF0E552E76E050EE7CFDBFF050E8E
:10BAF000DB5020E101010051146E156A0101145060
:10BB0000BF5D1550C05912E20A0E0101BF25E96E52
:10BB1000090E0101C021EA6EEF50E66E25EC3BF004
:10BB2000E552AEC1E6FFBBEC29F0E5520101786BAE
:10BB3000796B0CD0050EDB50146E156AFF0E1418CD
:10BB400001E1155003E10101786B796B0ED0E0EC57
:10BB50003AF0AEC1E6FFBBEC29F0E5520101786B8B
:10BB6000796B03D0040EDB6A00D0040EDB5002E0D8
:10BB700021EF67F0010EF36E040EF3CFDBFFFE0E34
:10BB80000101781902E1E868791902E117EF67F01D
:10BB9000760E0101781902E1030E791902E1ECEF4A
:10BBA00066F0610E0101781902E1370E791902E1A0
:10BBB000ECEF66F0770E0101781902E1030E7919B6
:10BBC00002E1ECEF66F0710E0101781902E1370E27
:10BBD000791902E1ECEF66F0750E0101781902E1C6
:10BBE000030E791902E1DCEF66F0850E0101781988
:10BBF00002E1030E791902E111EF66F0860E0101F0
:10BC0000781902E1030E791902E111EF66F09D0E39
:10BC10000101781902E1020E791902E1DCEF65F009
:10BC20009C0E0101781902E1020E791902E1CBEFB5
:10BC300065F09B0E0101781902E1020E791902E10B
:10BC4000BEEF65F09A0E0101781902E1020E791932
:10BC500002E18AEF65F0990E0101781902E1020E06
:10BC6000791902E17FEF65F0980E0101781902E180
:10BC7000020E791902E13CEF65F0600E01017819BE
:10BC800002E1020E791902E139EF65F0210E01019E
:10BC9000781902E1020E791902E1DBEF64F0220E5D
:10BCA0000101781902E1020E791902E1DBEF64F07B
:10BCB000290E0101781902E1020E791902E1DBEF88
:10BCC00064F0200E0101781902E1020E791902E1F7
:10BCD000B4EF64F0190E0101781902E1020E79192E
:10BCE00002E192EF64F0240E0101781902E1020EE4
:10BCF000791902E18FEF64F0230E0101781902E156
:10BD0000020E791902E117EF64F0710E0101781942
:10BD100002E1030E791902E1B7EF63F0700E010141
:10BD2000781902E1030E791902E155EF63F03A0E3A
:10BD30000101781902E1010E791902E133EF63F094
:10BD4000390E0101781902E1010E791902E10CEFB7
:10BD500063F00101785102E1010E791902E1F0EF7F
:10BD600062F0010E0101781902E1010E791902E178
:10BD7000C8EF62F0050E0101781902E1010E791990
:10BD800001E1F6D3030E0101781902E1010E7919E0
:10BD900001E1DED3040E0101781902E1010E7919E7
:10BDA00001E1C6D3020E0101781902E1010E7919F1
:10BDB00001E1AED3450E0101781902E1030E7919B4
:10BDC00001E1FCD2460E0101781902E1030E791956
:10BDD00001E1F4D2440E0101781902E1030E791950
:10BDE00001E1ECD2500E0101781902E1020E79193D
:10BDF00001E1E4D2510E0101781902E1020E791934
:10BE000001E1DCD2530E0101781902E1020E791929
:10BE100001E1D4D2410E0101781902E1030E791932
:10BE200001E16AD2420E0101781902E1030E79198B
:10BE300001E162D2400E0101781902E1030E791985
:10BE400001E15AD2520E0101781902E1020E79196C
:10BE500001E152D2540E0101781902E1020E791962
:10BE600001E14AD2380E0101781902E1010E791977
:10BE700001E13BD2370E0101781902E1010E791977
:10BE800001E12BD2360E0101781902E1010E791978
:10BE900001E11BD2350E0101781902E1010E791979
:10BEA00001E10BD2340E0101781902E1010E79197A
:10BEB00001E1F5D1060E0101781901E1795101E1A5
:10BEC000E0D1040E0101781901E1795101E1A2D11B
:10BED000170E0101781901E1795101E175D1160EB2
:10BEE0000101781901E1795101E154D1150E0101E7
:10BEF000781901E1795101E11DD1140E0101781980
:10BF000001E1795101E1E1D0130E0101781901E15C
:10BF1000795101E1CED0120E0101781901E1795178
:10BF200001E1BBD0110E0101781901E1795101E164
:10BF3000A8D0100E0101781901E1795101E195D0E5
:10BF4000070E0101781901E1795101E182D0050E56
:10BF50000101781901E1795170E0020E01017819AF
:10BF600001E1795162E0340E0101781902E1030E1A
:10BF700079191DE0350E0101781902E1030E7919D6
:10BF800016E0030E0101781901E1795110E03C0E31
:10BF90000101781902E1030E791909E03D0E010152
:10BFA000781902E1030E791902E01EEF67F0010132
:10BFB000AD813D0E0101781902E1030E791928E0E7
:10BFC0003C0E0101781902E1030E79191EE0030EFF
:10BFD0000101781901E1795115E0350E0101781957
:10BFE00002E1030E79190BE0340E0101781902E128
:10BFF000030E791901E00FD04AEC27F00CD06FEC5A
:10C0000027F009D001017A6B06D091EC35F003D00E
:10C010009CEC35F000D0AEC1E6FFBBEC29F0E55258
:10C020000101786B796B21EF67F00101786B796B17
:10C030000101010E7A6F21EF67F00101AD81AEC100
:10C04000E6FFC1EC28F0E5520101786B796B21EF36
:10C0500067F00101AD81AEC1E6FFAAEC29F0E5521F
:10C060000101786B796B21EF67F00101AD81AEC101
:10C07000E6FFFFEC28F0E5520101786B796B21EFC8
:10C0800067F00101AD81AEC1E6FF47EC29F0E55252
:10C090000101786B796B21EF67F00101AD81AEC1D1
:10C0A000E6FF5AEC29F0E5520101786B796B21EF3C
:10C0B00067F00101AD81AEC1E6FF6DEC29F0E552FC
:10C0C0000101786B796B21EF67F0010EE66E7FEC72
:10C0D0002BF0E552E76E050EE7CFDBFF050EDB50D8
:10C0E0001BE101010051146E156A01011450BF5D7E
:10C0F0001550C0590DE2200EE66EBFC1E6FFD5EC2B
:10C1000018F0E552E552AEC1E6FFBBEC29F0E5526E
:10C110000101786B796B0CD0050EDB50146E156A3B
:10C12000FF0E141801E1155003E10101786B796BE2
:10C1300021EF67F0010EE66E7FEC2BF0E552E76E23
:10C14000050EE7CFDBFF050EDB5016E101010051C4
:10C15000146E156A01011450BF5D1550C05908E2F4
:10C16000BFC1E6FFAEC1E6FF80EC29F0E552E55223
:10C170000101786B796B0CD0050EDB50146E156ADB
:10C18000FF0E141801E1155003E10101786B796B82
:10C1900021EF67F00101AD810D0EE66E0F0EE66E28
:10C1A00003ECB7F0E552E5520D0EE66E0F0EE66EAB
:10C1B000AEC1E6FF60EC2AF0E552E552E55201011E
:10C1C000786B796B21EF67F00101AD8130EC85F080
:10C1D000E66EE66A330EE66E610EE66E010EE66E00
:10C1E0000D0EE66E0F0EE66E37ECB7F0146E070E0E
:10C1F000E15E14500D0EE66E0F0EE66EAEC1E6FF68
:10C2000060EC2AF0E552E552E5520101786B796B5A
:10C2100021EF67F00101AD810101886BE66AE66AF2
:10C22000FBEC05F0E552E552E66A010EE66EFBEC2A
:10C2300005F0E552E552E66A020EE66EFBEC05F00B
:10C24000E552E552E66A030EE66EFBEC05F0E552B8
:10C25000E552E66A040EE66EFBEC05F0E552E552A7
:10C26000E66A050EE66EFBEC05F0E552E552AEC15E
:10C27000E6FFD2EC29F0E5520101786B796B21EFF2
:10C2800067F00101AD810101876BAEC1E6FFD2EC21
:10C2900029F0E5520101786B796B21EF67F001011C
:10C2A000AD810101776BAEC1E6FFBBEC29F0E55231
:10C2B0000101786B796B21EF67F00601030EFF6FC8
:10C2C0000101786B796B21EF67F00601010EFF6FBA
:10C2D0000101786B796B21EF67F00601020EFF6FA9
:10C2E0000101786B796B21EF67F00601FF690101AD
:10C2F000786B796B21EF67F00101AD81540E01017C
:10C30000781902E1020E791947E0520E01017819FD
:10C3100002E1020E79193BE0400E0101781902E1B9
:10C32000030E791928E0420E0101781902E1030E8B
:10C33000791914E0410E0101781902E1030E79190F
:10C3400001E02FD0E66AAEC1E6FF1CEC34F0E55206
:10C35000E552E76E0B0EE7CFDBFF23D0010EE66E52
:10C36000AEC1E6FF1CEC34F0E552E552E76E0B0E71
:10C37000E7CFDBFF16D0AEC1E6FF7DEC34F0E5522F
:10C38000E76E0B0EE7CFDBFF0B0EDB6A0AD0DFECAC
:10C3900036F00B0EDB6A05D00101AB6B0B0EDB6ACE
:10C3A00000D00B0EDB5005E1AEC1E6FFBBEC29F07F
:10C3B000E5520101786B796B21EF67F0010EE66EB3
:10C3C0007FEC2BF0E552E76E050EE7CFDBFF050EA5
:10C3D000DB5001E08FD001010051146E156A01019C
:10C3E0001450BF5D1550C05901E380D00A0E010101
:10C3F000BF25E96E090E0101C021EA6EEF5001016F
:10C40000BF6FC06B530E0101781902E1020E79195A
:10C410005BE0510E0101781902E1020E79194AE040
:10C42000500E0101781902E1020E791939E0440E2B
:10C430000101781902E1030E791928E0460E010185
:10C44000781902E1030E791914E0450E01017819FB
:10C4500002E1030E791901E041D0E66ABFC1E6FFAF
:10C460001CEC34F0E552E552E76E0B0EE7CFDBFF34
:10C4700035D0010EE66EBFC1E6FF1CEC34F0E5528C
:10C48000E552E76E0B0EE7CFDBFF28D0BFC1E6FF1A
:10C490007DEC34F0E552E76E0B0EE7CFDBFF1ED0EC
:10C4A000BFC1E6FFA8EC36F0E552E76E0B0EE7CF12
:10C4B000DBFF14D0BFC1E6FFC3EC36F0E552E76EF8
:10C4C0000B0EE7CFDBFF0AD0BFC1E6FFFCEC36F076
:10C4D000E552E76E0B0EE7CFDBFF00D00B0EDB5013
:10C4E00005E1AEC1E6FFBBEC29F0E5520101786B36
:10C4F000796B0CD0050EDB50146E156AFF0E141804
:10C5000001E1155003E10101786B796B21EF67F0D0
:10C510000101AD81FDEC6AF0000905E1AEC1E6FF65
:10C52000D2EC29F0E5520101786B796B21EF67F0CD
:10C530000101AD810BEC6BF0000905E1AEC1E6FF36
:10C54000D2EC29F0E5520101786B796B21EF67F0AD
:10C550000101AD811AEC6BF0000905E1AEC1E6FF07
:10C56000D2EC29F0E5520101786B796B21EF67F08D
:10C570000101AD8124EC6BF0000905E1AEC1E6FFDD
:10C58000D2EC29F0E5520101786B796B21EF67F06D
:10C590000101AD8135EC7BF000090FE0EC0EE66E99
:10C5A0005F0EE66E010EE66EAEC1E6FF6EEC2AF09F
:10C5B000E552E552E552E5520ED0E20EE66E5F0E10
:10C5C000E66E010EE66EAEC1E6FF6EEC2AF0E552B5
:10C5D000E552E552E5520101786B796B21EF67F086
:10C5E0000101AD8101018F5112E00101746B74C131
:10C5F000E6FF550EE66E030EE66E84EC6AF0E55239
:10C60000E552E552AEC1E6FFD2EC29F0E552010158
:10C61000786B796B21EF67F0020EE66E7FEC2BF002
:10C62000E552E76E050EE7CFDBFF050EDB500EE1AE
:10C63000BFC1E6FF30EC6DF0E552AEC1E6FFD2ECD3
:10C6400029F0E5520101786B796B0CD0050EDB50B7
:10C65000146E156AFF0E141801E1155003E1010173
:10C66000786B796BEED34F0EE66EE66AB20EE66E2D
:10C670005F0EE66E010EE66E0D0EE66E0F0EE66EB6
:10C68000F8ECABF0146E070EE15E14500D0EE66E82
:10C690000F0EE66EAEC1E6FF60EC2AF0E552E55201
:10C6A000E5520101786B796BCCD30D0EE66E0F0E5F
:10C6B000E66E040EE66EE3EC2BF0E552E552E55231
:10C6C000E76E050EE7CFDBFF050EDB5043E1300ED2
:10C6D0000F010D5D146E080E145C1EE20E0EE66E68
:10C6E0000F0EE66E5FECB2F0E552E552F350E66EE7
:10C6F000300E0F010D5DEA6A0A0FE96E090EEA229B
:10C70000EF50E66E8EEC37F0E552E552AEC1E6FF33
:10C71000BBEC29F0E5521AD0300E0F010D5D080870
:10C7200015E10E0EE66E0F0EE66E5FECB2F0E5520E
:10C73000E552F350E66E080EE66E8EEC37F0E552E9
:10C74000E552AEC1E6FFBBEC29F0E5520101786B82
:10C75000796B0CD0050EDB50146E156AFF0E1418A1
:10C7600001E1155003E10101786B796B6AD30D0E7D
:10C77000E66E0F0EE66E030EE66EE3EC2BF0E5526E
:10C78000E552E552E76E050EE7CFDBFF050EDB5005
:10C7900041E1300E0F010D5D146E080E145C1DE2B8
:10C7A000300E0F010F5DE66E300E0F010E5DE66E6E
:10C7B000300E0F010D5DEA6A0A0FE96E090EEA22DA
:10C7C000EF50E66ECEEC37F0E552E552E552AEC1E1
:10C7D000E6FFBBEC29F0E55219D0300E0F010D5DDC
:10C7E000080814E1300E0F010F5DE66E300E0F01E8
:10C7F0000E5DE66E080EE66ECEEC37F0E552E552C1
:10C80000E552AEC1E6FFBBEC29F0E5520101786BC1
:10C81000796B0CD0050EDB50146E156AFF0E1418E0
:10C8200001E1155003E10101786B796B0AD30D0E1C
:10C83000E66E0F0EE66E050EE66EE3EC2BF0E552AB
:10C84000E552E552E76E050EE7CFDBFF050EDB5044
:10C8500059E10D0EE66E0F0EE66E66ECABF0E5529A
:10C86000E552F3CF14F0F4CF15F0020ED880145433
:10C87000000E155447E2300E0F010D5D146E080EC8
:10C88000145C1DE20F0EE66E0F0EE66E5FECB2F06A
:10C89000E552E552F350E66E300E0F010E5DE66E86
:10C8A000300E0F010D5DE66EB2EC38F0E552E55248
:10C8B000E552AEC1E6FFD2EC29F0E5521FD0300EB2
:10C8C0000F010D5D08081AE10F0EE66E0F0EE66E01
:10C8D0005FECB2F0E552E552F350E66E300E0F0118
:10C8E0000E5DE66E080EE66EB2EC38F0E552E552EB
:10C8F000E552AEC1E6FFD2EC29F0E5520101786BBA
:10C90000796B0CD0050EDB50146E156AFF0E1418EF
:10C9100001E1155003E10101786B796B92D2DFECF4
:10C9200038F08FD2010EE66E7FEC2BF0E552E76E09
:10C93000050EE7CFDBFF050EDB5009E1BFC1E6FFC7
:10C9400017EC24F0E5520101786B796B0CD0050EE1
:10C95000DB50146E156AFF0E141801E1155003E147
:10C960000101786B796B6DD2010EE66E7FEC2BF0D6
:10C97000E552E76E050EE7CFDBFF050EDB500EE15B
:10C98000BFC1E6FF54EC24F0E552AEC1E6FFBBECBC
:10C9900029F0E5520101786B796B0CD0050EDB5064
:10C9A000146E156AFF0E141801E1155003E1010120
:10C9B000786B796B46D2070EE66E7FEC2BF0E55272
:10C9C000E76E050EE7CFDBFF050EDB5045E1290ED4
:10C9D0000101781902E1020E79192EE0220E0101FF
:10C9E000781902E1020E791918E0210E0101781977
:10C9F00002E1020E791901E02BD00101A00EBF5D0A
:10CA00000F0EC05909E2BFC15DF1C0C15EF1AEC1F8
:10CA1000E6FFBBEC29F0E5521BD00101FF0ED880E8
:10CA2000BF55000EC05507E3BFC15FF1AEC1E6FFC1
:10CA3000BBEC29F0E5520CD0BFC1E6FFC0C1E6FF58
:10CA4000AEC1E6FF52EC2AF0E552E552E55200D0C5
:10CA50000101786B796B0CD0050EDB50146E156AF2
:10CA6000FF0E141801E1155003E10101786B796B99
:10CA7000E8D1E5EC3BF0E5D1010EE66E7FEC2BF062
:10CA8000E552E76E050EE7CFDBFF050EDB502AE12E
:10CA90000101080EBF5D000EC05920E2450EE66E92
:10CAA0000D0EE66EA6EC00F0E552E55206C09AF1D6
:10CAB00007C09BF108C09CF109C09DF1010EBFC1E8
:10CAC000E7FFE75204E0E846FE0BE706FCE1010160
:10CAD000996FAEC1E6FFBBEC29F0E5520101786B1E
:10CAE000796B0CD0050EDB50146E156AFF0E14180E
:10CAF00001E1155003E10101786B796BA2D10101CD
:10CB0000996BAEC1E6FFBBEC29F0E5520101786BF1
:10CB1000796B97D1010EE66EE5EC2CF0E552E76EED
:10CB2000050EE7CFDBFF050EDB501BE1450EE66E81
:10CB30000D0EE66EA6EC00F0E552E55206C09FF140
:10CB400007C0A0F108C0A1F109C0A2F1C5C19EF1C2
:10CB5000AEC1E6FFBBEC29F0E5520101786B796BC1
:10CB60000CD0050EDB50146E156AFF0E141801E18F
:10CB7000155003E10101786B796B63D10101AD813F
:10CB800001019E6BAEC1E6FFBBEC29F0E55201014D
:10CB9000786B796B56D10101AD810801B46B080146
:10CBA000B36B0801B96BAEC1E6FFBBEC29F0E552EF
:10CBB0000101786B796B45D10101AD81B40EE66E50
:10CBC000080EE66E2A0EE66E030EE66EC1EC6AF003
:10CBD000E552E552E552E552B30EE66E080EE66EFA
:10CBE000290EE66E030EE66EC1EC6AF0E552E552E0
:10CBF000E552E552B90EE66E080EE66E2F0EE66EB1
:10CC0000030EE66EC1EC6AF0E552E552E552E552DC
:10CC1000AEC1E6FFBBEC29F0E5520101786B796B00
:10CC200010D10101ADB102D00F015E6B0F015E5159
:10CC3000020A01E1A2D0020A01E0BDD0860E010184
:10CC4000781902E1030E79191AE0850E01017819AD
:10CC500002E1030E791901E025D0E66A0D0EE66EB9
:10CC60000F0EE66E110EE66E93EC2AF0E552E552D9
:10CC7000E552E552E76E050EE7CFDBFF13D071C139
:10CC8000E6FF0D0EE66E0F0EE66E110EE66E16EC6A
:10CC90002BF0E552E552E552E552E76E050EE7CF7F
:10CCA000DBFF00D0050EDB5059E10DCF16F0176AFF
:10CCB00016BE176816C0E6FF17C0E6FFC3EC17F0F4
:10CCC000E552E552F3CF14F0F4CF15F014501510DF
:10CCD00006E0300E0F010D5D0F015F6F02D00F01F6
:10CCE0005F69080E0F015F5D09E20F015F51EA6A9B
:10CCF0000A0FE96E090EEA22EFCF5FFF0101005132
:10CD00000F015F5D26E2010E5FCFE7FFE75204E00F
:10CD1000E846FE0BE706FCE1146EB3C1E9FFB4C1BF
:10CD2000EAFF020EEB50141414E001016D510101F1
:10CD30006E11156E010E5FCFE7FFE75204E0E84683
:10CD4000FE0BE706FCE1151404E10F01020E5E6F15
:10CD500004D00101786B796B2ED00FD0050EDB501B
:10CD6000146E156AFF0E141801E1155005E101015A
:10CD7000786B796B20D001D01ED0250EE66E5FCF88
:10CD8000E6FF20EC19F0E552E552F35013E10E0EE8
:10CD9000E66E0F0EE66E5FCFE6FF4DEC7EF0E552DD
:10CDA000E552E552AEC1E6FFBBEC29F0E5520101C8
:10CDB000786B796B00D045D00101AD81A388A38A3F
:10CDC0000201010EFF6FAEC1E6FFBBEC29F0E55298
:10CDD0000101786B796B35D00D0EE66E0F0EE66EA5
:10CDE00078C1E6FF79C1E6FF35EC3BF0E552E5524C
:10CDF000E552E552E76E050EE7CFDBFF050EDB508F
:10CE000009E1AEC1E6FFBBEC29F0E5520101786B08
:10CE1000796B0CD0050EDB50146E156AFF0E1418DA
:10CE200001E1155003E10101786B796B0AD0010132
:10CE3000AD81FF000101786B796B03D0040EDB6AD2
:10CE400000D0040EDB5007E10101786B796B010122
:10CE5000AD6B05EC23F00101ADA10DD001017851BE
:10CE600001E1795101E006D00101B25102E1010175
:10CE7000AD9100D009D001017851791105E1070188
:10CE8000000E646F070E656F010E0101AD1508E11C
:10CE90000101B25105E10701005102E043EF3CF00E
:10CEA000070100510EE1010E0101AD150AE1060175
:10CEB000FE5107E1030E0101B21503E10101010E6C
:10CEC000756F130EE15C02E2E16AE552E16EE55234
:10CED000E7CFD9FF1200C3EC85F00B0EE1266FEC13
:10CEE00086F0070E06C0DBFF080E07C0DBFF090E49
:10CEF00008C0DBFF0A0E09C0DBFF0101995114E0F5
:10CF0000B1EC8BF09A51EE5C146E9B51EE58156E9D
:10CF10009C51EE58166E9D51EE58176ED8802C0E0F
:10CF200018EC8CF001E2996B9E5111E0B1EC8BF0A2
:10CF30009F51EE5C146EA051EE58156EA151EE5843
:10CF4000166EA251EE58D2EC88F001E29E6B0051B1
:10CF5000EFEC8DF0F4EC88F0BCEC88F003E0C5EC6D
:10CF600089F0FDE1BDEC87F000C1DFFFDF5001E19A
:10CF70008AD168EC8FF001017A5106E04DEC8EF019
:10CF8000EF9E060EDB6A77D15DEC91F003E1BDEC1C
:10CF900094F00EE17AEC8BF002E0000E01D0010E6D
:10CFA00015148B03F31C146EBDEC94F0141439E0CB
:10CFB000010EF36E060EF3CFDBFFDB5011E020EC29
:10CFC00093F0EF1C146E030EDB50AF15141408E041
:10CFD00020EC93F0EFCF15F0941DAF15151421E060
:10CFE00015EC86F060EC8CF011E104511915156E0A
:10CFF0000351181501111510146EBDEC94F01414A2
:10D0000005E178EC88F036C1EFFF0DD015EC86F025
:10D01000090E77EC8DF0E66E78EC88F08EEC87F0F8
:10D0200002D0060EDB6A060EDB5011E17AEC8BF0C3
:10D0300002E0000E01D0010E15148B03F3CF14F0A3
:10D04000BDEC94F0F31403E078EC88F0EF6A060E80
:10D05000DB5071E1030EDB5099156DE115EC86F0A4
:10D06000AFEC93F0DF0B41E1B2511EE0010EDB505B
:10D07000765D3BE00A5118E0AC5116E15DEC91F0B1
:10D0800013E1010EDB5003E1080EAE5D2EE020EC53
:10D0900093F058EC8CF076C1E7FFE75203E0A8EC80
:10D0A00088F0FDE1141421E10101A95128E02BECE5
:10D0B00094F001510211E552E71421E020EC93F0C5
:10D0C000EFCF16F0010E76C1E7FFE75203E0A8ECC0
:10D0D00088F0FDE1156E080E0101AE5D02E0000E64
:10D0E00001D0010E151016140AE00101A5512B11F3
:10D0F000E81C176E030EDB50031517141CE020EC20
:10D1000093F0EFCF18F030EC8DF003E0A8EC88F04E
:10D11000FDE1181407E0030E0101AD1503E05DEC1D
:10D1200091F009E015EC86F008EC95F0220B0CE08C
:10D130005DEC91F009E03FEC8DF006E115EC86F036
:10D140000A0E43EC92F01BD015EC86F077EC8DF0D4
:10D15000010B08E03FEC8DF005E178EC88F0EF5032
:10D160000EE107D078EC88F0EF5003E03FEC8DF053
:10D1700006E015EC86F00A0EF4EC85F0EF6A030E7B
:10D18000DB500801B91505E1030EDB1C0801F1179E
:10D1900051D0E4EC8BF004E0010E0801BB1503E173
:10D1A000060EDB5015E1030EDB1C0801F117B7C8B2
:10D1B000E6FFB8C8E6FF010E7FEC87F0B80E142634
:10D1C000000EFCEC85F069EC00F0E552E55230D041
:10D1D00068EC8CF0B80E1626000EA7EC94F06CEC00
:10D1E00093F028E1030EDB500801F113030EDB502E
:10D1F000010103151FE0040E0801BB151BE0030E1F
:10D20000DB1C0101A517030EDB502715941304EC5A
:10D2100087F0B2EC93F062EC90F09BEC88F002E1C6
:10D22000000E151807E0020EA6EC8DF0E8EC7EF07B
:10D23000E552E55215EC86F00A0E77EC8DF006E12A
:10D2400015EC86F077EC8DF0010B12E0030EDB504D
:10D250000801F1150DE101016D516E11146E030EFF
:10D26000DB506F15141404E14DEC8EF0EF8E03D0FB
:10D270004DEC8EF0EF9ED950040F94EC86F0030E27
:10D28000F0EC8FF073D60B0EE15C02E2E16AE5523E
:10D29000E16EC8EF85F099EC8DF000C1DFFFDF5043
:10D2A0001BE068EC8FF001011E510DE04DEC8EF09B
:10D2B000EF50800B08E034EC8CF048C1EFFF4DECF0
:10D2C0008EF0EF8C07D034EC8CF0EF5003E14DEC96
:10D2D0008EF0EF9CDF06E3D7020EE15C02E2E16A2A
:10D2E000E552E16EC8EF85F03AEC8CF0300E3CEF81
:10D2F0008AF03AEC8CF0310E3CEF8AF054EC94F06A
:10D3000001012E512F1138E00801E05113E033ECF8
:10D3100094F0DC5DEE50DD59EE50DE59EE50DF59F1
:10D3200009E20101AD510701001104E10801E06BC0
:10D33000DBDF22D00801E6511FE1E4EC8BF002E1D3
:10D34000A7511AE00801010EE06F2EC114F02FC1A1
:10D3500015F042EC8CF02EC106F02FC107F0BBECAB
:10D360008EF00801DC6FEE500320DD6FEE500420DC
:10D37000DE6FEE500520DF6F01012C512D1138E0DA
:10D380000801E55113E033EC94F0E15DEE50E25911
:10D39000EE50E359EE50E45909E20101AD510701A5
:10D3A000001104E10801E56BA4DF22D00801E65179
:10D3B0001FE1E4EC8BF002E1A7511AE00801010E35
:10D3C000E56F2CC114F02DC115F042EC8CF02CC18E
:10D3D00006F02DC107F0BBEC8EF00801E16FEE50B6
:10D3E0000320E26FEE500420E36FEE500520E46F5F
:10D3F0000801BC51BD1109E0420EE66E0D0EE66E4D
:10D400006CEC93F002E10101AB6BE4EC8BF00801F2
:10D41000E66F0101A76B040EE15C02E2E16AE552EE
:10D42000E16EC8EF85F099EC8DF0829A8394FE0E40
:10D43000DB50020B020802E0000E01D0010EE8B042
:10D440008386E8A0839683848394FE0EDB50010BD1
:10D45000E8B08386E8A0839683848394DE52800EAE
:10D46000DD6E080EDF6EDF5017E004EC87F0FD0E76
:10D47000E8EC8BF0146E010EDB50145C02E0000E41
:10D4800001D0010EE8B08386E8A08396838483945C
:10D49000010EF0EC8FF0E7D7828A020EE15C02E227
:10D4A000E16AE552E16EC8EF85F095969594949AFD
:10D4B000120093969392939093941200F00EC114DD
:10D4C0000709C16E0F0E9714976E989096909692DA
:10D4D00099961200E7EC05F071EC9AF0EADFE5DFCF
:10D4E000CDEC00F071ECACF055EC0EF05EEF6AF0B4
:10D4F0005DEC90F007E178EC86F0FA0EDBCFE6FF0A
:10D50000E7EC8FF0C8EF85F05DEC90F005E1D950C5
:10D5100092EC91F0E7EC8FF0C8EF85F05DEC90F0C5
:10D5200005E1D950F4EC8BF0E7EC8FF0C8EF85F013
:10D530005DEC90F005E1D950FAEC8BF0E7EC8FF060
:10D54000C8EF85F05DEC90F00CE178EC86F078ECBB
:10D5500086F0F4EC8EF0E9EC93F0F8EC85F019EC41
:10D560008AF0C8EF85F0C3EC85F041EC8FF0FA0E3D
:10D57000DBCFE6FFF8EC85F0A6EC87F0F6E0C8EF2D
:10D5800085F0C3EC85F041EC8FF0010E02EC91F0D8
:10D59000FAE0C8EF85F0C3EC85F041EC8FF0020EA5
:10D5A00002EC91F0FAE0C8EF85F0C3EC85F041ECB5
:10D5B0008FF0040E02EC91F0FAE0C8EF85F0C3ECB6
:10D5C00085F041EC8FF078EC86F0C1EC86F0F3CF7B
:10D5D00015F0F4CF16F0010EF324AEEC94F0E66AE9
:10D5E00094EC9CF0176E060EE15E1750E552E7CF03
:10D5F00014F0145CE6E0C8EF85F035EC7BF0000930
:10D6000009E066EC8DF0C5EC88F066EC8DF011EC6D
:10D6100089F0000C010C010EB5EC8BF00AE066EC11
:10D620008DF0E66AE66EE66A6C0EE66E11EC89F045
:10D63000000C010C010EB5EC8BF005E066EC8DF0F2
:10D64000E66A47EF93F0010C020EB5EC8BF006E0B2
:10D6500066EC8DF0E66A6C0E47EF93F0010C01EC7E
:10D660008EF0D950010FEBEC8EF00A0EEE6E090E23
:10D67000ED6E080EDF6EDF5013E070EC88F001E312
:10D68000DB2AEF50E66E010EDBCFE9FFDB2A020E4C
:10D69000DBCFEAFF01E3DB2A8EEC87F0DF06EBD776
:10D6A000F2EC8AF064EC86F0030EE15C02E2E16ADF
:10D6B000E552E16EC8EF85F0C3EC85F00B0EE12674
:10D6C000B8EC8FF00CE05CEC8FF016BE1768B7EC8E
:10D6D00092F005E0E7EC89F0F3E3DB2AF1D7DF6AAB
:10D6E000080EDF5C56E2B8EC8FF053E0B8EC8FF038
:10D6F000D00FE66ED950020F146EDF500F011424C4
:10D7000007EC89F08EEC87F0B7EC8AF0142407EC74
:10D7100089F0EF50070807E2B7EC8AF0142407EC11
:10D7200089F0070EEF6E010EDB6ADF504EEC87F0DA
:10D730001BE2D950020F156EDACF16F0DF50152418
:10D7400007EC89F0EFCF14F0D950020F176EDACF43
:10D7500018F0010EDB50172407EC89F0EF50145C31
:10D7600056E0010EDB2AE1D7E7EC89F001E3DB2A82
:10D77000B8EC8FF00CE05CEC8FF016BE1768B7ECDD
:10D7800092F005E0E7EC89F0F3E3DB2AF1D7DF2A3A
:10D79000A7D7080EDF5C48E20A0EDB68010EDB6AE1
:10D7A000DF504EEC87F020E2D950020F156EDACF31
:10D7B00016F0010EDB50152407EC89F0EF50176EC0
:10D7C000010E175204E0E846FE0B1706FCE1E81CC8
:10D7D000146E0A0EDBCFE7FF1450E7160A0EE7CFF0
:10D7E000DBFF010EDB2ADCD7DE52080EDD6E010EF8
:10D7F000DB5009E00A0EDB5006E00A0E8DEC88F0E3
:10D80000010EDB06F4D7010EDB50080802E1010E21
:10D8100011D0B7EC8AF00F01142407EC89F0010E47
:10D82000DBCFEFFFDF2AB5D7E0EC93F018DFE5524E
:10D83000E552000E146E0B0EE15C02E2E16AE55265
:10D84000E16E1450C8EF85F001C1E6FF010E73ECE4
:10D850008DF002C1E6FF020E73EC8DF003C1E6FF0E
:10D86000030E73EC8DF004C1E6FF040E73EC8DF033
:10D8700005C1E6FF050E73EF8DF0EFEC92F0DBCF04
:10D8800001F1BEEC8AF0031724EF90F0EFEC92F078
:10D89000DBCF02F1FE0EDB1C01010117FE0EDB1CCB
:10D8A000031724EF90F0EFEC92F0DBCF03F1BEEC26
:10D8B0008AF0011724EF90F0EFEC92F0DBCF04F147
:10D8C000BEEC8AF00317FE0EDB1C0117BDDFC8EFAC
:10D8D00085F099EC8DF0DF6A050EDF5C2EE28BECB3
:10D8E00093F0DF506FEC8EF0D4EC85F0B6EC93F053
:10D8F000010101510211E552E714BBEC8BF0E71274
:10D900009FEC92F0B6EC93F003510411E552E7144A
:10D91000E81CBBEC8BF0E7169FEC92F0DBCFE6FF48
:10D92000DF506FEC8EF0D8EC85F0F3EC92F0EE5215
:10D93000010EDBCFEFFFDF2ACFD7020EE15C02E260
:10D94000E16AE552E16EC8EF85F0DDEC8DF0D6ECD2
:10D950008CF0C5EC8AF0010ED6EC8BF08EDF7FECFC
:10D9600086F003E0A8EC88F0FDE19BEC86F0050E64
:10D97000DF5C03E26AEC8DF0FAD7060EE15C02E2AE
:10D98000E16AE552E16EC8EF85F0DDEC8DF0010E45
:10D99000DBCF01F1030EDBCF03F1C5EC8AF0020E01
:10D9A000D6EC8BF073DF7FEC86F003E0A8EC88F018
:10D9B000FDE19BEC86F0050EDF5C03E26AEC8DF086
:10D9C000FAD7060EE15C02E2E16AE552E16EC8EFC9
:10D9D00085F0DDEC8DF0020EDBCF02F1010EDBCF26
:10D9E00001F1C5EC8AF0030ED6EC8BF05CDF7FEC26
:10D9F00086F003E0A8EC88F0FDE19BEC86F0050ED4
:10DA0000DF5C03E26AEC8DF0FAD7060EE15C02E21D
:10DA1000E16AE552E16EC8EF85F0DDEC8DF0D6EC01
:10DA20008CF0010EDBCF01F1B6EC93F0040ED6ECD6
:10DA30008BF042DF7FEC86F003E0A8EC88F0FDE19C
:10DA40009BEC86F0050EDF5C03E26AEC8DF0FAD702
:10DA5000060EE15C02E2E16AE552E16EC8EF85F094
:10DA6000EFEC92F0DBCFD1F8D1C8E6FFF40E73EC07
:10DA70008DF0D1C8E6FF03EC03F0E552C8EF85F066
:10DA80002FEC8EF00BE2F8EC85F0580EE66E040EEB
:10DA90007AEC87F005EC91F0E0EC86F0C8EF85F0C9
:10DAA0003BEC8FF00BE290EC86F0580EE66E040E25
:10DAB0006FEC87F005EC91F0E0EC86F0C8EF85F0B4
:10DAC0002FEC8EF008E2F8EC85F064EC8CF07AEC48
:10DAD00087F0D9EC91F0C8EF85F03BEC8FF008E2CD
:10DAE00090EC86F064EC8CF06FEC87F0D9EC91F060
:10DAF000C8EF85F02FEC8EF00BE2F8EC85F0800E8D
:10DB0000E66E040E7AEC87F00BEC91F0E0EC86F018
:10DB1000C8EF85F03BEC8FF00BE290EC86F0800EC6
:10DB2000E66E040E6FEC87F00BEC91F0E0EC86F003
:10DB3000C8EF85F02FEC8EF00BE2F8EC85F0940E38
:10DB4000E66E040E7AEC87F011EC91F0E0EC86F0D2
:10DB5000C8EF85F03BEC8FF00BE290EC86F0940E72
:10DB6000E66E040E6FEC87F011EC91F0E0EC86F0BD
:10DB7000C8EF85F0AAEC94F0E66EE66AF8EC85F062
:10DB80004EEC8FF034EC91F034EC89F064EC86F0DC
:10DB9000C8EF85F0C3EC85F090EC86F0A80EE66E39
:10DBA000040E6FEC87F034EC89F064EC86F0C8EF7B
:10DBB00085F0F1EC93F00FE2060E6BEC89F0FE0EAF
:10DBC000DB5091EC8DF0CAECABF0166E060EE15E08
:10DBD0001650F6EC92F0C8EF85F02AEC91F0B8EC14
:10DBE0008FF00CE05CEC8FF016BE1768B7EC92F08B
:10DBF00005E0E7EC89F0F3E3DB2AF1D7FBEC88F0F2
:10DC00002BEC90F015EC86F0EBEC89F016BE176863
:10DC1000E6EC92F00AE015EC86F0EF5006E0040E18
:10DC2000DB2A050EEFE3DB2AEDD715EC86F0EF508B
:10DC300010E0040EDBCFE9FFDB2A050EDBCFEAFFA5
:10DC400001E3DB2AEF6AF8EC85F0E4EC93F0F4EC06
:10DC500087F0B8EC8FF00CE05CEC8FF016BE176824
:10DC6000B7EC92F005E0E7EC89F0F3E3DB2AF1D7BB
:10DC7000F1EC86F0080EEE5C000E3EEC88F018E247
:10DC8000FCEC8AF0EFCF14F0080E145C11E2B8EC53
:10DC90008FF00EE0C1EC88F0050EDBCFE6FFFCEC68
:10DCA0008AF0EF50E66E85DFD9EC8DF0000E01D0E2
:10DCB000010E146E060EE15C02E2E16AE552E16ECD
:10DCC0001450C8EF85F0F1EC93F00DE2060E35EC40
:10DCD0008AF0FE0EDB5091EC8DF0F8ECABF084ECAA
:10DCE00092F0F6EC92F0C8EF85F0EFEC92F0DB509A
:10DCF000EA6A4D0FE96E010E06EC8BF04B0F73ECE8
:10DD00008DF0C8EF85F0EFEC92F0DB50EA6A550F2A
:10DD1000E96E010E06EC8BF0530F73EC8DF0C8EF3B
:10DD200085F0EFEC92F0E7EC8DF0FD0EDBCFEFFF2E
:10DD3000FE0E5EEC93F063EC8AF0E3EC94F00E0ED2
:10DD4000E9EC93F0D8EC85F0C8EF85F0EFEC92F0B9
:10DD5000B4EC94F0FD0EDBCFEFFFFE0EB4EC94F0CC
:10DD6000EF5063EC8AF06FEC8EF0D8EC85F0C8EFE2
:10DD700085F060EC8FF0A0EC90F0DF6A080EDF5CBD
:10DD80000EE266EC90F0480EE926080EEA22E9C69B
:10DD9000EEFFEAC6EEFFEBC6EEFFDF2AEFD71BEC85
:10DDA00094F039EF8EF060EC8FF0EC0EE66E060E1C
:10DDB000E66E1A0EF8EC8EF0080EDF5C0EE266ECF2
:10DDC00090F0300EE926080EEA22ECC6EEFFEDC612
:10DDD000EEFFEEC6EEFFDF2AEFD7180EE66E300E2E
:10DDE000E66E080EE66E1D0E39EF8EF060EC8FF0D9
:10DDF000EF0EE66E060EE66E350EF8EC8EF0080EAF
:10DE0000DF5C0EE266EC90F0180EE926080EEA22BE
:10DE1000EFC6EEFFF0C6EEFFF1C6EEFFDF2AEFD74A
:10DE2000180EE66E180EE66E080EE66E380E39EF26
:10DE30008EF060EC8FF0F20EE66E060EE66E500E7F
:10DE4000F8EC8EF0080EDF5C0EE266EC90F0000E4F
:10DE5000E926080EEA22F2C6EEFFF3C6EEFFF4C68C
:10DE6000EEFFDF2AEFD7180EE66E000EE66E080E04
:10DE7000E66E530E39EF8EF060EC8FF0F50EE66E25
:10DE8000060EE66E6B0EF8EC8EF0080EDF5C0EE20E
:10DE900066EC90F0A10EE926060EEA22F5C6EEFF2A
:10DEA000F6C6EEFFF7C6EEFFDF2AEFD7180EE66ED6
:10DEB000A10EE66E060EE66E6E0E39EF8EF060EC89
:10DEC0008FF0F80EE66E060EE66E860EF8EC8EF01B
:10DED000080EDF5C0EE266EC90F0D10EE926060E2D
:10DEE000EA22F8C6EEFFF9C6EEFFFAC6EEFFDF2A19
:10DEF000EFD7180EE66ED10EE66E060EE66E890EB0
:10DF000039EF8EF060EC8FF0FC0EE66E0D0EE66ED3
:10DF1000B60EF8EC8EF0080EDF5C0EE266EC90F0C8
:10DF2000B90EE926060EEA22FCCDEEFFFDCDEEFF8E
:10DF3000FECDEEFFDF2AEFD7180EE66EB90EE66EC5
:10DF4000060EE66EB90E39EF8EF0E66A570E49EC12
:10DF500086F0C5EC88F0E66AE6EC9BF089EF87F086
:10DF6000CDEC8DF00101080E006FE66EC5EC88F077
:10DF7000D8EC85F00101056B066B06C1E6FF430E88
:10DF80007BEC8DF001010269010EE66E76DCE55254
:10DF9000E66A89DCE552E66A8FDCE552FE0E010195
:10DFA0000211E66E73DCE5520101021D076FE66E99
:10DFB0004B0E7BEC8DF001016D6B6DC1E6FF3CEC0F
:10DFC00089F0D8EC85F001016E6B6EC1E6FFD0ECF4
:10DFD0008BF0D8EC85F001016F6B6FC1E6FF4A0E44
:10DFE0007BEC8DF00101706B70C1E6FFD3EC8BF020
:10DFF000D8EC85F00101440E716FE66E400E7BECAB
:10E000008DF00101726B72C1E6FF470E7BEC8DF063
:10E010000101736B73C1E6FF480E7BEC8DF0E6687F
:10E02000E66ABBEC89F0E668E66AC0EC89F0E66A6D
:10E03000010EE66EBBEC89F0E66A010EE66EC0ECFE
:10E0400089F0E66A020EE66EBBEC89F0E66A020E23
:10E05000E66EC0EC89F0040EDF6EDF5002080CE2C1
:10E06000E66ADFCFE6FFBBEC89F0E66ADFCFE6FFCA
:10E07000C0EC89F0DF06F1D7F30EE66E080EE66E0F
:10E080002FEC6BF0E552E5520101010E086FE66ED0
:10E09000270E73EC8DF00101030E096FE66E280E5A
:10E0A00073EC8DF00101010E0A6FE66E290E73EC20
:10E0B0008DF00101010E0B6FE66E360E7BEC8DF0DC
:10E0C00001010C6B0CC1E6FF370E7BEC8DF00101FA
:10E0D000030E0D6FE66EB80E9EEC8DF00101030E7F
:10E0E0000E6FE66E350E7BEC8DF00101020E0F6FA8
:10E0F000E66E2A0E73EC8DF00101010E106FE66ED4
:10E100002B0E73EC8DF00101116B11C1E6FFC00EF7
:10E110009EEC8DF00101126B12C1E6FF380E7BEC14
:10E120008DF00101136B13C1E6FFC10E9EEC8DF063
:10E130000101146B14C1E6FF390E7BEC8DF0010177
:10E14000156B15C1E6FFC20E9EEC8DF0010116693C
:10E1500016C1E6FF3A0E7BEC8DF00101176B17C17B
:10E16000E6FF440E7BEC8DF00101186918C1E6FF53
:10E170003B0E7BEC8DF00101196919C1E6FF3C0EE5
:10E180007BEC8DF001011A6B1AC1E6FFC30E9EEC09
:10E190008DF001011B6B1BC1E6FF2C0E73EC8DF0A3
:10E1A0000101010E1C6FE66E2D0E73EC8DF0010166
:10E1B000010E1D6FE66E2E0E73EC8DF00101010E47
:10E1C0001E6FE66E2F0E73EC8DF001012A6B2AC1D3
:10E1D000E6FFB90E9EEC8DF001012B6B2BC1E6FF23
:10E1E000420E7BEC8DF0DF6A080EDF5C11E2DF503F
:10E1F000EA6ABE0FE96E080EEA22EF6ADF50EA6AA9
:10E20000C60FE96E080EEA22200EEF6EDF2AECD769
:10E2100082EC8AF064EC86F08BEC8AF064EC86F099
:10E2200001011F691FC1E6FF300E73EC8DF0010183
:10E23000010E206FE66E310E73EC8DF00101030EBE
:10E24000216FE66EA20E9EEC8DF00101226B22C1C1
:10E25000E6FFA30E9EEC8DF00101070E236FE66E24
:10E26000A40E9EEC8DF00101030E246FE66EA50E48
:10E270009EEC8DF00101030E256FE66EA60E9EEC5E
:10E280008DF00101266926C1E6FF4C0E7BEC8DF076
:10E290000101276927C1E6FF3E0E7BEC8DF00101ED
:10E2A000286928C1E6FF490E7BEC8DF00101296B3E
:10E2B00029C1E6FF3F0E7BEC8DF0DF6A080EDF5CC4
:10E2C00008E2E66ADF50DFEC91F0D8EC85F0DF2A57
:10E2D000F5D701012C6B2D6B2CC1E6FF2DC1E6FF9C
:10E2E000BC0ED0EC92F0FFEC85F0780E01012E6FA1
:10E2F0002F6BE66E2FC1E6FFBE0ED0EC92F0FFEC66
:10E3000085F00101010E306F44EC8DF0D8EC85F002
:10E3100001010C0E316FE66E330E73EC8DF00101CE
:10E32000010E326FE66E340E73EC8DF001010C0EAF
:10E33000336FE66E350E73EC8DF00101140E346F01
:10E34000E66E3D0E7BEC8DF00101280E356FE66E1A
:10E35000360E73EC8DF00101366B36C1E6FF370ED9
:10E3600073EC8DF001010F0E376FE66E380E73EC13
:10E370008DF0780E0801BC6FBD6BE66EBDC8E6FF80
:10E38000450E15EC8FF00101960E386FE66E390ED2
:10E3900073EC8DF00101010E396FE66ED40E9EEC28
:10E3A0008DF01E0E01013B6F3C6BE66E3CC1E6FF3B
:10E3B0003A0E19EC8FF0780E01013D6F3E6BE66E60
:10E3C0003EC1E6FF3C0E19EC8FF00101580E3F6F85
:10E3D000020E406F3FC1E6FFE66E3E0E19EC8FF075
:10E3E000010E0101416F426BE66E42C1E6FF400E35
:10E3F00019EC8FF00101140E436FE66E420E73ECC0
:10E400008DF00101020E446FE66E430E73EC8DF049
:10E4100001010A0E456FE66E440E73EC8DF00101AA
:10E42000320E466FE66E450E73EC8DF001010F0E55
:10E43000476FE66E410E7BEC8DF00101486948C1E3
:10E44000E6FF460E73EC8DF00101030E3A6FE66EA7
:10E45000B70E9EEC8DF00801580EAE6F020EAF6F36
:10E46000AEC8E6FFE66E240E15EC8FF00801100E24
:10E47000B06F0E0EB16FB0C8E6FFE66E260E15EC5B
:10E480008FF00801030EB26FE850E66EE66A280EC0
:10E4900015EC8FF00801010EB56FE66E2B0E7BECCC
:10E4A0008DF00801FE0EB66FE66E2C0E7BEC8DF043
:10E4B000B40E0801B76FB86BE66EB8C8E6FF2D0E54
:10E4C00015EC8FF00801BA6BBAC8E6FF300E7BEC92
:10E4D0008DF00801030EBB6FE66E310E7BEC8DF004
:10E4E0000801B36BB3C8E6FF290E7BEC8DF0080181
:10E4F000B46BB4C8E6FF2A0E7BEC8DF00801B96B53
:10E50000B9C8E6FF2F0E7BEC8DF001010A0E496FB2
:10E51000E66E470E73EC8DF001011E0E4B6FE66E3A
:10E52000480E73EC8DF001010A0E4A6FE66E490E3B
:10E5300073EC8DF00101010E4C6FE66E4A0E73EC28
:10E540008DF00801200ECE6F030ECF6FCEC8E6FF10
:10E55000E66EF10E19EC8FF00D017F0E1D6F120E9D
:10E56000E66E30EC6DF0E5520801D26BD2C8E6FFE2
:10E57000F50E73EC8DF00801D36BD3C8E6FFF60EF1
:10E5800073EC8DF00801280ED46F040ED56FD4C83B
:10E59000E6FFE66EF70E19EC8FF00801280ED66F35
:10E5A000E66EF90E73EC8DF00801140ED76FE66E6F
:10E5B000FA0E73EC8DF00801280ED86F040ED96F97
:10E5C000D8C8E6FFE66EFB0E19EC8FF00801140EBA
:10E5D000DA6FE66EFD0E73EC8DF00801180EDB6F3E
:10E5E000E66EFE0E73EC8DF0E4EC8CF050EC6DF00A
:10E5F000D9EC8DF0E4EC8CF06DEC6DF00FEC8BF061
:10E600008AEC6DF00FEC8BF0AAEC6DF0D9EC8DF08C
:10E610009E0EE66E5F0EE66E010EE66ECAEC6DF0C3
:10E62000D9EC8DF0DF6A080EDF5C0EE29D0EE66E1F
:10E630005F0EE66E010EE66EDFCFE6FF63EC6EF076
:10E64000D6EC94F0DF2AEFD70101020E696FE66E77
:10E650009C0E9EEC8DF001016A6B6AC1E6FF230EF1
:10E660007BEC8DF001016B6B6BC1E6FF9D0E9EECA8
:10E670008DF001016C69E5EC91F0060EE66EE66A3C
:10E68000960EE66E5F0EE66E010E86EC94F005ECDB
:10E690008AF00D01676B010EDF6E140EDF5C05E280
:10E6A00083EC8BF0EF6ADF2AF8D78C0E81EC8EF0CA
:10E6B00064EC86F00D01010E606FE66EF00E73ECF7
:10E6C0008DF00601E96BEA6BC5EC88F0FF0E19ECE2
:10E6D0008FF00601640EEB6F3EEC86F0E66ED8EC30
:10E6E00085F0120E0601EC6FED6BE66EE66A1A0E0F
:10E6F000D1EC8DF00601640EEE6FE66E1C0ED5ECCB
:10E700008DF0110E0601EF6FF06BE66EE66A350EC6
:10E71000D1EC8DF00601640EF16FE66E370ED5EC8C
:10E720008DF0130E0601F26FF36BE66EE66A500E83
:10E73000D1EC8DF00601640EF46FE66E520ED5EC4E
:10E740008DF01C0E0601F56FF66BE66EE66A6B0E39
:10E75000D1EC8DF00601640EF76FE66E6D0ED5EC10
:10E760008DF0180E0601F86FF96BE66EE66A860EFC
:10E77000D1EC8DF00601500EFA6FE66E880ED5ECE6
:10E780008DF0160E0301F96FFA6BE66EE66AA10EC4
:10E79000D1EC8DF00301400EFB6FE66EA30ED5ECBD
:10E7A0008DF00301FC6BFD6BC5EC88F0A40ED1EC81
:10E7B0008DF003017F0EFE6FE66EA60ED5EC8DF098
:10E7C0001A0E0D01ED6FEE6BE66EE66AA70ED1EC48
:10E7D0008DF00D01A00EEF6FE66EA90ED5EC8DF059
:10E7E0001B0E0D01F06FF16BE66EE66AAA0ED1EC1E
:10E7F0008DF00D01960EF26FE66EAC0ED5EC8DF03D
:10E80000300E0D01F36FF46BE66EE66AAD0ED1ECDF
:10E810008DF00D01780EF56FE66EAF0ED5EC8DF034
:10E82000270E0D01F66FF76BE66EE66AB00ED1ECBF
:10E830008DF00D01780EF86FE66EB20ED5EC8DF00E
:10E84000310E0D01F96FFA6BE66EE66AB30ED1EC8C
:10E850008DF00D01790EFB6FE66EB50ED5EC8DF0E7
:10E860000D01010EFC6F100EFD6F010EE66E100E15
:10E87000E66EB60ED1EC8DF00D015A0EFE6FE66E0F
:10E88000B80ED4EC92F0240E08016C6F6D6BE66E3E
:10E89000E66ADD0ED1EC8DF00801A00E6E6FE66E1B
:10E8A000DF0ED5EC8DF0210E08016F6F706BE66EF8
:10E8B000E66AE00ED1EC8DF00801A00E716FE66EF5
:10E8C000E20ED5EC8DF0230E0801666F676BE66EE5
:10E8D000E66AD70ED1EC8DF008017F0E686FE66E08
:10E8E000D90ED5EC8DF00801696B6A6BC5EC88F028
:10E8F000DA0ED1EC8DF00801640E6B6FE66EDC0E63
:10E90000D4EC92F00801900E636F410E646F900E8C
:10E91000E66E410EE66ED40ED1EC8DF008017F0E4E
:10E92000656FE66ED60ED5EC8DF0230E0801726F82
:10E93000736BE66EE66A1D0E15EC8FF008017F0E14
:10E94000746FE66E1F0E7BEC8DF00801756B766BB5
:10E95000C5EC88F0200E15EC8FF008017F0E776F64
:10E96000E66E220E7BEC8DF0250E0601FB6FFC6B34
:10E97000E66EE66A320E15EC8FF006017F0EFD6F33
:10E98000E66E340E7BEC8DF001015A0E606FE66E80
:10E99000BB0E9EEC8DF0B9EC6EF0D3EC6EF0F6ECA5
:10E9A0006EF019EC6FF03CEC6FF05FEC6FF082EC06
:10E9B0006FF000010A0EE06FE16BE26BE36BE66E55
:10E9C00062EC8DF0C40EEFEC8EF00001640EE46F8B
:10E9D000E56BE66BE76BE66E62EC8DF0C80EEFEC74
:10E9E0008EF00001E80EE86F030EE96FEA6BEB6B47
:10E9F000E80E49EC86F0E66AE66ACC0EEFEC8EF0A3
:10EA00000001880EEC6F130EED6FEE6BEF6B880E4E
:10EA1000E66E130EE66EE66AE66AD00EEFEC8EF056
:10EA20000101070E746FE66E550E7BEC8DF0080E3B
:10EA3000DF6EDF5017E07F0EE66EE66ADF0498ECCB
:10EA400087F07F0E3EEC86F0DF04EBEC91F0DF0404
:10EA500098EC87F0760E49EC86F0DF0498EC87F0AE
:10EA6000DF06E7D77F0EE66EE66A080E98EC87F0C1
:10EA70007F0E3EEC86F0080EEBEC91F0080E98EC61
:10EA800087F0760E49EC86F0080E98EC87F059EC8A
:10EA9000A9F0E552C8EF85F0C3EC85F0080EDEEC76
:10EAA0008AF0040F5BEC93F0E66AE4EC85F0800EEC
:10EAB0001EEC8AF0080EDF6EDF504CE068EC8FF041
:10EAC00052EC87F0040EE8EC8BF002E0010E17D058
:10EAD00052EC87F0050EE8EC8BF002E0020E0FD04E
:10EAE00052EC87F0060EE8EC8BF002E0040E07D043
:10EAF00052EC87F0070EE8EC8BF005E0080EF36EA1
:10EB0000030EF3CFDBFF49EC8EF0EE52030EDBCFAA
:10EB1000EFFFDB50040A13E00C0A11E0090A07E0DA
:10EB2000030A14E1020EDB500101061508E149EC6D
:10EB30008EF0090EF4EC85F035C1EFFF07D049ECFB
:10EB40008EF0090EF4EC85F036C1EFFF020EF0EC0A
:10EB50008FF0B2D7080EE15C02E2E16AE552E16EA5
:10EB6000C8EF85F0C3EC85F0FD0EDB500801B5154C
:10EB700004E0FE0EDB50B31303D0FE0EDB1CB31714
:10EB8000FD0EDB50B61504E0FE0EDB50B41303D0CF
:10EB9000FE0EDB1CB417FD0EDB50BA1504E0FE0EB2
:10EBA000DB50B91303D0FE0EDB1CB917C8EF85F09C
:10EBB000B3C8E6FF290E7BEC8DF0B4C8E6FF2A0E41
:10EBC0007BEC8DF0B9C8E6FF2F0E7BEF8DF001ECEA
:10EBD0008EF062DF800E1EEC8AF0080EDF6EDF50D2
:10EBE00066E0B6EC93F0020EE8EC8BF05CE068ECCB
:10EBF0008FF0DB50DCEC85F0EE52EF50080A48E075
:10EC00000A0A12E0060A09E0050A4DE1BCEC8FF0A1
:10EC1000600E78EC89F0010E40D0BCEC8FF0400E15
:10EC200078EC89F0040E39D0020EDB500101051595
:10EC30000AE0020EDB1C6C17FDEC8FF0EF6E100E7D
:10EC4000E66E020E1BD07FEC88F04AC1EFFF86EC27
:10EC500088F04CC1EFFF205102E1000E01D0010EFF
:10EC6000200DF3504009E66E010EAEEC86F08EECFE
:10EC700087F0020EDB506C13020EE66EDBCFE6FF70
:10EC800071DFE552E552020EDB1C010107170BD0C4
:10EC9000FDEC8FF078EC89F0080EE66E52EC87F010
:10ECA00061DFE552E552020EF0EC8FF098D717ECD9
:10ECB0008BF064EC86F021EC8BF064EC86F0C9EC10
:10ECC00088F064EC86F0E5EC91F007C1E6FF4B0EAE
:10ECD0007BEC8DF06DDF030EE15C02E2E16AE55250
:10ECE000E16EC8EF85F045EC8EF0000EE66E010E89
:10ECF000E66EC5EC88F0D4EC85F0010E0101005DF4
:10ED000002E2010E006F060EE66E010EE66E430E85
:10ED100088EC8DF0070EE66E010EE66E4B0E88EC69
:10ED20008DF0010EE66E010E3EEC86F0E66AD4EC44
:10ED300085F0020EE66E010EE66E020E7FEC8DF09F
:10ED4000030EE66E010E49EC86F0E66AD4EC85F01F
:10ED5000040EE66E010EE66E040E7FEC8DF0050EDD
:10ED6000E66E010EE66E050E7FEC8DF06D0EE66E22
:10ED7000010EE66E87EC93F06E0EE66E010EE66E07
:10ED8000D0EC8BF0D4EC85F06F0EE66E010EE66EE3
:10ED90004A0E88EC8DF0700EE66E010EE66ED3EC36
:10EDA0008BF0D4EC85F0710EE66E010EE66E400E2F
:10EDB00088EC8DF0720EE66E010EE66E470E88EC62
:10EDC0008DF0730EE66E010EE66E480E88EC8DF047
:10EDD000DE6ADD6AECEC86F0050E66EC91F01DE271
:10EDE000E3EC8AF020EC88F006EC88F0FFEC86F08B
:10EDF000D4EC85F0E3EC8AF020EC88F0EE5206ECDF
:10EE000088F0010E1626000EA7EC94F0D4EC85F0E5
:10EE1000DF2A010EDFE3DB2ADDD7F2EC8AF0E4EC37
:10EE200085F0080EE66E010EE66E270E7FEC8DF083
:10EE3000090EE66E010EE66E280E7FEC8DF00A0ECE
:10EE4000E66E010EE66E290E7FEC8DF00B0EE66E7F
:10EE5000010EE66E360E88EC8DF00C0EE66E010E9D
:10EE6000E66E370E88EC8DF00D0EE66E010EE66E46
:10EE7000B80EA2EC8DF00E0EE66E010EE66E350EAB
:10EE800088EC8DF00F0EE66E010EE66E2A0E7FEC1A
:10EE90008DF0100EE66E010EE66E2B0E7FEC8DF0FF
:10EEA000110EE66E010EE66EC00EA2EC8DF0120E93
:10EEB000E66E010EE66E380E88EC8DF0130EE66EEF
:10EEC000010EE66EC10EA2EC8DF0140EE66E010E80
:10EED000E66E390E88EC8DF0150EE66E010EE66ECC
:10EEE000C20EA2EC8DF0160EE66E010EE66E3A0E24
:10EEF00088EC8DF0170EE66E010EE66E440E88EC7F
:10EF00008DF0180EE66E010EE66E3B0E88EC8DF06D
:10EF1000190EE66E010EE66E3C0E88EC8DF01A0EB0
:10EF2000E66E010EE66EC30EA2EC8DF01B0EE66ED1
:10EF3000010EE66E2C0E7FEC8DF01C0EE66E010EBF
:10EF4000E66E2D0E7FEC8DF01D0EE66E010EE66E68
:10EF50002E0E7FEC8DF01E0EE66E010EE66E2F0E6D
:10EF60007FEC8DF02A0EE66E010EE66EB90EA2EC75
:10EF70008DF02B0EE66E010EE66E420E88EC8DF0E3
:10EF800082EC8AF0E4EC85F08BEC8AF0E4EC85F01E
:10EF9000DE6ADD6AECEC86F0080E66EC91F016E2B3
:10EFA000E00E146EE3EC8AF0BE0EE926080EEA22AB
:10EFB0001450EF16E3EC8AF0C60EE926080EEA229A
:10EFC000EF8ADF2A010EE6E3DB2AE4D71F0EE66EA6
:10EFD000010EE66E300E7FEC8DF0200EE66E010E17
:10EFE000E66E310E7FEC8DF0210EE66E010EE66EC0
:10EFF000A20EA2EC8DF0220EE66E010EE66EA30EBE
:10F00000A2EC8DF0230EE66E010EE66EA40EA2ECCD
:10F010008DF0240EE66E010EE66EA50EA2EC8DF0CC
:10F02000250EE66E010EE66EA60EA2EC8DF0260E03
:10F03000E66E010EE66E4C0E88EC8DF00CEC94F052
:10F04000280EE66E010EE66E490E88EC8DF0290E54
:10F05000E66E010EE66E3F0E88EC8DF02E0EE66E2B
:10F06000010EE66EBE0ED0EC92F0B8EC86F02C0EDF
:10F07000E66E010EE66EBC0ED0EC92F0B8EC86F0B7
:10F08000300EE66E010E44EC8DF0D4EC85F0310EBE
:10F09000E66E010EE66E330E7FEC8DF0320EE66EFC
:10F0A000010EE66E340E7FEC8DF0330EE66E010E2F
:10F0B000E66E350E7FEC8DF0340EE66E010EE66ED8
:10F0C0003D0E88EC8DF0350EE66E010EE66E360EC6
:10F0D0007FEC8DF0360EE66E010EE66E370E7FEC9D
:10F0E0008DF0370EE66E010EE66E380E7FEC8DF079
:10F0F000BC0EE66E080EE66E450E62EC91F03A0E1E
:10F10000E66E010EE66EB70EA2EC8DF0AE0EE66E68
:10F11000080EE66E240E62EC91F0B00EE66E080E5C
:10F12000E66E260E62EC91F0B20EE66E080EE66E0A
:10F13000280E88EC8DF0B50EE66E080EE66E2B0EEE
:10F1400088EC8DF0B60EE66E080EE66E2C0E88EC9E
:10F150008DF0B70EE66E080EE66E2D0E62EC91F0A5
:10F16000BA0EE66E080EE66E300E88EC8DF0BB0E21
:10F17000E66E080EE66E310E88EC8DF0B30EE66E8C
:10F18000080EE66E290E88EC8DF0B40EE66E080EC1
:10F19000E66E2A0E88EC8DF0B90EE66E080EE66E6D
:10F1A0002F0E88EC8DF0380EE66E010EE66E390EED
:10F1B0007FEC8DF0390EE66E010EE66ED40EA2ECF9
:10F1C0008DF03B0EE66E010EE66E3A0E64EC8FF0AB
:10F1D0003D0EE66E010EE66E3C0E64EC8FF03F0EC7
:10F1E000E66E010EE66E3E0E64EC8FF0410EE66EAA
:10F1F000010EE66E400E64EC8FF0430EE66E010EDB
:10F20000E66E420E7FEC8DF0440EE66E010EE66E69
:10F21000430E7FEC8DF0450EE66E010EE66E440E59
:10F220007FEC8DF0460EE66E010EE66E450E7FEC2D
:10F230008DF0470EE66E010EE66E410E88EC8DF005
:10F24000480EE66E010EE66E460E7FEC8DF0490E1E
:10F25000E66E010EE66E470E7FEC8DF04A0EE66E0E
:10F26000010EE66E490E7FEC8DF04B0EE66E010E40
:10F27000E66E480E7FEC8DF04C0EE66E010EE66EEB
:10F280004A0E7FEC8DF0CE0EE66E080EE66EF10EA5
:10F2900064EC8FF0D20EE66E080EE66EF50E7FEC93
:10F2A0008DF0D30EE66E080EE66EF60E7FEC8DF056
:10F2B000D40EE66E080EE66EF70E64EC8FF0D80EF4
:10F2C000E66E080EE66EFB0E64EC8FF0D60EE66E70
:10F2D000080EE66EF90E7FEC8DF0DA0EE66E080E83
:10F2E000E66EFD0E7FEC8DF0D10EE66E080EE66E3A
:10F2F000F40E7FEC8DF0D70EE66E080EE66EFA0E79
:10F300007FEC8DF0DB0EE66E080EE66EFE0E7FECF7
:10F310008DF0140EE66E05EC91F032EC90F064EC9A
:10F320008CF0E66E740E32EC90F00BEC91F032EC57
:10F3300090F011EC91F08FEC93F034EC89F0E4EC68
:10F3400085F0380EE66EC70EE66E020EE66EB00E63
:10F350008FEC93F0030EE66EA0EC90F0030EE66ED9
:10F36000EC0EE66E060EE66E1A0E83EC8DF0EF0ED6
:10F37000E66E060EE66E350E83EC8DF0F20EE66E4E
:10F38000060EE66E500E83EC8DF0F50EE66E060E60
:10F39000E66E6B0E83EC8DF0F80EE66E060EE66EF2
:10F3A000860E83EC8DF0F90EE66E030EE66EA10E6E
:10F3B00083EC8DF0FC0EE66E030EE66EA40E83EC7D
:10F3C0008DF0ED0EE66E0D0EE66EA70E83EC8DF061
:10F3D000F00EE66E0D0EE66EAA0E83EC8DF0F30EC7
:10F3E000E66E0D0EE66EAD0E83EC8DF0F60EE66E5B
:10F3F0000D0EE66EB00E83EC8DF0F90EE66E0D0E7E
:10F40000E66EB30E83EC8DF0FC0EE66E0D0EE66E2E
:10F41000B60E83EC8DF0600EE66E080EE66ED10E31
:10F4200083EC8DF06C0EE66E080EE66EDD0E83EC5E
:10F430008DF06F0EE66E080EE66EE00E83EC8DF03A
:10F44000660EE66E080EE66ED70E83EC8DF0690E42
:10F45000E66E080EE66EDA0E83EC8DF0630EE66E55
:10F46000080EE66ED40E83EC8DF0720EE66E080E7A
:10F47000E66E1D0EF0EC91F0750EE66E080EE66E6F
:10F48000200EF0EC91F0FB0EE66E060EE66E320EEC
:10F4900049EC86F0E4EC85F0600EE66E010EE66E57
:10F4A000BB0EA2EC8DF01BEC94F078EC8EF0300EDD
:10F4B000E66E080EE66E1D0E78EC8EF0180EE66E07
:10F4C000080EE66E380E78EC8EF0000EE66E080E32
:10F4D000E66E530E78EC8EF0A10EE66E060EE66E2A
:10F4E0006E0E78EC8EF0D10EE66E060EE66E890E8C
:10F4F00078EC8EF0B90EE66E060EE66EB90EF5ECFF
:10F5000093F0040EE66EE00EE66E000EE66EC40E9C
:10F510008BEC94F0E40EE66E000EE66EC80E8BECFB
:10F5200094F0E80EE66E000EE66ECC0E8BEC94F0D6
:10F53000EC0EE66E000EE66ED00E87EC8EF0600EDE
:10F54000E66E0D0EE66EF00E7FEC8DF0690EE66E47
:10F55000010EE66E9C0EA2EC8DF06A0EE66E010EB8
:10F56000E66E230E88EC8DF06B0EE66E010EE66EF5
:10F570009D0EA2EC8DF06C0EE66E010EE66E49EC6F
:10F580008DF0D4EC85F04CEC75F08C0E81EC8EF0A7
:10F59000E4EC85F017EC8BF0E4EC85F021EC8BF0DB
:10F5A000E4EC85F0C9EC88F0E4EC85F0240EE66E1E
:10F5B000640EE66E060EE66E700E87EC8EF0040E9C
:10F5C000E15C02E2E16AE552E16EC8EF85F09992F2
:10F5D0008782640EEBEC8CF087921200EFEC92F0D5
:10F5E00081EC89F0EF509BEC88F004E1155002E1CA
:10F5F000000E01D0010EC8EF85F001EC8EF0F7ECA3
:10F6000091F00AE00A0EEBEC8CF0F7EC91F002E0DE
:10F61000000E03D0010E01D0010E2DEC8AF002E2A3
:10F62000E16AE552E16E1450C8EF85F099EC8DF077
:10F63000DE6ADD6AECEC86F0080E66EC91F00BE217
:10F64000DFCFE6FFDADFE552000905E0DF2A010E31
:10F65000F1E3DB2AEFD7DF50E0EC8BF002E2E16A66
:10F66000E552E16E1450C8EF85F099EC8DF0010180
:10F67000746BDF6A740EE66E010EE66E550E88EC52
:10F680008DF0070E0101745D02E1010EDF6EDF50A7
:10F69000E0EC8BF002E2E16AE552E16E1450C8EF53
:10F6A00085F0CDEC8DF0DF6AFE0EDB0406E1B8ECF0
:10F6B00087F0550EE66E390E09D0FE0EDB500208BB
:10F6C0000FE1B8EC87F0550EE66E6F0EE66ED4ECE7
:10F6D00085F0070E146EDF50145C04E1010E03D0B8
:10F6E000000E01D0000EE552C8EF85F0E668E6682E
:10F6F00062EC8DF02FECB1F0050EE15E1200AB0E66
:10F700003EEC86F0C5EC88F04AEF8CF0E66A190E04
:10F71000E66EE66A040EE66E4AEF8CF0C3EC85F006
:10F72000080EE1260101876B140E9DEC87F00101A4
:10F73000A46FE66AF1EC05F0E5520101886FE8502C
:10F74000146E156AD890155004E6C80E145C000EAD
:10F75000155802E2A4050BE088519BEC88F001E10A
:10F76000155002E0A4051FE0010E876F1CD0882B06
:10F7700088C1E6FFE66A89EC92F0D0B205D0030EAC
:10F7800017EC91F0030E0DD0D0B805D0040E17EC95
:10F7900091F0040E06D0D0B606D0050E17EC91F00D
:10F7A000050EFCEC86F00101A46BD082D088D086D7
:10F7B00055EC9BF0DF6EDF5003E00101010EF86FA6
:10F7C0000101875106E151DF000903E073EC76F097
:10F7D00079D0E66A140EFCEC86F00101876B885143
:10F7E0009BEC88F01CE115501AE1886B876BE66A88
:10F7F000E66A89EC92F0E66A010EFCEC86F0E66AB5
:10F80000020EFCEC86F0E66A030EFCEC86F0E66A7B
:10F81000040EFCEC86F0E66A050EFCEC86F0A5EC26
:10F820006FF0B0EC6FF0E668E7EC75F0E55268EC6D
:10F8300016F0FDC8E6FFFEC8E6FF620EE66E2A0E71
:10F84000E66E010E44EC8DF08DEC16F057EC8FF067
:10F85000FBC8E6FFFCC8E6FF220EE66E2A0EE66E47
:10F86000010EE66EFBC814F0FCC815F0320ECBECAE
:10F870008BF053EC90F08DEC16F084EC92F036DFC8
:10F8800033EC87F00A0E8EEC92F00B0EFCEC86F057
:10F8900036DF33EC87F00C0E8EEC92F00D0EFCECA4
:10F8A00086F034DF33EC87F00E0E8EEC92F00F0E04
:10F8B000FCEC86F0010EE66E140EFCEC86F0010105
:10F8C000010EA46FB3DEDF6E5AEC8DF002E2DFCFE3
:10F8D00000F192EC92F003E0A8EC88F0FDE1D5ECA9
:10F8E00086F0DB1C62EC90F001010117020EDB5088
:10F8F0000217020EDB500317020EDB500417020E34
:10F90000DB501F17A56BA66B4CEC75F0DF6A010E80
:10F91000DB6A050EDF5C06E2F3EC92F08CEC8BF018
:10F92000DF2AF7D7010EDB1C12E0010EDB1C0601FB
:10F930009C11E66E040EE66EBBEC89F0010EDB5006
:10F9400006019C15E66E040EE66EC0EC89F026C139
:10F9500095F1DF6A050EDF5C0CE2F3EC92F0020E2B
:10F96000DB50EF160EEC95F002E0ABEC8DF0DF2AE9
:10F97000F1D725EC93F0F4EC88F0BCEC88F003E0D0
:10F98000C5EC89F0FDE1BDEC87F000C1DFFFDF5081
:10F9900074E015EC86F0EF6A15EC86F0070E1DECAE
:10F9A00091F0030E1DEC91F0040E1DEC91F0F4ECBF
:10F9B00085F0020EEF6E08EC87F0EF6ADF04EA6A6A
:10F9C000D80FE96E000EEA22600EEF6EC5EC88F0EB
:10F9D000156ADF34FE0B1536146E900E1426000ED9
:10F9E0001522020E145E000E155A53EC90F085ECB1
:10F9F00087F0E552DF04EA6A120FE96E090EEA2287
:10FA0000EF6A15EC86F0020ECAEC94F0030EDB50A0
:10FA10000801B31505E0AEC8E6FFAFC8E6FF08D0A1
:10FA2000030EDB50B41508E0B0C8E6FFB1C8E6FF2E
:10FA3000F2EC8CF0A7EC90F0DF0493EC8BF0B2C802
:10FA4000EFFF030EDB500801B9150EE0B7C8E6FF63
:10FA5000B8C8E6FFF2EC8CF0B80E1426000EFCECF1
:10FA600085F085EC87F0E552030EB1EC86F0D950B5
:10FA7000040F94EC86F0DF068AD7E66A080EE66E7D
:10FA80008EEC37F0E552E552CEC8E6FFCFC8E6FF70
:10FA900042EC03F0E552E552D1C8E6FF03EC03F077
:10FAA000E552E66A9AEC89F0010EE66E9AEC89F06E
:10FAB000020EE66E9AEC89F0030EE66E9AEC89F07F
:10FAC0000101880EB36F060EB46FB56BB26BE66AB8
:10FAD00062EC8DF0450EE66E0D0EE66E90EC00F0D9
:10FAE00089EC87F06FEC86F006C0B6F107C0B7F17D
:10FAF00008C0B8F109C0B9F10101AD6B080EAE6FD5
:10FB0000916F90EC8CF001017A6BB06BAF6BB16BC5
:10FB10000501506B0F01006B0101896B8D6B8E6BC2
:10FB20008F6B6FEC86F006C07BF107C07CF108C0DC
:10FB30007DF109C07EF171EC8BF03BEC8BF00101A3
:10FB40008A6B8B6B8C6B926B936B946B0601FE6B69
:10FB50000601FF6B0101010E776FE80E5D6F030E6A
:10FB60005E6F7F0E5F6F996B9A6B9B6B9C6B9D6B4F
:10FB70009E6B9F6BA06BA16BA26BA36B96ECA9F025
:10FB80000101A86BA96BAA6BAB6BDF6A050EDF5C8A
:10FB900003E26AEC8DF0FAD70101A45107E0080EE8
:10FBA000AE6FAD81E66ED2EC29F0E552080EE15C55
:10FBB00002E2E16AE552E16EC8EF85F0CDEC8DF02E
:10FBC0004AEC8FF067E2BCEC86F003E02FEC87F0A4
:10FBD000FDE1F350DF6EDF500801D21503E064EC65
:10FBE0008CF003D0580EE66E040EE66E8EEC91F0AB
:10FBF0007AEC87F0DF500801D31508E0940EE66E2A
:10FC0000040EE66E8EEC91F00AEC8AF08EEC91F028
:10FC1000E66E8EEC91F0E66E90EC94F0090ED9EC65
:10FC200088F04EEC8FF08EEC91F07AEC87F04EEC91
:10FC30008FF04EEC8FF090EC94F0170ED9EC88F02A
:10FC40000BEC8EF0EE52EF040FE1D7C8E6FF0A0E80
:10FC500022EC87F0D6C8E6FF190E22EC87F0D4C854
:10FC6000E6FFD5C8E6FF0ED0DBC8E6FF0A0E22ECA1
:10FC700087F0DAC8E6FF190E22EC87F0D8C8E6FF55
:10FC8000D9C8E6FF0B0E98EC93F014EC19F0D9EC00
:10FC90008DF0E552E552C8EF85F001EC8EF036ECC0
:10FCA0008FF029EC93F0100ED880F354000EF4542A
:10FCB00008E2100EE76ECEEC86F0E750F4EC85F02B
:10FCC000EF6A310E6BEC89F04CEC8DF034EC91F076
:10FCD0004CEC8DF04CEC8DF090EC94F0160ED9ECD1
:10FCE00088F0DE6A200EDD6E020E60C1DBFFDECF23
:10FCF000E6FF43EC87F0DD5238EC88F0030EE15C60
:10FD000002E2E16AE552E16EC8EF85F099EC8DF010
:10FD1000BCEC86F003E02FEC87F0FDE1F350DF6EE2
:10FD20004AEC8FF03EE2E66A1BEC89F0010EE66ECB
:10FD30001BEC89F0020EE66E1BEC89F0030EE66EFA
:10FD40001BEC89F00FEC8EF039DFE55260CDE6FF59
:10FD5000220E22EC87F0DF500101291522E0230E4C
:10FD600014EC87F0FE0EDB50EA6AC60FE96E080E4F
:10FD7000EA22EF50800B03E0240E14EC87F0D950F8
:10FD8000010F04EC95F063EC8AF0DFEC91F0D4EC19
:10FD900085F0010EDB5005E004EC87F0260E22EC26
:10FDA00087F0020EE15C02E2E16AE552E16EC8EF23
:10FDB00085F0CDEC8DF000C1DFFFDF5006E0DF0401
:10FDC000E66EA4DFE552DF06F8D7E552C8EF85F00E
:10FDD0003FEC90F0010197EC92F008EC95F01414D0
:10FDE000151402EC89F097EC92F0030E77EC8DF08D
:10FDF000141415143AEC90F097EC92F0AFEC93F0E9
:10FE00001414151435EC8DF0BCEC88F003E0C5EC4F
:10FE100089F0FDE1DF6E25EC93F0FEEC91F0030E2E
:10FE200000C1DBFFDB5001E180D0B8EC8FF0DF14C4
:10FE300076E0040EDB50DF1426E00101921D146E03
:10FE4000C1EC88F05EEC8DF01414E66E40EC8EF0A0
:10FE50008EEC87F0DF500115931504E1931D95ECAE
:10FE600094F0EF16A51D146EDF500315141403E073
:10FE700040EC8EF0EF6A0351A515E81C146EDF50BC
:10FE80009415141403E040EC8EF0EF6A050EDB507D
:10FE9000DF1404E040EC8EF0DF50EF12ACEC8CF09D
:10FEA000880E145E060E155A050E0D6E0E6A14C0ED
:10FEB00008F015C009F009ECB5F008C014F009C04D
:10FEC00015F0010E08C0E7FFE75203E0A8EC88F048
:10FED000FDE10101951511E142EC86F0AFEC93F0E4
:10FEE000DF140BE1DF50071504E040EC8EF0075102
:10FEF00003D0071D95EC94F0EF16060EDB50DF14CF
:10FF000005E040EC8EF0060EDB50EF16060EDB1C13
:10FF1000DF1405E0060EDB1C95EC94F0EF16DF9085
:10FF2000DF42EBEC90F0DB067DD7070EE15C02E2EE
:10FF3000E16AE552E16EC8EF85F0BBEC92F003E0B8
:10FF40002FEC87F0FDE152EC8EF011E09BEC92F08B
:10FF5000DF50EF12DF500101031505E0DF1CA5178C
:10FF6000DF502715941328EC86F0010E01D0000E07
:10FF7000E552C8EF85F0BBEC92F003E02FEC87F080
:10FF8000FDE152EC8EF010E0DF1C146E9BEC92F061
:10FF90001450EF16DF500101031502E0DF1CA51716
:10FFA00028EC86F0010E01D0000EE552C8EF85F076
:10FFB0009BEC92F0EF6AB3EC8FF0ECEC92F001EC7A
:10FFC00094F00101A51728EF86F0EFEC92F0D4EC45
:10FFD0008EF0146E58EC90F0EF12B3EC8FF0040E2C
:10FFE000F4EC85F0FE0EDBCFEFFF28EC86F0C8EFD7
:10FFF00085F072EC92F066EC92F0DF5205E0DFCF14
:020000040001F9
:10000000F3FFC9EC89F0FDE1E552E710156E2EEC27
:1000100086F01514146E58EC90F0EF120101011DDA
:100020000715156E66EC92F0DF5205E0DFCFF3FFA7
:10003000C9EC89F0FDE1E552E7101510146E2EECC5
:1000400086F01414E66E040EC7EC92F028EC86F0ED
:10005000E552C8EF85F0BBEC92F003E02FEC87F09F
:10006000FDE1F350DF6E26EC89F0EB50DF14010167
:100070000315A61507E0DF50A513DF502815CEECB9
:1000800090F001D0010EE552C8EF85F0BBEC92F084
:1000900003E02FEC87F0FDE19AEC94F007E0DF1C21
:1000A000A517DF502715CEEC90F001D0010EE552D8
:1000B000C8EF85F0BBEC92F003E02FEC87F0FDE198
:1000C0009AEC94F005E0DF5027134EEC8CF001D051
:1000D000010EE552C8EF85F0BBEC92F003E02FEC87
:1000E00087F0FDE19AEC94F005E0DF1C27174EEC59
:1000F0008CF001D0010EE552C8EF85F0CDEC8DF00B
:100100000101031DA517035127159413DF6A050E7E
:10011000DF5C11E2F3EC92F0EE52EFCF15F001014B
:10012000031D1510146EF3EC92F058EC90F0EF16DE
:100130006AEC8DF0ECD7E552C8EF85F0C3EC85F0A2
:10014000F9EC8CF003E0A8EC88F0FDE1E81CDF6E30
:10015000010EDB6A050E4EEC87F021E2E6EC94F02E
:10016000DF50EF16010EB4EC94F058EC8CF05EEC1E
:1001700093F01414E66EE6EC94F0020EC7EC92F0E5
:10018000010EFCEC94F0E66EE6EC94F00BEC95F0CE
:10019000E6EC94F0ECEC92F0010EDB2ADBD726C102
:1001A00095F1020EE15C02E2E16AE552E16EC8EF10
:1001B00085F0C3EC85F0F9EC8CF003E0A8EC88F056
:1001C000FDE1E81CDF6E050E24EC86F039E2FE0E40
:1001D000E7EC8DF0DF50EF16FE0EB4EC94F0EFCFAD
:1001E00014F0FE0E5EEC93F0141463EC8AF0CCEC89
:1001F00085F0020EC7EC92F0FE0EFCEC94F063EC7E
:100200008AF0CCEC85F00BEC95F0FE0EE7EC8DF06F
:10021000ECEC92F0BCEC86F003E02FEC87F0FDE113
:10022000F35001012615146EBCEC86F003E02FECB0
:1002300087F0FDE1F350F31C010195151410956F43
:10024000010EDB6A050E4EEC87F018E294EC8AF0A2
:1002500012E0E6EC94F0DF500EEC93F058EC90F0E6
:100260000EEC93F058EC91F00EEC93F0040EF4ECDD
:1002700085F01450EF16010EDB2AE4D7020EE15C84
:1002800002E2E16AE552E16EC8EF85F02AEC91F0F6
:1002900080EC93F09C0EEE6E060EED6E03EC86F095
:1002A000020ECAEC94F003EC86F0CAEC94F005EC74
:1002B00092F070EC88F001E3DB2AEFCFDFFFDF5034
:1002C0001BE084EC93F013E0300EDF5C146E080E3C
:1002D000145CEFE2C7EC8FF0ECE2010EF36EDB5042
:1002E00003E02FEC87F0FDE158EC8EF0E2D75AECFA
:1002F00094F0DFE1010E2AD0D2EC8FF0040EF36E01
:10030000050EE6EC8EF00AE2A5EC93F0050EE7ECA4
:100310008DF0ECEC92F0050EDB2AF0D7040EE66EC1
:1003200048DFE552100E01012615146EEF0E9515EB
:100330001410956F050EDB6AABEC89F006E2050E32
:10034000A6EC8DF0FDEC8CF0F7D7000E146E060EC7
:10035000E15C02E2E16AE552E16E1450C8EF85F01B
:100360003FEC90F042EC86F0EFCFDFFFDF500CE087
:100370005CEC8FF016BE1768B7EC92F005E0E7EC86
:1003800089F0F0E3DB2AEED7AFEC8FF0F350F410F6
:1003900037E0300EDF5C35EC8DF0050EF36E060EA7
:1003A000E6EC8EF02DE2E7EC89F001E3DB2A060EA5
:1003B000DB50E3EC94F0E6EC86F005EC92F070ECA8
:1003C00088F001E3DB2AEFCFDFFFDF501BE084EC96
:1003D00093F013E0300EDF5C146E080E145CEFE255
:1003E000C7EC8FF0ECE2010EF36EDB5003E02FEC74
:1003F00087F0FDE158EC8EF0E2D75AEC94F0DFE1A3
:10040000010E22D0D2EC8FF0ABEC89F00CE2060E9C
:10041000DB50F36E050EDB50F35C02E0A5EC93F0CD
:10042000050EDB2AF1D7060EDBCFE6FFC2DEE55272
:10043000050EDB6AABEC89F006E2050EA6EC8DF04A
:10044000FDEC8CF0F7D7000E146E070EE15C02E2B3
:10045000E16AE552E16E14509BD3CDEC8DF013ECC4
:100460008EF06CDEDF6A050EDF5C03E26AEC8DF075
:10047000FAD7E5528DD399EC8DF0DF6A70EC88F0F5
:1004800001E3DB2AD9EC8AF01CE004EC87F0E66A91
:1004900000EC95F0F3E120EC91F0F4CF15F0F3507F
:1004A000F4100FE0380E4EEC87F00BE2010EDB503B
:1004B000D00FA7EC91F003E0C5EC89F0FDE1DF126D
:1004C000DDD7DF50E0EC8BF002E2E16AE552E16E4D
:1004D00014505ED301EC8EF0D5DBD9EC8AF00CE041
:1004E0005CEC8FF016BE1768B7EC92F005E0E7EC15
:1004F00089F0F2E3DB2AF0D720EC91F08CEC8DF060
:1005000003E002EC8DF002E3010E3BD0E7EC89F052
:1005100001E3DB2A62EC93F0F3EC92F08CEC8BF0CD
:10052000DBCFE6FFDFCFE6FFBBEC89F0020EDB6A34
:100530006AEC87F01DE2DF50F36E020EDB50F35CD5
:1005400014E004EC87F0020E5EEC93F0E552E71441
:100550000CE0010EDB1C146E020E5EEC93F0141422
:10056000E66E52EC87F0BBEC89F0020EDB2AE0D796
:1005700051EC8DF06AEC87F003E2DBEC93F0FAD7F4
:10058000000E2DEC8AF002E2E16AE552E16E1450B1
:10059000FFD201EC8EF076DBD9EC8AF00CE05CEC5B
:1005A0008FF016BE1768B7EC92F005E0E7EC89F023
:1005B000F2E3DB2AF0D720EC91F08CEC8DF003E035
:1005C00002EC8DF002E3010E16D0E7EC89F001E3B6
:1005D000DB2A62EC93F0B0EC90F0E66EDFCFE6FF42
:1005E000C0EC89F051EC8DF06AEC87F003E2DBECB3
:1005F00093F0FAD7000E2DEC8AF002E2E16AE552A0
:10060000E16E1450C5D201EC8EF08BEC8EF006E258
:1006100053EC8FF0FE0EEFCFDBFF02D0010E3BD08C
:10062000020EDB6A6AEC87F02DE213EC8EF0020E0C
:10063000B4EC94F0010EEFCFDBFFFD0EDB500DE0CC
:100640009BDB03E02FEC87F0FDE1F350146E010E0D
:10065000DBCFE7FFF350E7120AD08EDB03E02FEC8D
:1006600087F0FDE1F350F31CBBEC8BF0E7169FEC39
:1006700092F0DBCFE6FF52EC87F0C0EC89F0020E7F
:10068000DB2AD0D751EC8DF06AEC87F003E2DBEC8B
:1006900093F0FAD7000E2DEC8AF002E2E16AE552FF
:1006A000E16E145075D24FEC91F0F80EDBCFE6FFFF
:1006B000F90EDBCFE6FF65DB020EF3CFDBFF080EA2
:1006C000DB6ADE6ADD6A88DBFA0EDBCF16F0FB0E32
:1006D000DBCF17F01650145C1750155862E2080E65
:1006E000DB505FE12BEC8BF0060EF626000EF722B6
:1006F000F8220900F5CF18F00800F5CF19F01850CE
:1007000019104FE0F80EDBCF08F0F90EDBCF09F03F
:10071000030E08C0DBFF040E09C0DBFF2BEC8BF0DF
:10072000F6CF14F0F7CF15F0F8CF16F09EEC8CF062
:10073000070E16C0DBFF4CDAEFCF14F045EC8AF061
:10074000145C11E145DAEF500EE0030EDB2A040ED3
:1007500001E3DB2AD950050FEBEC8EF0EE2A000EF8
:10076000EE22EE22E8D734DAEF5003E0080EDB6A1F
:100770000AD045EC8AF002E0010E01D0020EF36EC1
:10078000080EF3CFDBFFD950FC0F7FEC92F0090E7F
:10079000EE26000EEE22EE22DF2A010E94E3DB2A83
:1007A00092D7080EDB5002080AE116DB1406000E91
:1007B000155AF60EDBCFE9FFF70E09EC8DF0080EA7
:1007C000DB50146E0A0EE15C02E2E16AE552E16E72
:1007D0001450DED1D8D9090EE126FBEC88F0070EC3
:1007E00008C0DBFF080E09C0DBFF060EDB6ADE6A0D
:1007F000DD6AF2DAFC0EDB50176AE850145C175021
:10080000155849E2060EDB50020845E0F90EDBCF31
:1008100008F0FA0EDBCF09F0020E08C0DBFF030E72
:1008200009C0DBFF070EDBCF08F0080EDBCF09F0B5
:100830002BEC90F0E8D9EFCF14F0F7D9EF50145C1F
:100840000EE1E1D9EF500BE0020EDB2A030E01E3CB
:10085000DB2A040EDB2A050EEDE3DB2AEBD7D3D926
:10086000EF500AE1E2D9EF5002E0010E01D0020E92
:10087000F36E060EF3CFDBFFFB0EDB50146E156A32
:10088000B1EC8BF01450EE261550ED22DF2A010E4C
:10089000B0E3DB2AAED7060EDB5002080AE19CDA91
:1008A0001406000E155AF70EDBCFE9FFF80E09EC1F
:1008B0008DF0060EDB50146E090EE15C02E2E16A77
:1008C000E552E16E145064D101EC8EF08BEC93F0A4
:1008D0008FD97DDB000902E0FF0E2FD0DF6A140EF6
:1008E000DF5C06E283EC8BF0EF5002E0DF2AF7D703
:1008F000140EDF5C21E2F8EC94F0070EF35C000EBE
:10090000F4581AE209EC92F0610F146E0D0E74D9CE
:100910002CECABF0D6EC94F0070EE66E09EC92F0FE
:10092000E40F146E010E68D978EC6AF0166E050EAD
:10093000E15E1650DF5001D0FF0E2DEC8AF002E28E
:10094000E16AE552E16E145023D199EC8DF0F4EC9C
:1009500094F08CEC8DF00DE0F4EC94F0B1EC89F0B7
:10096000070EF35C000EF45804E210EC92F000095C
:1009700002E0FF0E0CD03CD9610EE66E0D0EBADA25
:10098000070EAEEC94F0E40E79D99ED9000EE0EC9F
:100990008BF002E2E16AE552E16E1450F9D001EC0D
:1009A0008EF0020E146EE66E8BEC93F021D908ECFB
:1009B00090F0156E080E16EC92F002E0FF0E02D0D9
:1009C000010EDB502DEC8AF002E2E16AE552E16EA5
:1009D0001450DED001EC8EF010EC92F062EC90F04E
:1009E000020817E1F9D9153414E214500008000E7A
:1009F00015540FE2E3EC8AF0070ED7EC90F010EC00
:100A00008DF0EAD9070EC2EC93F083EC91F0DF5041
:100A100001D0FF0E2DEC8AF002E2E16AE552E16EB0
:100A20001450B6D0EFEC92F0DB50000817E2140E31
:100A30000BD914E216EC89F0610EE9260D0EEA22BC
:100A4000EF500CE0F3DB10EC8DF0FE0EDB50070DE9
:100A5000C6D883EC91F0FE0EDB5001D0FF0E98D08B
:100A6000CDEC8DF0DF68DF500AE0DF50EA6A000F5E
:100A7000E96E0E0EEA22EF5002E1DF06F4D7DF50F6
:100A8000146E156AFF0ECBEC8BF01450E55280D03B
:100A9000D9CFE6FFE1CFD9FFE652010E0101AD1536
:100AA0001BE101017851791117E10601FE5114E1B2
:100AB00091EC04F0000910E1450EE66E0D0EE66EB5
:100AC000A6EC00F0E552E55206C0B6F107C0B7F15A
:100AD00008C0B8F109C0B9F1450EE66E0D0EE66E1C
:100AE000A6EC00F0E552E5520101B651065C146E29
:100AF0000101B7510758156E0101B8510858166E1B
:100B00000101B9510958176ED880780E1454000E9F
:100B10001554000E1654000E175410E2010EE66E26
:100B2000F1EC05F0E552DF6EDF2ADFCFE6FF010EC4
:100B3000E66EFBEC05F0E552E552FF009D50020B1E
:100B400009E09D50010B06E0F250800B03E0F250EB
:100B5000400B10E1020EE66EF1EC05F0E552DF6E9F
:100B6000DF2ADFCFE6FF020EE66EFBEC05F0E55272
:100B7000E552FF000501505101E10400E552E55244
:100B8000E7CFD9FF1200D9CFE6FFE1CFD9FF12009E
:100B9000E552E7CFD9FF1200050D4EEC90F0880E1C
:100BA000E926060EEA221200C1EC6AF0CBEF92F0C1
:100BB00084EC6AF0D9EF8DF00B0D4EEC90F0000E46
:100BC000E926040EEA221200B3EC6AF006EF8EF07A
:100BD000030EDBCFE9FF040EDBCFEAFF1200F3CFF9
:100BE00014F0F4CF15F01200E926000EEA221200EC
:100BF000FDEC93F00FEF8EF0152253EF90F08EEC9A
:100C00006AF0CBEF92F0020EDBCFE9FF030EDBCFF1
:100C1000EAFF1200050EDBCFE9FF060EDBCFEAFF8D
:100C20001200EA6ADB346DEF91F0040EDBCFE9FFCE
:100C3000050EDBCFEAFF1200640E1426060E152205
:100C4000F0510F01D5EF93F0F36EFE0EE6EF8EF04C
:100C5000B3C1E6FFB4C1E6FF93EF93F0B3EC8FF0BE
:100C6000EF501200A5ECB5F006EC8EF01DEC92F002
:100C7000060EDBCFE6FF070E8AEF91F0E66E010E5F
:100C8000E66E1200FD0EDBCFE9FFFE0EDBCFEAFFC2
:100C90001200E66E030EE66E120005EC93F057ECC0
:100CA0008FF0EAEF8DF0ECEC8FF0120FE96E090E89
:100CB000EA221200E76E9FEF92F0010EDBCFE9FF10
:100CC000020EDBCFEAFF120078EC6AF006EF8EF03E
:100CD00038EC91F00B0E145E000E155A1200450E02
:100CE000E66E0D0EE66EA6EC00F0E552E55212003F
:100CF000FB0EDBCFE6FFFC0EDBCFE6FF1200E5527A
:100D00000FEC8EF0E7EC75F0E5520FEC8EF069EC2D
:100D10006CF0E5520101936B93C192F192EF92F066
:100D200024EC92F0B6EF93F0EBEC8EF00B0EEE5E4F
:100D3000000EEF5A1200E81C3AEC90F0DB50010173
:100D40000117050EDB500217050EDB500317050EC9
:100D5000DB5004179EEC80F0DF6A1200DB502BEFB3
:100D600092F0DBCFF3FFF390F342F3CFDBFF1200FF
:100D7000CBEC6AF0CBEF92F0010EF36EFE0EDB507F
:100D8000120066ECABF0E552E5521200E66EEAECBA
:100D90008DF05EEF94F0030D4EEF90F0FC0EDBCF84
:100DA000E9FFFD0EDBCFEAFF1200E76E020EE7CF90
:100DB000DBFF12000FEC8EF060EC2AF0D9EF8DF023
:100DC000E66EE66AA2EC6AF0CBEF92F0880E14268B
:100DD000060E1522CDEF8EF0DECF14F0DDCF15F02C
:100DE0001200D9CFE9FFDACFEAFF1200EA6A0A0F50
:100DF000E96E090EEA221200E66E89EF92F016C043
:100E0000E6FF17C0E6FF1200010EDBCFE6FF12007F
:100E1000DF04E96EEA6AD890E936EA36C80EE926B8
:100E2000000EEA22EE52120098EC93F0D5EC18F086
:100E3000E552E552120018EC16F064C7E9FF65C7E9
:100E4000EAFF120098EC93F00EEC19F0D9EF8DF058
:100E5000ECEC8FF0700FE96E000EEA221200D890D1
:100E6000F336E80612001DEC92F0FF0EE76E1DEC63
:100E700090F0E7501416156A1450E66E1200B6ECA6
:100E800093F0E66A1200DECFE6FFDDCFE6FF120048
:100E900025EC91F003EC9DF0CBEF92F0F36E010E98
:100EA000E6EF8EF0020EDBCFE6FF1200FE0EDBCF88
:100EB000C1F146C141FDAEC1E6FFB1EC23F0E55200
:100EC0000101AD811200ECEC8FF0680FE96E000EAD
:100ED000EA221200050EF36E020EE6EF8EF0E66EC9
:100EE0004DECABF006EF8EF0AEC1E6FF60EC2AF001
:100EF000D9EF8DF0E66E2CECABF0CBEF92F0156AEB
:100F0000DB34FE0B1536146E120069EC00F0D9EFDD
:100F10008DF0146E060EE15E14501200E552E7509B
:100F2000EF6E1200E12631EC92F0010EDF5212005A
:100F3000E66E94EC38F0D9EF8DF0E66EF1EC05F04A
:100F4000E552120036EC8FF06DEF94F0E66A94EC07
:100F50009CF0156E060E16EF92F074ECABF0D9EC27
:100F60008DF0140E075C000E0858000E0958120090
:100F7000D9CFE6FFDACFE6FF1200E76E030EE7CF28
:100F8000DBFF1200C3EC17F0E552E5521200E66AEF
:100F90008DEC9BF057EF8FF00C6E0D6A0E6A1AC045
:100FA00007F01BC008F01CC009F02FECB5F004C01E
:100FB0001AF005C01BF006C01CF017500424146E74
:100FC00018500520156E19500620166E120008ECF8
:100FD00090F0146E080EE15E1450120098EC93F03D
:100FE000F3EC18F006EF8EF006C0DEFF07C0DEFF60
:100FF00008C0DEFF09C0DDFFDD52DD521200FE0E2B
:10100000DBCF76F10101010EB26F1200E9CF14F0CF
:10101000EACF15F0E9CFE6FFEACFE6FFDECF16F024
:10102000DDCF17F0050E1702F3CF17F01602F3CF3E
:1010300016F0F45017260E0E1626000E1722120078
:10104000050ED7EC90F0880EE926060EEA22120073
:10105000D5EC17F0E552E5521200B2EC93F0E66ED3
:1010600080EC93F076EC92F023EC94F066EF91F044
:101070000FEC8EF09EEC19F0CBEF92F0EE58000ED4
:10108000EE58000EEE581200B3EC8EF0152201015E
:10109000B35114181200A5ECB5F006EC8EF00A0E50
:1010A000F3CFDBFF0B0EF4CFDBFF12001C50185CFC
:1010B000146E1D501958156E1E501A58166E1F507A
:1010C0001B58176E1200EE50185C146EEE50195833
:1010D000156EEE501A58166EEE501B58176E120011
:1010E000FD0EDBCFE9FFDB2AFE0EDBCFEAFF1200AD
:1010F000ECEC8FF0800FE96E000EEA221200ECECAF
:101100008FF04D0FE96E010EEA221200ECEC8FF029
:10111000550FE96E010EEA221200DBCFF3FFF39EBA
:10112000F346F3CFDBFF12002E0EE66E610EE66E85
:10113000010EE66E1200146E156AFF0E14181200EE
:10114000C0EC91F02BEC90F080EC93F075EF94F004
:10115000E846FE0BE70612001DEC90F015C014F0F7
:10116000156A1450E66E1200F350DF6E8BEF93F0A9
:101170002BEC94F0FFEF90F00005146E010E14526A
:101180001200040EDBCFE6FF1200000EE66EE66AE8
:101190001200080EE66E610EE66E010EE66E940E0B
:1011A000D0EF92F0176ED8801E0E1454000E38EF58
:1011B00092F098EC93F0F3EC18F0166E050EE15EE9
:1011C00016501200030E14C0DBFF040E15C0DBFF27
:1011D0001200D950FD0F7FEF92F0040EDBCF14F018
:1011E000050EDBCF15F01200040E14C0DBFF050E58
:1011F00015C0DBFF1200FD0EDBCF08F0FE0EDBCFCB
:1012000009F01200E76E040EE7CFDBFF1200E96E73
:10121000000EDA20EA6E1200146EEF501414E66E1F
:101220001200E66AC9EC9CF057EF8FF0FE0EDB501F
:10123000070D4EEF90F00FEC8EF0C9EC38F0E55250
:10124000E5521200B3EC8FF0030E1200B3EC8FF0F6
:10125000020E1200146E050EDBCFE7FF1450E716E6
:10126000050EE7CFDBFF1200050EE66E4EEC8FF0A9
:101270005B0EE66EE66A12009E0ED0EF92F005EC71
:1012800093F0146E0B0EE15E1450EAEF8DF0020E37
:10129000DBCF07F0030EDBCF08F0040EDBCF09F045
:1012A000050EDBCF0AF00A34000E0A1812001A24C9
:1012B000186E000E1B20196E18C0E6FFE66E78EC63
:1012C0006AF01C6E050EE15E1C501200FEEC91F0FF
:1012D00000C1DFFF1200E66EE66A36EF8FF0A51759
:1012E000EF50E81C9417EF500315271594131200C4
:1012F000EF6E020EDB5001016C13020EDB50071380
:101300001200DB50EA6AD80FE96E000EEA221200E2
:10131000E552E552F3CFDEFFF4CFDDFF1200F36EAE
:10132000FD0EE6EF8EF037ECB7F0146E090EE15EBD
:1013300014501200080EE66EC9EC38F0E552E55282
:101340001200D9EC8DF0DF6EDF501200EBEC8EF066
:10135000EE50ED101200F36EDBCFF4FFE850F45CBA
:101360001200F3CF16F0F4CF17F01200010EB5C142
:10137000E7FFE752120091EC6EF0E552E5521200E1
:10138000A6EC6EF0E552E5521200E846FE0B14069C
:101390001200E846FE0BF306120053EC90F0EAEC64
:1013A00017F0E552E552F350E66E8DEC24F0E5526D
:1013B0001200DECF07F0DECF08F0DECF09F0DDCF80
:1013C0000AF0DD52DD520A34000E0A181200FD0E3A
:1013D000DB2AFE0E1200EFCF16F0176A1200E66E3F
:1013E000D950080F1CEC8EF06DEF94F0ECEC8FF000
:1013F000600FE96E000EEA221200EA22EECFE6FF4D
:10140000EECFE6FFEFCFE6FF1200E66EF8ECABF0B2
:1014100057EF8FF0E66ED6ECAAF0CBEF92F0E652E3
:1014200031EF92F00FEC8EF0D1EC33F0E552DF6E3D
:101430001200E66A8DEC9BF084EF92F0F36E020EE0
:10144000F3CFDBFF1200010EDB500101AE5D120095
:101450009217EF50E81C93171200146E030EE15C14
:101460001200FE0EDB5008081200E66EE66AFB0E64
:10147000DBCFE6FF24EF92F0E66EE66AB5EC15F0FE
:10148000D6EC94F00F01086B1200050EDBCFF6FFCF
:10149000060EDBCFF7FF070EDBCFF8FF0800F55095
:1014A0001200E1EC23F0080E0101AE5D12003AECEF
:1014B0002DF0E552E552000912000854000E0954BF
:1014C000000E0A541200E66EFE0EDB501200DFCF53
:1014D000E6FFE66A1200146E040EE15C12000101E0
:1014E000EF51040D12000A0EDBCFE6FF0B0E8AEF60
:1014F00091F0030EDBCF14F0040EDBCF15F0080ED5
:1015000066EF91F0080EE66EBE0EE66E080EE66E11
:10151000A70ED0EF92F0080EE66EC60EE66E080E2D
:10152000E66EAF0ED0EF92F0FE0EDB50F36E010EC2
:10153000DB50F35C12002FEC91F08FEFADF0DF0485
:10154000EA6A780FE96E000EEA221200DF2A020E24
:10155000DBCFF3FFF39EF3461200DF502BEF92F048
:10156000640E1426060E1522FD0EDB501200D95013
:10157000020F146EDACF15F0DF501200FE0EDB1CE6
:1015800001010217FE0EDB1C1200040EDBCF04F17A
:10159000B6EF93F093EC93F0020EDB2A1200E66EA6
:1015A0007AECADF0E552120006C0DEFF07C0DDFFA9
:1015B0001200010EEFCFDBFFEF501200E126040E08
:1015C000E66ED9501200DECFE9FFDDCFEAFF120050
:1015D000EF50E66EF0C1E6FFEFC1E6FF7DEC38F0BC
:1015E000E5521200080EE66E0A0EE66E090EE66E71
:1015F000060EE66EE66A1200DFCFE9FF010EDBCFD2
:10160000EAFF0A0EE926090EEA221200EA22FD0E7E
:10161000DBCFEFFFFDEC93F0FE0EDB501200C9DADA
:10162000A10EE66E5F0EE66E010EE66E1200080E6B
:10163000E66E4D0EE66E010EE66E4B0EE66EE66A47
:101640001200080EE66E550EE66E010EE66E530EA3
:10165000E66EE66A1200FC0EDBCFF6FFFD0EDBCF76
:10166000F7FFFE0EDBCFF8FF1200DFCFE6FF9EECA8
:1016700019F0CBEF92F006C07FF107C080F108C0EF
:1016800081F109C082F112001450185C15501958EC
:1016900016501A5817501B5812000101AE51EA6A31
:1016A000700FE96E000EEA22EF501200E0EC93F0AA
:1016B000020EE66E120005EC93F0166E1200030E99
:1016C000DBCFE7FFF350E712030EE7CFDBFF12009B
:1016D000AEC1E6FFBBEC29F0E5520101786B796BF6
:1016E000120006C083F107C084F108C085F109C06B
:1016F00086F112001A1D156E030EDB50F36E030EF9
:10170000DB50F35C1200070EDF02F350EA6A610F50
:10171000E96E0D0EEA221200010EDBCFE7FFEF505B
:10172000E7129FEF92F0EA6AB00FE96E000EEA222C
:101730001200EA6A000FE96E070EEA221200F3CFE8
:1017400018F0F4CF19F0F3501200186A196A010E5C
:101750001A6E1B6A1200141401010115E81C6D17A2
:101760001200D950070FEBEF8EF0E66E51EC7BF0D4
:10177000E55200091200146E010EDBCFE7FF145092
:101780001200010EF36EFD0EDB5012006E1D156E81
:101790006D1D146E1200D8801456000E15561200DE
:1017A000A00ED0EF92F0A10ED0EF92F0DB50E552F8
:1017B000E710E66E1200140EF35C000EF4581200EF
:1017C000146E020EE15C1200020E0101AD15120052
:1017D000DB50E552E7141200DB5001010115120045
:1017E000E652030EE66E1200FB0FE66EFF0EDA20E5
:1017F000D0EF92F0F90FE66EFF0EDA20E66E040EDF
:10180000E66E1200070E7615E66E56EC1DF0E552F8
:1018100000091200020EE126DE52010EDD6E00C14B
:10182000DFFF1200D8DA1450EE121550ED1212003C
:101830001454010E38EF92F0080EDB50EA6ADF0F05
:10184000E96E010EEA221200010EF36E090EF3CFCB
:10185000DBFF080EDB6A1200166E020EEB50161448
:10186000156E010EEB501200B7DB880FE96E000E0B
:10187000EA2212000101080EAE6FF20EE66E080EAB
:10188000E66E1200166A176A3C0E0B6E0C6A0D6A41
:101890000E6A1200D6ECB1F0CBEF92F0C0D946EC54
:1018A00080F0E552000E1200020EDB500F0B12000A
:1018B000EFCF14F0010E1200E126010100511200D9
:1018C000EE52EF50020812006C0EE66E040E12008B
:1018D000010E176ADB34FE0B1736166E1200E80E87
:1018E000E66E610EE66E010EE66E1200DF04E66E35
:1018F000F7EC1BF0E55200091200E552E7CF17F0B4
:10190000E552E7CF16F01200E552E7CF15F0E552A9
:10191000E7CF14F0120083D950EC22F0E552120008
:101920000701006B000E646F070E656F1200FB0E5F
:10193000DBCFE9FFFC0EDBCFEAFF1200050E14C07F
:10194000DBFF060E15C0DBFF12000101020EB26FB5
:10195000FE0EDBCF76F11200FD0EDBCF14F0FE0E93
:10196000DBCF15F01200F36E080EE6EF8EF0DFCF3E
:10197000E6FF54EC24F0E552DF2A1200F4DA010EFF
:10198000EB501200F3501B6A700F1A6E020E1B22EE
:101990001200EF50E66EF0C1E6FF13EF6AF0050D9E
:1019A000F3CFB3F1F4CFB4F1880E1200020EDBCF07
:1019B00002F1030EDBCF03F1120078EC6AF0186E2F
:1019C000050EE15E18501200A90EE66E5F0EE66E7F
:1019D000010EE66E1200E66EE66A15EC00F0E552C6
:1019E000E5521200DF04146E156AD89014361536CD
:1019F0001200020EE12692EF92F093EC93F0050EA6
:101A0000DB2A1200010EDB50D00FDF6E050EDF5C0B
:101A10001200DBCFEAFF14C0EEFF15C0EDFF12008D
:101A2000610EE9260D0EEA22EF6AE66A1200DF6A0D
:101A3000010EF36E020E12009AEC1FF0E55200093F
:101A400012003FC1E6FF40C1E6FF120014503D5DA9
:101A500015503E59120024EC21F0E552E5521200D7
:101A6000010EAEC1E7FFE7521200E76E060EE7CFA8
:101A7000DBFF1200EFCFDFFF010EDF521200030E7B
:101A8000DB5001019E151200E66E320EE66EE66A2C
:101A90001200BA0ED0EF92F0C60EE66E030EE66E9E
:101AA00012009EEC80F0020EDB6A1200020EDB5088
:101AB0000215120001010051DF5C1200DF1CE5522B
:101AC000E7141200E66AE66AE66A1200E66A360E73
:101AD000E66E1200DF507BEC93F0FCEC85F093ECAB
:101AE00093F0DF2A1200E66EE66AD8EF85F0F4EC98
:101AF00085F0EF50120049EC86F0D8EF85F0E66EE5
:101B0000E66AD4EF85F0F5EC93F0030EE66E120072
:101B100049EC86F0D4EF85F0EFEC85F0F350F4104B
:101B20001200070DEFEC85F0C70E1426020EFCEF35
:101B300085F0C3EC85F0020EE1261200D0EC92F0A5
:101B4000D8EF85F0D0EC92F0D4EF85F0DB507BEC51
:101B500093F0FCEF85F0F3EC92F0EE52EFCF14F03F
:101B60000EEC95F01414E66EF3EC92F0020EC7EC56
:101B700092F00EEC95F001010115E66EF3EC92F097
:101B80000BEC95F0F3EC92F0ECEF92F07FEC87F039
:101B9000900E1426000EFCEF85F0C3EC85F0E652A3
:101BA00012003EEC86F0FFEF85F03EEC86F0D8EFB9
:101BB00085F0E552E552E5521200C3EC85F0060EC1
:101BC000FDDC010F5BEC93F0E66AE4EF85F0DB509F
:101BD000CCEF85F0970EE66E050EE66E12000B0D4B
:101BE000EFEC85F068EF86F0DFCFE6FFB2EC93F024
:101BF000E3EC94F0E6EF86F072DCEFEC85F01CEF9E
:101C000086F0C3EC85F0030EE1261200146E050E7B
:101C1000E15E14501200FE0EDB50DCEF85F0FE0E8C
:101C2000DBCFE6FF1200190EE66E880EE66E060E9A
:101C3000E66E0E0E8FEF93F004EC95F0E66E120058
:101C40000CEC89F0020EC7EF92F0146E04EC87F0F2
:101C500035DF14105AEC86F0DBCFE6FF1200C3EC40
:101C600085F0F8EC94F0DBEF8BF0E8EC85F066EFB4
:101C700094F03EEC86F064EC86F0E552C8EF85F017
:101C80005DEC86F0080EF4EF85F0AAEC94F0E12606
:101C90001200010EDB50DCEF85F0010E11EC86F036
:101CA000EE521200F350DF6E2EEC86F0DF141200BD
:101CB000F35002EC89F003EC86F0040EDB50EF12D7
:101CC000C1EC88F00101015102110411E552E71441
:101CD000146E03EC86F0EE521450EF121200E3EC97
:101CE00094F00E0E1426000E1522010EE9EF93F06B
:101CF000F5EC93F0180EE66E12000AEC86F0020E78
:101D0000120086EC94F0E66EE40E3EEF86F0D0EC26
:101D100092F0E4EF85F0080E24EF86F0C1EC88F035
:101D2000E66A2BEC94F0E66A52EC87F0E66A04EC83
:101D300087F0E66A67EC8AF08851E66EE66A120080
:101D4000D9CF14F0DACF15F0080EDB500F01D924EB
:101D500007EC89F0EF50E66E080EAEEC86F0E55227
:101D6000E750EF6E120023EC94F0C2EC93F0880E73
:101D70001426060E120016C008F017C009F05EEC1B
:101D8000B8F002C014F003C015F004C016F005C08E
:101D900017F033EC94F002241200020E14C0DBFFA3
:101DA000030E15C0DBFF1200DBCFE6FF2EEC86F042
:101DB000E552E7141200EF51040DEFEC85F01CEF33
:101DC00086F0C3EC85F0050EE1261200DBCFF4FFB0
:101DD000F350F45C1200E96EDACFEAFF1200E0DBA8
:101DE00098EC6AF089EF87F029EC93F0010E12006D
:101DF000F5EC93F0DF6A1200C3EC85F0080EE126E3
:101E0000BAEC93F043EC87F057EF8AF0BDEC87F023
:101E1000010EDB500215D5EC86F0030EDB501200EC
:101E2000C3EC85F00101B251120049EC86F0FFEFDE
:101E300085F0E66EE66AFFEF85F0FE0E4EEC94F05C
:101E40000F01D5EC93F0EF50E66E1200280EE66E0F
:101E5000610EE66E010EE66EC5EF88F00BEC95F0B4
:101E600001EF94F0F1EC86F075EF94F0FC0EDBCF0F
:101E7000E6FFFDEF93F0C3EC85F090EC86F0ADEF5C
:101E800087F0030E146EE66E78EF86F0FE0EDB50E0
:101E9000CBEF86F00101005124EF86F0A80EE66E2C
:101EA000040EE66E1200FE0EDB50F6EF86F0146EA6
:101EB000070EE15E1450120042EC86F0EBEF89F061
:101EC000C3EC85F0F0EF8BF0E66EE66AB8EF86F0D3
:101ED000DF045AEF86F0FE0EDB50070DB1EC89F0FF
:101EE000B00E1626000EA7EC94F0DDEF8CF0F30E8A
:101EF000146E070E7615D0EC93F01450EF16A35124
:101F00001200F8EC85F0E4EC93F0D4EC8AF043ECAA
:101F100087F057EF8AF0B8EC87F0F9DBDF1C146E1E
:101F20002EEC86F0ABEF8BF0E8EC85F0050EF4ECD0
:101F300085F0020EEF6E120043EC87F0E66A94EC37
:101F40009CF089EF87F0E66EF0C0E6FF1AEC19F01E
:101F500089EF87F00AEC86F0EE52EF04120067EC8E
:101F60008AF0C2EF87F0B3C1E9FFB4C1EAFF120003
:101F700042EC86F0EF5012007FEC88F049C1EFFF91
:101F800086EC88F04BC1EFFF010EAEEF86F0300E0D
:101F9000DF5CF6EC86F0010EEFCFDBFF01010051B4
